:100000000C9433090C9490090C9490090C94900969
:100010000C9490090C9490090C9490090C949009FC
:100020000C9490090C94D91C0C9490090C94900990
:100030000C9454380C9490090C9490090C949009E9
:100040000C9490090C9490090C94F7180C94900956
:100050000C94970F0C9490090C94610F0C949009D8
:100060000C941F200C9490090C9479330C949009F3
:100070000C947C9A0C9490090C94CD8F0C9490095C
:100080000C9490090C9490090C94900948204D20F0
:1000900052205B20722089209920A920E42075231A
:1000A000892000221122412260227D22D722322380
:1000B000E525C6265C27DD271528C5288C29ED29CE
:1000C0005F2A9F2AF72A252B522BB72B022C4D2C67
:1000D000B12CAD2D9833CC330D347F349734D734D5
:1000E0009D35A136A136A136A136A136A136A1365D
:1000F000A136A136A136A136563658365D3675364C
:10010000773628721C73A173C872F57325746772F1
:10011000F772BE806281E78149829D820683848A6C
:100120008783B983B983B983B983B983B983B98321
:10013000B983B983E7836284F38418855B85B385CB
:1001400049865487BB87BB87BB87BB87BB87BB8779
:10015000BB87BB87BB87F387118836889288CE8898
:1001600032895F89FF89848A5F8A5F8A5F8A5F8AB2
:100170005F8A5F8A5F8A5F8A8B988E988E988E9846
:1001800097989A989D98AF98AC980A0D3D3D3D3D43
:100190003D3D3D3D3D3D3D3D3D3D3D3D3D3D3D3D8F
:1001A0003D3D3D3D3D3D3D3D3D3D3D3D3D3D3D00BC
:1001B0000A0D426174743A002025642043656C6C1A
:1001C000732000204C6F77207761726E696E673AFA
:1001D0002025642E25640020204175746F6C616EAB
:1001E00064696E673A2025642E2564000A0D466F07
:1001F000756E6420424C2D4374726C3A2000256465
:10020000000A0D0A0D2121204D495353494E472024
:10021000424C2D4354524C3A202564202121000A9F
:100220000D43616C6962726174696E6720707265FA
:1002300073737572652073656E736F722E2E004F27
:100240004B0A0D000A0D466C696768742D74696D60
:1002500065202575206D696E20546F74616C3A2598
:1002600075206D696E00416E676C654E69636B2029
:10027000202020202020416E676C65526F6C6C201E
:100280002020202020204163634E69636B202020C2
:10029000202020202020416363526F6C6C2020209E
:1002A0002020202020205961774779726F2020205C
:1002B000202020202020416C746974756465205BC7
:1002C000302E316D5D204163635A20202020202094
:1002D0002020202020204761732020202020202063
:1002E000202020202020436F6D70617373205661A1
:1002F0006C7565202020566F6C74616765205B30DB
:100300002E31565D20205265636569766572204CFA
:100310006576656C20204779726F20436F6D706140
:100320007373202020204D6F746F722031202020A5
:100330002020202020204D6F746F7220322020203A
:100340002020202020204D6F746F72203320202029
:100350002020202020204D6F746F72203420202018
:100360002020202020203136202020202020202066
:100370002020202020203137202020202020202055
:100380002020202020203138202020202020202044
:100390002020202020203139202020202020202033
:1003A000202020202020536572766F2020202020DE
:1003B000202020202020486F7665726761732020FE
:1003C00020202020202043757272656E74205B30DF
:1003D0002E31415D20204361706163697479205B37
:1003E0006D41685D202048656967687420536574B5
:1003F000706F696E7420323520202020202020204C
:1004000020202020202032362020202020202020C4
:10041000202020202020436F6D706173732053656E
:1004200074706F696E744932432D4572726F722019
:10043000202020202020424C204C696D697420200F
:100440002020202020204750535F4E69636B2020DE
:100450002020202020204750535F526F6C6C2020BA
:1004600020202020202021212120494E434F4D5083
:10047000415449424C4520212121002E000A0D20E3
:10048000444143206F7220493243204552524F521B
:100490002120436865636B204932432C2033567218
:1004A00065662C2044414320616E6420424C2D43FC
:1004B00074726C005B25695D005B25695D002B2013
:1004C0004D696B726F4B6F70746572202B004857CB
:1004D0003A5625642E25642053573A25642E25303C
:1004E00032642563200053657474696E673A25642D
:1004F000202573004D69786572204572726F7221F4
:10050000004552522532643A004861726477617244
:1005100065204572726F7220313A256420212100D6
:100520004D697373696E6720424C2D4374726C3A47
:10053000256420212100493243204552524F522147
:10054000212100424C2D53656C66746573742045FF
:1005500072723A253264004865696768743A2020EF
:1005600025356900536574706F696E743A25356975
:100570000050726573737572653A253569004F6670
:10058000667365743A2020253569002841290025C5
:1005900069006163742E2062656172696E67004E46
:1005A00069636B3A20202020202025356900526F96
:1005B0006C6C3A20202020202025356900436F6D87
:1005C000706173733A202020253569004B25693A04
:1005D00025346920204B25693A25346920004E696D
:1005E0003A2534692020526F3A2534692000477338
:1005F0003A253469202047693A2534692000503172
:100600003A253469202050323A253469200050338D
:100610003A253469202050343A253469200047793E
:10062000726F202D2053656E736F72004E69636B7D
:100630002025346920282533692E25782900526F1A
:100640006C6C2025346920282533692E25782900F3
:1006500059617720202534692028253369290041F4
:100660004343202D2053656E736F72004E69636B98
:100670002025346920282533692900526F6C6C20AD
:10068000253469202825336929005A202020202577
:10069000346920282533692900566F6C74616765B9
:1006A0003A2020202533692E253169560043757282
:1006B00072656E743A2020202533692E25316941F8
:1006C00000506F7765723A2020202020253469572A
:1006D000004469736368617267653A202535696D06
:1006E00041680052656365697665720052432D5119
:1006F00075616C6974793A202534690052432D4341
:1007000068616E6E656C733A25346900436F6D7075
:10071000617373004D61676E65743A202020253542
:1007200069004779726F3A20202020202535690022
:10073000536574706F696E743A2025356900506F87
:10074000746925693A202025336900506F74692542
:10075000693A202025336900536572766F202000A6
:10076000536574706F696E74202025336900506F73
:10077000736974696F6E3A202533690052616E6740
:10078000653A2533692D25336900424C2D43747237
:100790006C204572726F72732000253364202533FC
:1007A0006420253364202533642000424C205465A6
:1007B0006D70657261747572650025336420253330
:1007C0006420253364202533642000424C20437587
:1007D0007272656E740028696E20302E31412900D6
:1007E0002533642025336420253364202533642099
:1007F00000424C2D4374726C20666F756E6420004D
:100800002025632020202563202020256320202010
:10081000256320002025632020202563202020251B
:1008200063202020256320002025632020202D2008
:1008300020202D2020202D200031300031310031AA
:100840003200466C696768742D54696D652020001C
:10085000546F74616C3A2535756D696E004163742F
:100860003A20202535756D696E00287265736574B0
:1008700029000A0D2D2D3E20486172647761726552
:100880002056657273696F6E2042797465204368E3
:10089000616E676564203C2D2D000A0D47656E650D
:1008A000726174696E672064656661756C7420504E
:1008B0006172616D657465722053657420256400F2
:1008C0000A0D5573696E6720506172616D657465BC
:1008D0007220536574202564000A0D47656E6572A9
:1008E0006174696E672064656661756C74204D691A
:1008F000786572205461626C65000A0D4D697865F7
:10090000722D436F6E6669673A202725732720286A
:100910002575204D6F746F727329000A0D41434392
:10092000206E6F742063616C69627261746564210A
:100930000D0A0000008F001E01AD013B02CA0258E3
:1009400003E603740402058F051B06A7063307BEE2
:10095000074808D2085B09E3096B0AF20A780BFD25
:100960000B810C040D860D070E870E060F840F00F9
:10097000107B10F5106E11E5115B12CF124213B30C
:100980001323149214FE146A15D3153B16A11605F1
:10099000176717C81727188318DE1837198E19E339
:1009A00019361A871AD61A231B6E1BB61BFD1B415C
:1009B0001C831CC31C001D3C1D751DAB1DE01D12BE
:1009C0001E421E6F1E9A1EC31EE91E0D1F2E1F4DB6
:1009D0001F691F841F9B1FB01FC31FD31FE11FEC84
:1009E0001FF51FFB1FFF1F0020000005000500046E
:1009F00001060108000601020004000400070007C8
:100A000000070007000700070007000301030105B6
:100A10000017010F01060009010A0119010501056E
:100A20000119011A010F01010009004E6F204572E2
:100A3000726F722020202020202020004E6F742012
:100A4000636F6D70617469626C652020004D4B337B
:100A50004D6167206E6F7420636F6D7061004E6F23
:100A600020464320636F6D6D756E6963617400434A
:100A70006F6D7061737320636F6D6D756E69630068
:100A800047505320636F6D6D756E69636174696F54
:100A900000636F6D706173732076616C75652020E3
:100AA00020005243205369676E616C206C6F737431
:100AB000202000464320737069207278206572728E
:100AC0006F7220004E6F204E4320636F6D6D756E08
:100AD00069636174004643204E69636B20477972F5
:100AE0006F2020202000464320526F6C6C204779F5
:100AF000726F2020202000464320596177204779DB
:100B0000726F2020202020004643204E69636B2016
:100B1000414343202020202000464320526F6C6C2C
:100B2000204143432020202020004643205A2D41CD
:100B30004343202020202020202000507265737322
:100B40007572652073656E736F72200049324320A1
:100B500046432D3E424C2D4374726C2000426C2063
:100B60004D697373696E67202020202020004D6935
:100B7000786572204572726F722020202020004319
:100B800061726566726565204572726F7220200021
:100B900047505320466978206C6F737420202020C2
:100BA000004D61676E6574204572726F722020205F
:100BB00020004D6F746F72207265737461727420BF
:100BC000202000424C204C696D69746174696F6E1D
:100BD000202020004750532052616E67652020205E
:100BE00020202020004E6F2053442D43617264204A
:100BF00020202020200053442D4C6F6767696E67CA
:100C0000206572726F7200466C79696E672072613E
:100C10006E676521202020004D617820416C746949
:100C20007475646521202020004E6F2047505320AA
:100C300066697820202020202000636F6D7061732A
:100C400073206E6F742063616C2E00424C2D5365CF
:100C50006C66746573742020202020005365742016
:100C6000203A002021212020204C414E44494E476B
:100C7000202020202121202000202121204C6950EB
:100C80006F20766F6C746167652021212020002021
:100C9000202020204D696B726F4B6F70746572203D
:100CA0002020202000202020202020202020202064
:100CB00020202020202020202020002020253269F4
:100CC0002E2531695620200020202532692E25311D
:100CD0006956202000414C543A2534696D20256323
:100CE00000414C543A2534696D202000414C543A5F
:100CF0002D2D2D2D200020202532693A25303269F6
:100D000020200020202532693A2530326920200039
:100D10004449523A202533642563004300200020D3
:100D20002025356920200020202535692020004914
:100D30003A2532692E2531694120003A003A003ABD
:100D4000002D2D2D2D2D2D2D2D2D2B2D2D2D2D2D02
:100D50002D2D2D2D2D2D002D2D2D2D2D2D2D2D2DF0
:100D60002D2D2D2D2D2D2D2D2D2D2D2D003A0053DA
:100D700041543A2532642000444953543A2533649F
:100D80006D004420003344002121004D41473A25A5
:100D9000337525252000484D3A25336425632025E9
:100DA0006300696E636C3A253264256328253269D5
:100DB0002900202020202532756D2F733A202048ED
:100DC0004D3A2533642563202563004552523A206D
:100DD0002532642021004552523A20002121204C26
:100DE00069506F20766F6C74616765202121002047
:100DF0007777772E4D696B726F4B6F707465722EBB
:100E00006465202000202532693A2530326920208F
:100E10002532692E25316956202534696D416800D7
:100E2000202532693A2530326920202532692E2565
:100E3000316956202534696D4168004449523A258C
:100E40003364256300414C543A2534696D00414CAC
:100E5000543A2534696D00414C543A2D2D2D2D20E6
:100E600000256300484D3A2533642563202044491A
:100E700053543A2533646D202563005057523A2568
:100E800032692E25316941202825695729200043E0
:100E900046002020004750533A2532756D2F7320AD
:100EA0005341543A256420002020334420004E4F03
:100EB000464958004447505320002020204E6F20C0
:100EC0004E6176694374726C20202020202020001F
:100ED0002532692E2569202532692E256920253283
:100EE000692E2569202532692E256941002533693F
:100EF0002025336920253369202533692563430084
:100F00002532692E2569202532692E256941002563
:100F100032692E2569202532692E256920253269FE
:100F20002E2569202532692E256941002533692047
:100F30002533692563432020202020202020002500
:100F400033692025336920253369202533692563DA
:100F500043004552523A2025326420210045525226
:100F60003A20002121204C69506F20766F6C74610B
:100F7000676520212100207777772E4D696B726F8E
:100F80004B6F707465722E64652020005365747415
:100F9000696E673A257520257320004D696E3A25E4
:100FA00032692E253169562025732000414C543A70
:100FB00000504F54493A2533752000284F4E2920C0
:100FC0002000284F46462920004C494D49540056E0
:100FD0004152494F0044495341424C454400434625
:100FE0003A0044495341424C45440020284F4E2981
:100FF000200020284F464629002054454143480000
:101000004750533A0044495341424C454400284616
:10101000524545290028484F4D452900284149445B
:1010200029200028484F4C4429002046533A257572
:1010300073656B2000484F4D4520414C543A0025C4
:10104000756D00484F4C4420004E693A25346920A4
:10105000526F3A25346920433A2533690047733A81
:101060002534692059613A253469200050313A25E8
:1010700034692050323A25346920333A25336900E7
:1010800050343A2534692050353A25346920363AAF
:1010900025336900434F55504C494E47204F464633
:1010A0002120004C4F4F50494E47212000484821F5
:1010B0002000434F4D50415353204F4646212000BE
:1010C000004F505152535453565748005859005AE4
:1010D0005545464748410049424A4A000000000041
:1010E000000000000000444C4D00000000004E00D5
:1010F00000004B00430A0D7777772E4D696B726FB6
:101100004B6F707465722E646520286329204869CE
:1011100053797374656D7320476D6248000A0D74CE
:10112000686520757365206F662074686973207325
:101130006F667477617265206973206F6E6C7920B9
:101140007065726D6974746564200A0D6F6E206F2E
:10115000726967696E616C204D696B726F4B6F705D
:101160007465722D486172647761726500557365AC
:101170007200486F54542056340041435420445365
:101180004C004A657469005370656B7472756D002C
:1011900050504D000A0D52656365697665723A20BC
:1011A00000532E42757300756E6B6E6F776E2E2036
:1011B0005573696E672050504D2E2E2E006E6F7441
:1011C00020737570706F7274656420627920686135
:1011D00072647761726521000A0D202D204C49420E
:1011E000204E4F5420434F4D50415449424C4520CE
:1011F00021212121000A0D0A0D212120426F6F7447
:101200006C6F61646572206E6F7420636F6D7061C6
:101210007469626C6520746F2048617264776172D2
:1012200065203E20322E322021210A0D0A0D000AAF
:101230000D466C69676874436F6E74726F6C0A0D4B
:1012400048617264776172653A25642E25640A0DDF
:10125000536F6674776172653A5625642E25303275
:1012600064256320000011241FBECFEFD0E4DEBF51
:10127000CDBF12E0A0E0B1E0EAEDFAE301E00BBF80
:1012800002C007900D92A63EB107D9F71CE0A6EE6A
:10129000B2E001C01D92AE3BB107E1F77AEAE2E0AD
:1012A000F0E081E280935700D4907E010894E11C25
:1012B000F11C20EF37EF41E050E087016FE0DA01E9
:1012C000C9012F5F3F4F4F4F5F4FABBFFC0187916D
:1012D000F80181938F01615067FFF1CF84EE8ABDE1
:1012E000898580936905893138F086E080931401FF
:1012F00087E0809313017BEAF7016EE08191782704
:101300007095615067FFFACF8889781729F0F7E95F
:10131000DF1611F40000FECF0E94790A0C946C9D38
:101320000C9400008AE891E09F938F938DE096E102
:101330009F938F93E0919805F091990509950F90EF
:101340000F900F900F90089580913D08E82FFF2790
:10135000EE0FFF1FEC58F64F808191818D5E9F4FFD
:1013600014F010920401808191818A5B9F4FCCF42C
:10137000809104018823A9F481E080930401809185
:10138000CC058F5F8093CC05853038F088EE93E0F4
:1013900090931C0380931B03089566E970E00E94FC
:1013A0009A3B0895CF93DF93C82F882389F080EB71
:1013B00091E09F938F938DE096E19F938F93E091BF
:1013C0009805F091990509950F900F900F900F9047
:1013D00080912601909127016BE270E00E94DF9CD2
:1013E000962F9F5F9093000180916008823318F5DB
:1013F000989F802D112480930201CC23F1F068EC9A
:1014000070E0892F0E949A3B8091000199279F9359
:101410008F9388EB91E09F938F938DE096E19F935C
:101420008F93E0919805F091990509958DB79EB736
:1014300006968DBF02C0809302019091AB08923353
:1014400038F480910001899F802D11248093AB088E
:101450008091AB0890910201981720F491509093DD
:10146000AB089F5FCC2309F441C0892F6AE00E943A
:10147000BF9C892F99279F938F93809102010E948F
:10148000BF9C99279F938F9383EC91E09F938F93B9
:10149000CDE0D6E1DF93CF93E0919805F0919905E7
:1014A00009958DB79EB708968DBF8091AB088823AC
:1014B000E9F06AE00E94BF9C892F99279F938F9340
:1014C0008091AB080E94BF9C99279F938F9387EDD3
:1014D00091E09F938F93DF93CF93E0919805F091E4
:1014E000990509958DB79EB708968DBFDF91CF916D
:1014F0000895CFEFD0E4DEBFCDBF88249924C1E0AA
:101500007C2E14B815B88AE08AB98FE58BB9B7EE8E
:10151000CB2EB3E0DB2E2EEC3FEFC20ED31ED7FE58
:10152000FACF6624199B08C04C9B04C085E18093C8
:10153000030108C086E101C089E18093030181E0D5
:101540008093060481E887B93E9A8FEF88B98BE1D2
:1015500084B981E085B9469A84B7877F84BF80913A
:1015600060008861809360001092600084EC99E0D4
:1015700090931C0380931B03109254041092530405
:10158000109279091092780910925604109255041D
:10159000109258041092570420910301243128F02E
:1015A00084EC94E0A0E0B0E004C08BE095E0A0E023
:1015B000B0E08093420190934301A0934401B09323
:1015C00045012A3011F0243110F0289801C0289AE2
:1015D0002C3010F0293111F4299A01C029980E9469
:1015E000481A0E94191A0E9415160E941B380E9460
:1015F0005A1E81E00E942D330E94CE700E94937A81
:1016000085E00E940399809103018C3010F08931AC
:1016100011F4299A01C0299878940E94143280917B
:10162000680382608093680310926B030E94A7474F
:1016300084EF91E00E94DF196C018091680380FDC6
:1016400005C0C6010E94E8198823B9F38CEE91E029
:101650009F938F93ADE0AA2EA6E1BA2EBF92AF92D0
:10166000E0919805F0919905099580EA9FE00E9424
:10167000DF196C01C0E0D0E00F900F900F900F9039
:1016800006E119E0FAECEF2EF8E0FF2E0E94A747E2
:101690008091680380FD05C0C6010E94E819882377
:1016A000B9F3F70180811816ACF40BC00E94A7476C
:1016B0008091680380FD05C0C6010E94E819882357
:1016C000B9F3C6010E94E819882321F4F80180814A
:1016D000882364F7F801808187FF19C02196DF9382
:1016E000CF9321978EEF91E09F938F93BF92AF920C
:1016F000E0919805F091990509958091E7028F5F37
:101700008093E7022DB73EB72A5F3F4F2DBF21964A
:1017100084E090E0E80EF91E085F1F4FCC30D10541
:1017200008F4B4CFC0E0D0E003E119E0EAECEE2E1B
:10173000E8E0FE2EF801838187FD1DC0F70180815E
:101740001816CCF42196DF93CF93219781E092E095
:101750009F938F938DE096E19F938F93E0919805EF
:10176000F0919905099582E0809319032DB73EB752
:101770002A5F3F4F2DBFF8018381807883832196B4
:1017800024E030E0E20EF31E085F1F4FCC30D1059D
:1017900088F20E94920990913B088091E702981785
:1017A00028F48091B20580618093B2058FE192E0C8
:1017B0009F938F93CDE0D6E1DF93CF93E09198058F
:1017C000F0919905099588EE93E00E94DF196C016C
:1017D0000E94981E0F900F900F900F90C6010E94CC
:1017E000E8198823D9F38FE392E09F938F93DF93D7
:1017F000CF93E0919805F0919905099580E00E94BA
:101800007E3C809103010F900F900F900F908A30D3
:1018100011F0843110F0289801C0289A80ED97E0EB
:1018200090931C0380931B0385E58093CE058EE087
:1018300090E00E9434309927182F00278FE090E025
:101840000E943430080F111D1093ED020093EC023A
:101850008AE090E00E9434309927182F00278BE00F
:1018600090E00E943430080F111D1093EB0200939A
:10187000EA020F5F1F4F39F08091EC029091ED0268
:101880008F5F9F4F41F41092ED021092EC02109284
:10189000EB021092EA028091EA029091EB029F9390
:1018A0008F938091EC029091ED029F938F9384E44B
:1018B00092E09F938F93DF93CF93E0919805F091FF
:1018C000990509950E945D2588E893E190933D0173
:1018D00080933C01C1E0C093CD058C2F0E94D209BA
:1018E000809163080E944F980E94920980ED97E0D2
:1018F0000E94DF196C018AEF90E00E94DF1983E0FB
:10190000809395071092E6028091AE082DB73EB7FE
:10191000285F3F4F2DBF84FF02C0C093EE0212BC70
:1019200011BC8091F002882311F04798FECF80917E
:101930001F03882309F4B4C280911801882309F495
:10194000AFC2F89480911F03815080931F03789455
:101950008091CC05882319F00E94A40902C00E943E
:101960002E4B0E94A747209103012A3011F0243109
:1019700010F0289801C0289A80914704882331F0FC
:10198000809147048150809347040EC080916F007E
:10199000806280936F001092750910927409809193
:1019A000B20588608093B20580913C0190913D0121
:1019B000019790933D0180933C0180913C0190916F
:1019C0003D01892B21F0809169038823C9F1809121
:1019D0003C0190913D01892BD9F40E94573385E059
:1019E00090E090933D0180933C018091CF079091CE
:1019F000D00701969093D0078093CF078091B205CE
:101A000081608093B20580919607826080939607EB
:101A100080910B0190910C018F5F9F4FC1F48091D9
:101A200046048823A1F088EA91E690931C038093F2
:101A30001B0380E890E090930C0180930B0107C09A
:101A40002A3011F0243110F0289801C0289A0E9401
:101A5000FF9980911F03882309F020C280916405BB
:101A6000882319F00E94048B19C280911A038823DD
:101A700011F40E94EF7080911101882311F00E94EF
:101A8000A21A0E945F160E94EC11C6010E94E8197A
:101A9000882309F4FFC184E190E0C80ED91E0E949A
:101AA000601A80916308863019F40E94828004C015
:101AB000843011F40E94D48B80910604882331F184
:101AC0008091DC079091DD078C52914074F08091F9
:101AD000A5079091A60780509240C4F48091DC073E
:101AE0009091DD07835593408CF0639432E3361573
:101AF00070F480914604882331F08091B1058062B2
:101B00008093B10504C08093320401C066248091A3
:101B10006903882329F48091F80A8E3150F405C0B6
:101B20008091B20582608093B205809196078260B1
:101B30000FC080911B0390911C03892B59F4809155
:101B40003C0190913D01079728F0809196078D7F89
:101B5000809396078091EE02882361F0809147047C
:101B6000873940F01092EE0288E893E190931C03CD
:101B700080931B0380910601882321F0815080937C
:101B800006012EC08093D80510921A0410921904F1
:101B90001092180410921704109216041092150453
:101BA000809147048823E1F480910B0190910C010E
:101BB0008F5F9F4FA9F42091EE02223089F088E9CF
:101BC0009AE390931C0380931B0380E09CE0909326
:101BD0000C0180930B01222319F082E08093EE0226
:101BE0008091A401893C70F081508093A401809180
:101BF000B2058B7F8093B2058091B505816080939B
:101C0000B50551C080917A0A8823F9F08091B20518
:101C100084608093B20589E08093280580910B0150
:101C200090910C018F5F9F4F81F48091460488232F
:101C300061F088E99AE390931C0380931B0380E092
:101C400098EA90930C0180930B0110921A05109260
:101C5000190510921805109217051092160510928A
:101C60006D0A8FEF8093E20A1092AC0A1092AB0AD1
:101C70001092AE0A1092AD0A8FEF9FEF9093AA0ACE
:101C80008093A90A109236041092370410923804F7
:101C90001092390410923A048091B5058E7F80939A
:101CA000B5051092A40160910201262F332780917F
:101CB00026019091270128173907F4F080910E042E
:101CC000806280930E0480910B0190910C018F5FD4
:101CD0009F4F91F480912601909127010B9764F01A
:101CE00080E797E190931C0380931B0380E093E0CF
:101CF00090930C0180930B0112BC11BC8091EF02F8
:101D00008F5F8093EF02813309F07BC01092EF0266
:101D100080914E05882319F0815080934E05809163
:101D20000E0481FF0AC08091E8029091E9020196B9
:101D30009093E9028093E80204C05AEA852E55E0A8
:101D4000952E80910F04909110048050944008F0DB
:101D500049C02091DE073091DF074091E0075091A4
:101D6000E10780911E0190911F01A0912001B09187
:101D70002101281739074A075B0764F48091DE07C1
:101D80009091DF07A091E007B091E1070596A11DB2
:101D9000B11D20C02091DE073091DF074091E007A0
:101DA0005091E10780911E0190911F01A0912001A7
:101DB000B091210182179307A407B5079CF4809185
:101DC000DE079091DF07A091E007B091E10705974A
:101DD000A109B1098093DE079093DF07A093E00784
:101DE000B093E107862F9927019620912601309123
:101DF0002701821793072CF480910E048F7D809326
:101E00000E040894811C911C82E788168BE09806CA
:101E100009F040C0882499242091EC023091ED0211
:101E20002F5F3F4F3093ED022093EC028091EA0246
:101E30009091EB0201969093EB028093EA02832F3C
:101E40009927682F8EE090E00E943C308091EC0250
:101E50009091ED029070682F8FE090E00E943C30EE
:101E60008091EA029091EB02892F9927682F8AE0EE
:101E700090E00E943C308091EA029091EB029070D9
:101E8000682F8BE090E00E943C3084E190E00E945B
:101E9000DF196C010E941C760E94CB7A71107A9433
:101EA000772039F40E94E075882319F08CE0782EB1
:101EB00038CD80911A03882309F033CD0E94EF704A
:101EC00030CD1F920F920FB60F9211248F939F93D4
:101ED000EF93FF93809108018823E1F480910A0336
:101EE00090910B03019690930B0380930A03FC01DE
:101EF000E754F94FE081ED3019F08C3D910539F44C
:101F000010920B0310920A0381E080930801E09382
:101F1000C60004C010920B0310920A03FF91EF91C8
:101F20009F918F910F900FBE0F901F9018951F9249
:101F30000F920FB60F9211242F933F934F935F93FD
:101F40006F937F938F939F93AF93BF93CF93EF93B1
:101F5000FF9390E08091F002813029F48091C600D7
:101F60008093CE00D1C08091F002823029F480911C
:101F7000C6008093DB05C8C08091C6008093020331
:101F8000509110035C3D10F0909311038091020377
:101F90008D3009F06AC080911103823009F065C06C
:101FA00090931103852F992785529A4FFC01329700
:101FB000408120910C0330910D03241B3109DC0179
:101FC00011978C91281B3109C9019F7090930D03C3
:101FD00080930C0346E0969587954A95E1F7982FF4
:101FE000935C90930E032F733070235C20930F0348
:101FF0008081981729F48C91281711F491E006C07C
:1020000090E08091FF028F5F8093FF028091010337
:10201000882309F079C0992309F476C081E0809380
:102020000103580F5093FE025150E52FFF27E55250
:10203000FA4F8DE080838091DD05823509F064C020
:10204000C0914604CC2309F05FC00E945D2588E161
:1020500090E02CE00FB6F894A895809360000FBE36
:1020600020936000C09319034FC020911103822F69
:10207000992781309105F9F0823091051CF4892B64
:1020800021F040C0029711F13DC0809102038332DC
:1020900039F480910103882319F481E080931103BE
:1020A000809102038093DB0581E08093100380918F
:1020B0000203992722C02F5F20931103E52FFF27EA
:1020C000E552FA4F80910203808309C0E52FFF2774
:1020D000E552FA4F8091020380835C3D20F45F5FFC
:1020E0005093100302C010921103209102038091BB
:1020F0000C0390910D03820F911D90930D0380931B
:102100000C0302C010921103FF91EF91CF91BF9188
:10211000AF919F918F917F916F915F914F913F917F
:102120002F910F900FBE0F901F901895AC01A0E05B
:10213000B0E09D01A817B90748F4E9EBF6E08191FA
:10214000280F311D1196A417B507C8F33F70FD0184
:10215000E754F94FC90156E0969587955A95E1F7EE
:10216000835C80831196FD01E754F94F2F73307023
:10217000822F835C8083A654B94F8DE08C9310929C
:1021800008018091B9068093C6000895A0E0B0E0F0
:10219000ECECF0E10C94389D2C859D850E85BB24DC
:1021A00083E28093B9069F599093BA062093BB06A9
:1021B00033E0E32EF12C002309F49EC0CF84D888AD
:1021C000BE016D5E7F4FA989BA890150109709F44D
:1021D00093C01097B9F0F601EB0DF11DB394908107
:1021E000119791F4002349F1FB016E5F7F4FDB01F2
:1021F000C080D1806E5F7F4F0D90BC91A02DBB241D
:10220000015002C090E019C01097B9F0F601EB0D33
:10221000F11DB3944081119791F4002341F1FB012A
:102220006E5F7F4FDB01C080D1806E5F7F4F0D906E
:10223000BC91A02DBB24015002C040E018C01097F3
:10224000B1F0F601EB0DF11DB3941081119781F4FB
:10225000002371F0FB013296DB01CD90DC90BF01D1
:102260006E5F7F4FA081B181BB24015001C010E09F
:10227000F701E754F94F892F86958695835C808313
:102280000894E11CF11CF701E754F94F892F9927B5
:102290008370907024E0880F991F2A95E1F75527E5
:1022A0009A0194E0369527959A95E1F7822B835C05
:1022B00080830894E11CF11CF701E754F94F4F703B
:1022C0005070440F551F440F551F812F992726E04A
:1022D000969587952A95E1F7842B835C80830894F3
:1022E000E11CF11CF701E754F94F1F73135C1083D5
:1022F0000894E11CF11C6ACFC7010E949610E9E026
:102300000C94549DA3E07A2F4091FE024650442342
:1023100009F458C0E72FFF27E552FA4F80818D530B
:102320007F5FE72FFF27E552FA4F20812D537F5F14
:10233000E72FFF27E552FA4F30813D537F5FE72FAC
:10234000FF27E552FA4F60816D537F5F9927880F11
:10235000991F880F991F522F52955F70582B822F0B
:1023600099278F709070F4E0880F991FFA95E1F724
:10237000232F26952695282B832F992783709070DD
:10238000E6E0880F991FEA95E1F7682B41504F3F2F
:10239000C9F0EA2FFF27E552FA4F5083AF5F415053
:1023A0004F3F81F0EA2FFF27E552FA4F2083AF5FBE
:1023B00041504F3F39F0EA2FFF27E552FA4F608333
:1023C000AF5FA5CF8EED95E09093FD028093FC0268
:1023D000A350A093FB020895A2E0B0E0E2EFF1E188
:1023E0000C943E9D80910103882309F412C40E943D
:1023F00082118091DC05823609F0DEC28091DD0514
:1024000099278037910509F4AFC081379105C4F44D
:102410008A36910509F43BC28B36910544F48B341E
:10242000910571F18636910509F464C1C5C28D36F6
:10243000910509F469C08E36910509F44DC0BCC2FE
:102440008437910541F1853791054CF48137910529
:1024500009F491C08337910509F4E4C0ADC2873710
:10246000910509F4D6C1883791052CF4853791057B
:1024700009F492C1A1C28937910509F477C19CC2C0
:10248000E091FC02F091FD02808191819093910195
:102490008093900191C28091FE02A091FC02B091C4
:1024A000FD02853140F080E1E6EBF5E00D90019210
:1024B0008A95E1F70DC08D919D910D90BC91A02D55
:1024C0008093B6059093B705A093B805B093B9056E
:1024D00080EF8093F9024BC0809108018823E1F3DB
:1024E0008DE490E09F938F938DEB98E09F938F9373
:1024F00081E08F938F938EE48F930E94C6108DB7E7
:102500009EB707968DBF58C2A091FC02B091FD0204
:102510001C91113081F48DE4EDEBF8E00D90019207
:102520008A95E1F70E944F3119838091B2058F7E21
:102530008093B20501C01982809108018823E1F3DC
:1025400081E090E09F938F93CE0101969F938F93AC
:1025500081E08F938F938DE48F930E94C610ADB767
:10256000BEB71796ADBF28C281E0809304038FEFFA
:102570008093060121C280914604882309F01CC281
:10258000E091FC02F091FD02E0818E2F8A508A30AA
:1025900058F48983882311F481E003C0863010F059
:1025A00085E0898361E00EC08E2F84518A3070F4FB
:1025B0008983882311F481E003C0863010F085E020
:1025C000898360E089810E94D13112C0E983EF3FA5
:1025D00019F40E94B23189838981882311F481E042
:1025E00003C0863010F085E0898389810E945230D3
:1025F000809108018823E1F380E890E09F938F9316
:102600008CE398E09F938F9381E090E09F938F936A
:10261000CE0101969F938F9382E08F9381E08F93F9
:1026200081E52DC12091FC023091FD02D9018C91F0
:102630008150853008F045C0F9018181813609F06B
:1026400040C0809146048823E1F52F5F3F4F80E82A
:10265000ECE3F8E0D9010D9001928A95E1F7F901D8
:1026600082910E94BF3080917D089927AA27BB27BD
:10267000BC01CD0124EC39E040E050E00E94A09C78
:10268000DC01CB018093880190938901A0938A019A
:10269000B0938B0180917E089927AA27BB27BC01A4
:1026A000CD010E94A09CDC01CB018093840190931A
:1026B0008501A0938601B09387010E94B23189837E
:1026C00001C01982809108018823E1F381E090E044
:1026D0009F938F93CE0101969F938F9381E08F9369
:1026E0008F9383E58F930E94C6108DB79EB7079690
:1026F0008DBF2BC080914604882309F05DC1E09115
:10270000FC02F091FD02E0818E2F8150853018F49B
:102710008E2F0E9452300E94B2318983809108012D
:102720008823E1F381E090E09F938F93CE0101969F
:102730009F938F9381E08F938F9386E48F930E9472
:10274000C610ADB7BEB71796ADBF109146041123A2
:1027500041F46EE670E089810E949A3B812F0E94CD
:10276000D209809163080E944F9826C1198229815D
:10277000A091FC02B091FD02E4E7F9E08D91992768
:1027800087FD909593A382A3822F8F5F8983282F43
:1027900032968C3098F310C1E091FC02F091FD026A
:1027A00080810E9471378A83882319F481E08983AC
:1027B00001C01982809108018823E1F388E090E04C
:1027C0009F938F938BE099E09F938F9321E030E06C
:1027D0003F932F938091FC029091FD029F938F93E2
:1027E0003F932F93CE0102969F938F933F932F9306
:1027F000CE01820F931F9F938F9384E08F9381E08C
:102800008F9385E58F930E94C610EDB7FEB7739640
:102810003CC08091FB02893008F4CEC02091FC02BC
:102820003091FD022F5F3F4F88E0ABE0B9E0F90146
:1028300001900D928A95E1F7D9018E910E94C436DC
:102840008A83882319F481E0898301C019828091E9
:1028500008018823E1F321E030E03F932F93CE017C
:1028600002969F938F933F932F93CE01820F931FD6
:102870009F938F9382E08F9381E08F9387E58F936F
:102880000E94C610EDB7FEB73B96EDBF95C0809194
:102890004604882309F090C00E94069889838230FC
:1028A00019F0843009F088C020E430E0F894809179
:1028B000C1008F738093C1008091C9008F73809392
:1028C000C9008091C100877E8093C1008091C900BA
:1028D000877E8093C9008091C80087FF03C08091E4
:1028E000CE00F9CF8091C00087FF03C08091C60061
:1028F000F9CFE091FC02F091FD02E081E13021F49A
:1029000082E08093F0022EC0E43611F421E830E03A
:1029100081E08093F002832F99278093CD0020934C
:10292000CC008091CD008093C5008091CC00809335
:10293000C4008091CA008F7D8093CA008091CA0034
:102940008F7E8093CA008091C9008B7F8093C900DD
:102950008091CA0084608093CA008091CA0082601E
:102960008093CA008091CA00877F8093CA008091BB
:10297000C200877F8093C2008091C9008E7F8093C0
:10298000C9008091C10088618093C1008091C90015
:1029900088618093C9008091C10080688093C100E4
:1029A0008091C90080688093C90010926E001092D7
:1029B0006F001092700078948091DD05992784361D
:1029C000910509F4BBC085369105ACF481369105BB
:1029D00009F46FC0823691052CF48B34910509F40B
:1029E0005DC00FC18236910509F470C08336910530
:1029F00009F47FC006C18C36910509F4EDC08D360F
:102A000091054CF48736910509F4F8C08836910594
:102A100009F4B2C0F6C08437910529F086379105D4
:102A200009F4E8C0EEC08091FE02A091FC02B091D2
:102A3000FD02803140F080E1E6EBF5E00D9001927F
:102A40008A95E1F70DC08D919D910D90BC91A02DBF
:102A50008093B6059093B705A093B805B093B905D8
:102A6000809108018823E1F31F92809105018F93E3
:102A700084E58F930E94C6108AEF8093F9028FEF4E
:102A80008093060180EA9FE00E94DF199093F20292
:102A90008093F1020F900F900F90B3C0E091FC0271
:102AA000F091FD028081918190939101809390013A
:102AB000A8C0E091FC02F091FD02808180930701A3
:102AC000803298F08FE1809307010FC0A091FC0243
:102AD000B091FD028BE0EEECF5E00D9001928A954D
:102AE000E1F78091D7058093D7078FEF8093060198
:102AF00088C08091F5029091F602892B89F4E091CB
:102B0000FC02F091FD02E081EE2351F08AE0E89FA3
:102B1000C00111240E94DF199093A9058093A80594
:102B2000E091FC02F091FD0290818AE0989FC00143
:102B300011249093F6028093F50215C08FEF8093D5
:102B40000601E091FC02F091FD0290818AE0989FDD
:102B5000C00111249093F8028093F702892B19F099
:102B600081E08093060380EA9FE00E94DF19909342
:102B7000F2028093F10245C08FEF80930601E0914D
:102B8000FC02F091FD02908197FD08C082E08093E5
:102B900003031092F4021092F3021AC090958091F0
:102BA0006103892B8093610391818AE0989FC00122
:102BB00011249093F4028093F30284E08093030342
:102BC00080EA9FE00E94DF199093F2028093F10265
:102BD00081E08093070315C08FEF80930601E09199
:102BE000FC02F091FD0280818093620381E080937A
:102BF000080307C081E08093050303C081E0809350
:102C00000903109201031092FD021092FC0210922F
:102C1000FB02E3E0CE5F0C945A9D982F8091C00098
:102C200085FFFCCF9093C60008950F931F9388E112
:102C30008093C1008091C00082608093C000809129
:102C4000C10080688093C1008091C100806480933E
:102C5000C10000E010E00093C5008AE290E080939C
:102C6000C4008091F7029091F8020E94DF199093BE
:102C7000AB058093AA058CED90E00E94DF1990933C
:102C8000DA058093D90582E08093AC058093AD0589
:102C900081E08093B0058BE08093AE051092AF0584
:102CA0001092B405809103018093B3051093FD0247
:102CB0000093FC021092FB021F910F910895A0E176
:102CC000B0E0E5E6F6E10C943D9D80910801882393
:102CD00009F489C28091F1029091F2020E94E819F0
:102CE000882361F01092F4021092F3021092F8021D
:102CF0001092F7021092F6021092F5028091F30200
:102D00009091F402892B41F08091B7069091B8061A
:102D10000E94E819882329F480910703882309F485
:102D200060C080910801882309F45BC0809103038F
:102D30000BEE17E08430A8F00E94732580E590E048
:102D40009F938F931F930F9381E08F938F9388E4CA
:102D50008F930E94C6102DB73EB7295F3F4F2DBFFE
:102D600034C01092630386E694E09F938F9386E6C7
:102D700095E29F938F93E0919805F09199050995BD
:102D800084E190E09F938F931F930F9381E090E0F5
:102D90009F938F9383E093E09F938F9382E08F9331
:102DA00081E08F9388E48F930E94C6108091030383
:102DB000982F8F5F809303032DB73EB7215F3F4F5E
:102DC0002DBF943010F0109203038091F302909184
:102DD000F4020E94DF199093B8068093B706109210
:102DE000070380910803882351F18091080188230B
:102DF00031F10E94732580E590E09F938F938BEED5
:102E000097E09F938F9321E030E03F932F9388E2E8
:102E100091E09F938F933F932F9382E693E09F934C
:102E20008F9383E08F9381E08F938CE48F930E9444
:102E3000C610109208038DB79EB70F968DBF809174
:102E400005038823D1F0809108018823B1F08AE03E
:102E500090E09F938F938CEA95E09F938F9381E00E
:102E60008F938F9386E58F930E94C610109205036F
:102E70002DB73EB7295F3F4F2DBF809109038823AF
:102E8000D9F0809108018823B9F08BE090E09F93FE
:102E90008F938EEC95E09F938F9381E08F93809139
:102EA00005018F9387E48F930E94C6101092090347
:102EB0008DB79EB707968DBF8091F7029091F8026B
:102EC000892B41F08091AA059091AB050E94E819E9
:102ED000882321F480910603882341F18091080121
:102EE000882321F10E94A43A82E490E09F938F937B
:102EF00085E997E09F938F9381E08F938F9384E48C
:102F00008F930E94C610109206032DB73EB7295F1B
:102F10003F4F2DBF8091F7029091F802009731F05A
:102F20000E94DF199093AB058093AA058091F5026A
:102F30009091F602892B09F497C08091A805909191
:102F4000A9050E94E819882309F48EC08091080120
:102F5000882309F489C08091800A9091810A909316
:102F60009B0580939A058091820A9091830A9093A1
:102F70009D0580939C052091620A3091630A4091DF
:102F8000640A5091650ADA01C90163E0880F991F4C
:102F9000AA1FBB1F6A95D1F7820F931FA41FB51FED
:102FA000820F931FA41FB51F20914201309143014E
:102FB0004091440150914501BC01CD010E94149DF6
:102FC00030939F0520939E058091690490916A0437
:102FD000A0916B04B0916C0449E0B595A7959795C5
:102FE00087954A95D1F78093A005809165049091CB
:102FF0006604A0916704B091680439E0B595A7957F
:10300000979587953A95D1F78093A10580917104A2
:1030100090917204A0917304B091740429E0B59565
:10302000A795979587952A95D1F78093A2058EE06D
:1030300090E09F938F938AE995E09F938F9381E02F
:103040008F938F9383E48F930E94C6108091F50233
:103050009091F6020E94DF199093A9058093A8052C
:103060008DB79EB707968DBF809107018F3F79F18D
:10307000992704E0880F991F0A95E1F78A599D4F17
:1030800040E150E0BC01CE0101960E94EA9A80E145
:1030900090E09F938F93CE0101969F938F9381E051
:1030A00090E09F938F9387E091E09F938F9382E0CE
:1030B0008F9381E08F9381E48F930E94C6108FEFEE
:1030C000809307012DB73EB7255F3F4F2DBF8091FD
:1030D000D7078823C9F0809108018823A9F081E0EF
:1030E00090E09F938F9387ED97E09F938F9381E07C
:1030F0008F938F9382E48F930E94C6101092D7070C
:103100008DB79EB707968DBF809104038823D1F0B9
:10311000809108018823B1F086E490E09F938F931B
:1031200084E799E09F938F9381E08F938F9380E55D
:103130008F930E94C610109204032DB73EB7295FEB
:103140003F4F2DBF8091D9059091DA050E94E81973
:10315000882309F448C080910801882309F443C0FA
:103160008091800A9091810A9093C7058093C6054B
:103170008091820A9091830A9093C9058093C80533
:10318000809123048093CA05809122048093CB050B
:1031900088E090E09F938F9386EC95E09F938F93C8
:1031A00081E08F9383E08F938BE68F930E94C6100C
:1031B0008091CC052DB73EB7295F3F4F2DBF85309D
:1031C00018F086E08093CC058091A401882319F43F
:1031D00083E690E002C087EE93E00E94DF199093AF
:1031E000DA058093D905E4E0C05F0C94599D1F92E5
:1031F0000F920FB60F9211242F933F935F936F930B
:103200007F938F939F93AF93BF93EF93FF9380919F
:103210001A03882329F080911A03815080931A039E
:1032200080913D05882319F0815080933D05809160
:1032300022038150809322038F3F09F051C089E01F
:103240008093220380912003909121030196909313
:10325000210380932003809112018F5F81708093FE
:103260001201882349F480911F03843028F480914F
:103270001F038F5F80931F03349903C081E0809305
:10328000180380911B0390911C03892B11F18091ED
:103290001B0390911C030B9750F080911B0390919E
:1032A0001C030A9790931C0380931B0304C0109285
:1032B0001C0310921B0380911B0390911C0320910F
:1032C0000B0130910C0182239323892B41F0479A03
:1032D00007C08FEF9FEF90930C0180930B014798ED
:1032E00080911803882309F45AC02091A401222355
:1032F00009F055C08091520A83FF51C086B19927C9
:10330000FC01E071F07084FF13C080911D03909167
:103310001E03019690931E0380931D0380911D034D
:1033200090911E03895E9340D0F12093180337C01B
:1033300080911D0390911E03892B69F180911D03DB
:1033400090911E038A56914030F580911D03909113
:103350001E0369E270E00E94CB9C80911D03909156
:103360001E03860F971F90931E0380931D03809169
:103370001D0390911E030B9750F080911D039091B7
:103380001E030A97909391018093900104C0F093DB
:103390009101E093900110921E0310921D03FF9182
:1033A000EF91BF91AF919F918F917F916F915F91BD
:1033B0003F912F910F900FBE0F901F901895209165
:1033C000200330912103280F391FC9010196089568
:1033D0002091200330912103821B930B892F992781
:1033E0008695807490700895CF93DF930E94DF19C3
:1033F000EC01CE010E94E8198823D9F3DF91CF9127
:103400000895CF93DF930E94DF19EC0109C08091EA
:103410001801882329F0909318018FEC80937A008B
:10342000CE010E94E819982F882389F3DF91CF916C
:1034300008959FB7F8945F983E9A469A8091B0009D
:103440008F708093B0008091B00083608093B00053
:103450008091B1008B738093B1008091B1008B603B
:103460008093B1001092B2008FEF8093B3008091EF
:10347000B00080688093B000809170008A7F809354
:103480007000809170008260809370009FBF0895EB
:103490008AE090E00E94DF199093D9078093D807C3
:1034A00082E085BD83EB84BD8FEF88BD84EB87BD53
:1034B00086E086BD80916E00816080936E000895E5
:1034C0008091AD0820916F0182FF30C090916C080F
:1034D0008CE3989FB001112490916B0880E5989F30
:1034E000A0011124922F905897FD9D5F9595959579
:1034F00086E09802C00111242091090130910A014F
:10350000281B390B30930A012093090142175307F6
:103510002CF050930A0140930901089526173707AC
:1035200084F070930A01609309010895822F99270E
:1035300036E0880F991F3A95E1F790930A0180933E
:1035400009010895EF92FF920F931F93CF93DF939A
:1035500080917308E82FFF27E85BFE4F9681C081BA
:1035600080911101813009F026C18091AF0887FF59
:1035700005C0C0E0D0E0E0E0F0E046C0892F992728
:1035800087FD9095A92FB92F2091A1043091A20415
:103590004091A3045091A404BC01CD010E94A09CC1
:1035A00097FF04C061587F4F8F4F9F4F7B018C0165
:1035B00087E015950795F794E7948A95D1F78C2FB6
:1035C000992787FD9095A92FB92F209199043091C3
:1035D0009A0440919B0450919C04BC01CD010E942F
:1035E000A09C97FF04C061587F4F8F4F9F4FB7E05B
:1035F0009595879577956795BA95D1F7F801E70185
:10360000C61BD70BE80BF90B209121053091220541
:10361000C901A3E0880F991FAA95E1F7821B930BBC
:10362000AA2797FDA095BA2FC81BD90BEA0BFB0B55
:1036300080916D019927AA27BB27BC01CD019E016E
:10364000AF010E94A09C97FF04C061507E4F8F4F36
:103650009F4FFC01EB0179E0F595E795D795C7956C
:103660007A95D1F71091AD086091090170910A0126
:1036700012FF05C07093100160930F0118C04091B4
:103680000F015091100180917208282F3327CB0130
:10369000841B950BB9010E94DF9C80910F019091D2
:1036A0001001860F971F9093100180930F0110FF58
:1036B00014C080910F019091100197FD0F9664E066
:1036C000959587956A95E1F7AA2797FDA095BA2F5A
:1036D000C80FD91FEA1FFB1F15C080910F019091E1
:1036E000100197FD0F9654E0959587955A95E1F74F
:1036F000AA2797FDA095BA2F8C1B9D0BAE0BBF0B75
:10370000FD01EC012091A608222321F133278091AD
:10371000140390911503829FA001839F500D929FE7
:10372000500D1124CA01AA2797FDA095BA2F8C0F1E
:103730009D1FAE1FBF1F2F5F3F4F442737FD409592
:10374000542FBC01CD010E94149D3093150320938A
:10375000140304C0D0931503C093140380916B0825
:10376000282F3327220F331F220F331F809114037A
:1037700090911503821793077CF080916C08282F95
:103780003327220F331F220F331F80911403909190
:1037900015032817390724F43093150320931403D5
:1037A00080910301843108F4FDC0809111018F5F85
:1037B00080931101F9C0892F992787FD9095A92F32
:1037C000B92F2091990430919A0440919B04509113
:1037D0009C04BC01CD010E94A09C97FF04C06158CD
:1037E0007F4F8F4F9F4F7B018C0187E01595079589
:1037F000F794E7948A95D1F78C2F992787FD9095B8
:10380000A92FB92F2091A1043091A2044091A304C3
:103810005091A404BC01CD010E94A09C9B01AC016D
:1038200097FF04C021583F4F4F4F5F4FC7E055955A
:10383000479537952795CA95D1F72E0D3F1D401F07
:10384000511F80916C019927AA27BB27BC01CD018C
:103850000E94A09C97FF04C061507E4F8F4F9F4FE6
:10386000FC01EB01B9E0F595E795D795C795BA95B9
:10387000D1F780916E019927A6E0880F991FAA952C
:10388000E1F740910D0150910E012091720833270C
:10389000841B950BB9010E94DF9C80910D019091D2
:1038A0000E01860F971F90930E0180930D0180915A
:1038B000AD0881FF14C080910D0190910E0197FD1C
:1038C0000F9674E0959587957A95E1F7AA2797FD6D
:1038D000A095BA2FC80FD91FEA1FFB1F15C08091F2
:1038E0000D0190910E0197FD0F9664E095958795D7
:1038F0006A95E1F7AA2797FDA095BA2F8C1B9D0B1F
:10390000AE0BBF0BFD01EC012091A708222321F192
:1039100033278091120390911303829FA001839F0C
:10392000500D929F500D1124CA01AA2797FDA09512
:10393000BA2F8C0F9D1FAE1FBF1F2F5F3F4F442715
:1039400037FD4095542FBC01CD010E94149D30934A
:1039500013032093120304C0D0931303C0931203E4
:1039600080916F08282F3327220F331F220F331F18
:103970008091120390911303821793077CF080913A
:103980007008282F3327220F331F220F331F8091F7
:103990001203909113032817390724F4309313036B
:1039A0002093120310921101E6E0CDB7DEB70C941C
:1039B000579D1F920F920FB60F9211242F933F9392
:1039C0004F935F938F939F93EF93FF9380910301A6
:1039D00090912303843108F04CC0992309F029C148
:1039E0008091B00086FF24C08091B0008F7B8093CF
:1039F000B000809114039091150387559E4F9093CA
:103A000017038093160325E08D3D920718F08CED87
:103A100095E005C08757914030F487E791E0909397
:103A20001703809316038091160390911703C2C069
:103A30008091B00080648093B00080917108282F3D
:103A400033278DED96E0289FA001299F500D389FC8
:103A5000500D1124CA012091240330912503821BAB
:103A6000930B909317038093160381E080931101C9
:103A7000DDC0992309F0DDC08091B00086FF9FC0B2
:103A80008091B0008F7B8093B000E091260320915D
:103A90007108EE23D9F433278DED96E0289FA0011D
:103AA000299F500D389F500D1124CA0120912403E5
:103AB00030912503821B930B909317038093160379
:103AC0001092250310922403469AB0C02E1738F4A2
:103AD0008AE090E09093170380931603A7C089EAC9
:103AE00093E090931703809316038E2F99278330CA
:103AF0009105D9F08430910534F48130910549F075
:103B0000029761F020C08430910591F0059799F0FB
:103B10001AC0809114039091150304C08091120380
:103B20009091130387559E4F1DC080912D0A05C0AB
:103B30008091060A02C08091360A9927880F991F42
:103B4000880F991FEFCFFF27EE0FFF1FEC58F64F9E
:103B500020813181220F331F80911603909117032A
:103B6000820F931F9093170380931603809116037F
:103B70009091170355E08D3D950718F08CED95E079
:103B800005C08757914030F487E791E09093170381
:103B90008093160320911603309117032C5B30405D
:103BA00030931703209316038091240390912503EB
:103BB000820F931F909325038093240337C0809135
:103BC000B00080648093B0008CEB90E0909317037A
:103BD00080931603809124039091250384549F4F72
:103BE000909325038093240380911903882321F067
:103BF00080914704882321F480911903823011F4C5
:103C0000469801C0469A809126038F5F80932603D1
:103C1000282F3327809171089927019682179307DF
:103C20002CF481E0809311011092260381E08093AF
:103C30002303209116033091170341E02F373407F7
:103C400030F08FEF8093B3002F5F30400FC02F3FD5
:103C50003105C9F0C0F0A9014F5F50404F37510501
:103C600050F480E88093B30020583040309317031D
:103C70002093160312C08FEF8093B3005093170365
:103C8000409316030AC0809116038093B3001092EC
:103C900017031092160310922303FF91EF919F9147
:103CA0008F915F914F913F912F910F900FBE0F9089
:103CB0001F90189510927C008FEC80937A000895E5
:103CC00080910604609116017091170120913303D1
:103CD000882379F0CB01AA27BB27332727FD30950E
:103CE000432F532FBC01CD010E94A09CDC01CB01CE
:103CF00016C084E0660F771F8A95E1F7CB01AA27EB
:103D0000BB27332727FD3095432F532FBC01CD010F
:103D10000E94A09CDC01CB010497A109B10980930A
:103D20002B0390932C03A0932D03B0932E0308959F
:103D3000CF93DF93109233030E94601E83E090E0E4
:103D40000E943430C82FDD27C03FD10508F42A96E1
:103D5000C7BD8C2F809588BD86E990E00E94011A2E
:103D600080911C0190911D018152934010F0C0EF91
:103D7000D0E0C630D10510F1C7BD8C2F809588BD2D
:103D800084E690E00E94011A8BE794E09F938F9362
:103D90008DE096E19F938F93E0919805F0919905BE
:103DA000099580911C0190911D010F900F900F902B
:103DB0000F908152934010F42197DBCFC093E80716
:103DC0006C2F83E090E00E943C308091490880FF96
:103DD0000AC08091E8078A508C3D28F08091B10597
:103DE00080648093B10580E1809315018091060481
:103DF0008823E9F080910301873150F4CC38D10554
:103E0000B0F480EA90E08C1B9D0B6AE170E009C081
:103E1000CA3AD10560F48CEB90E08C1B9D0B63E1FA
:103E200070E00E94CB9CCB01805F80931501809154
:103E30001501282F332780911C0190911D01829F2D
:103E4000A001839F500D929F500D1124CA01AA27F3
:103E5000BB2780931E0190931F01A0932001B09374
:103E600021018CE291E00E94011ADF91CF91089527
:103E7000EF92FF921F93CF9310E080ED97E00E94A6
:103E8000DF197C01CCE8133019F4CB3008F0C9E01D
:103E900010E080914203909143038C5F934024F49F
:103EA00080911B0181500AC080914203909143038D
:103EB0008750944034F080911B018F5F80931B01E9
:103EC00001C011E080914003909141038C5F9340C9
:103ED00024F480911A0181500AC08091400390918E
:103EE00041038750944034F080911A018F5F809392
:103EF0001A0101C01F5F80913E0390913F038C5FC8
:103F0000934024F48091190181500AC080913E03AE
:103F100090913F0387509440C4F0809119018F5FC6
:103F20008093190113C08DE794E09F938F938DE0E8
:103F300096E19F938F93E0919805F09199050995EB
:103F40000F900F900F900F905FC01F5F82E18093E2
:103F50006E03809168038E7F8093680385EA809367
:103F6000BC0080911B018A3040F48091B1058160D2
:103F70008093B1058AE080931B0180911B01863FED
:103F800040F08091B10581608093B10585EF809309
:103F90001B0180911A018A3040F48091B105826042
:103FA0008093B1058AE080931A0180911A01863FBF
:103FB00040F08091B10582608093B10585EF8093D8
:103FC0001A01809119018A3040F48091B105846012
:103FD0008093B1058AE08093190180911901863F91
:103FE00040F08091B10584608093B10585EF8093A6
:103FF000190180916E03882339F0C7010E94E819E6
:10400000882309F090CFF5CF109218018FEC8093A0
:104010007A00809118018823E1F3CA3020F48AE005
:1040200090E00E94011AC15009F02DCF86E490E083
:104030000E94011ACF911F91FF90EF9008951F9257
:104040000F920FB60F921124EF92FF920F931F93CE
:104050002F933F934F935F936F937F938F939F9390
:10406000AF93BF93CF93DF93EF93FF9380914B0375
:10407000282F3327442755278F5F80934B03F9015F
:104080002231310508F0F2C4EA5BFF4F0C94669DC3
:10409000809178009091790046C08091780090914D
:1040A0007900B8C1809178009091790090934F0386
:1040B00080934E03E3C18091AB049091AC042091B6
:1040C000780030917900821B930B9093DB078093EB
:1040D000DA078091DA079091DB0790935903809378
:1040E0005803EBC180917800909179002091AD0444
:1040F0003091AE04821B930B9093E7078093E60701
:104100008091E6079091E70790935B0380935A03B1
:10411000AFC4809152039091530320917800309165
:104120007900820F931F909353038093520381E091
:10413000A0C4809150039091510320917800309158
:104140007900820F931F909351038093500384E072
:1041500090C48091AE0883FF1AC08091260190918F
:1041600027019C01220F331F280F391F409178002F
:10417000509179008BE090E0489FB001499F700D0D
:10418000589F700D1124CB016EE170E00FC080913B
:104190002601909127019C01220F331F280F391F00
:1041A000809178009091790063E070E00E94CB9C50
:1041B000260F371F3695279536952795309327017B
:1041C0002093260185E055C4809178009091790074
:1041D0009093DD078093DC078091DC079091DD07E9
:1041E0004091A7045091A804841B950B6091A604EC
:1041F000262F332727FD3095821B930B909339038D
:104200008093380380910604882309F071C080915F
:1042100038039091390302977CF172E04E3E5707C4
:104220000CF0A7C020914C0330914D032B5F3F4F02
:1042300030934D0320934C032550304080910F0460
:1042400090911004845F914030F4215F3F4F309390
:104250004D0320934C0380914C0390914D03853680
:1042600091050CF486C04F5F5F4F5093A8044093B4
:10427000A7048456904037C0809138039091390349
:104280008F5F9F4F0CF075C082E0473258070CF4E7
:1042900070C020914C0330914D0325503040309335
:1042A0004D0320934C032B5F3F4F80910F0490915F
:1042B0001004845F914030F42F50304030934D0310
:1042C00020934C0380914C0390914D037FEF8C39E8
:1042D00097070CF04EC0415050405093A8044093B3
:1042E000A7048C599F4F90934D0380934C0341C07A
:1042F0008091220A9091230A8F5C9F41D4F1809192
:104300003803909139030297ACF020914C0330911F
:104310004D03C901019690934D0380934C03895836
:1043200093413CF166301CF46F5F6093A6042758FC
:1043300033411BC080913803909139038F5F9F4FA9
:10434000C4F420914C0330914D03C901019790931F
:104350004D0380934C0388579C4E5CF46B3F1CF0DC
:1043600061506093A60429573C4E30934D0320932F
:104370004C0380913803909139039C01442737FD09
:104380004095542F8091610490916204A091630440
:10439000B0916404820F931FA41FB51F8093610422
:1043A00090936204A0936304B09364042091610429
:1043B00030916204409163045091640457FF04C03B
:1043C00021503C4F4F4F5F4F6AE0559547953795C9
:1043D00027956A95D1F78091610490916204A0912C
:1043E0006304B0916404821B930BA40BB50B809300
:1043F000610490936204A0936304B093640430C199
:104400008091500390915103209178003091790070
:10441000820F931F909351038093500310924A038D
:104420002AC3809103018A3071F4809178009091C1
:10443000790020914E0330914F03820F931F019614
:104440009695879517C040914E0350914F03843144
:1044500058F02091780030917900240F351F8FEFAC
:1044600097E0821B930B06C08091780090917900B1
:10447000840F951F90933F0380933E038091140116
:10448000F8C28091AB049091AC04209178003091F7
:104490007900821B930B9093DB078093DA0780915E
:1044A000DA079091DB072091580330915903820F6E
:1044B000931F90933D0380933C0380911301D9C2D5
:1044C00080917800909179002091AD043091AE04F4
:1044D000821B930B9093E7078093E6078091E60792
:1044E0009091E70720915A0330915B03820F931F4D
:1044F00090933B0380933A03BBC2209152033091C7
:1045000053038091780090917900280F391F3093E0
:10451000530320935203809103018A3019F4220F30
:10452000331F04C0220F331F220F331F3093530356
:10453000209352032091520330915303C90137FD58
:10454000079603E0959587950A95E1F790934303C5
:10455000809342038091540390915503820F931FDF
:1045600097FD0196959587959093550380935403F5
:104570002091B7043091B804821B930B90932501CE
:1045800080932401209148033091490380912401B4
:1045900090912501280F391F37FF02C02F5F3F4F31
:1045A000359527953093490320934803C0CD20913A
:1045B0005003309151038091780090917900280F39
:1045C000391F3093510320935003809103018A30A7
:1045D00019F4220F331F04C0220F331F220F331F81
:1045E0003093510320935003209150033091510395
:1045F000C90137FD0796A3E095958795AA95E1F740
:104600009093410380934003809156039091570308
:10461000820F931F97FD0196959587959093570369
:10462000809356032091B5043091B604821B930BFE
:1046300090932301809322012091460330914703F8
:104640008091220190912301280F391F37FF02C06A
:104650002F5F3F4F359527953093470320934603AF
:1046600083E007C280910604882309F180E00E945C
:1046700087969B01AC0120503F4F4F4F5F4F57FF34
:1046800006C09B01AC0121503D4F4F4F5F4F79E079
:1046900055954795379527957A95D1F72093270318
:1046A000309328034093290350932A0310C080912C
:1046B000410490914204A0914304B091440480933A
:1046C000270390932803A0932903B0932A03109201
:1046D0004B0381E08093180180912F039091300368
:1046E00001969093300380932F03809178009091EE
:1046F000790090931D0180931C018091060488230A
:1047000009F472C080911C0190911D017C01002769
:10471000112780912B0390912C03A0912D03B09130
:104720002E03E81AF90A0A0B1B0BE0925C03F092C5
:104730005D0300935E0310935F0380911501282FA2
:1047400033274427552780911E0190911F01A09186
:104750002001B0912101BC01CD010E94149D8091E6
:104760001E0190911F01A0912001B0912101821B97
:10477000930BA40BB50B80931E0190931F01A09384
:104780002001B093210180911E0190911F01A09101
:104790002001B09121018E0D9F1DA01FB11F80939C
:1047A0001E0190931F01A0932001B09321018091DD
:1047B000DE079091DF07A091E007B091E10720911B
:1047C0001E0130911F014091200150912101821B57
:1047D000930BA40BB50B8093410490934204A093D8
:1047E0004304B093440444C180911C0190911D0185
:1047F000AA27BB27C0915C03D0915D03E0915E03C3
:10480000F0915F03C80FD91FEA1FFB1FC0935C0321
:10481000D0935D03E0935E03F0935F0380916003A8
:104820008F5F80936003803108F422C180911E0164
:1048300090911F01A0912001B09121019C01AD0137
:1048400063E0220F331F441F551F6A95D1F7281BC1
:10485000390B4A0B5B0B2C0F3D1F4E1F5F1F8091C6
:104860002B0390912C03A0912D03B0912E03281BB4
:10487000390B4A0B5B0B57FF04C0295F3F4F4F4F6B
:104880005F4F03E055954795379527950A95D1F7E2
:1048900020931E0130931F0140932001509321016A
:1048A000C091DE07D091DF07E091E007F091E107CA
:1048B00080911E0190911F01A0912001B0912101D2
:1048C000C81BD90BEA0BFB0BC0934104D0934204E5
:1048D000E0934304F0934404209134033091350372
:1048E000409136035091370357FF04C0215F3F4F7B
:1048F0004F4F5F4F14E055954795379527951A957B
:10490000D1F78091340390913503A0913603B09193
:104910003703821B930BA40BB50B80933403909346
:104920003503A0933603B0933703809134039091FD
:104930003503A0913603B09137038C0F9D1FAE1F36
:10494000BF1F8093340390933503A0933603B09335
:1049500037038091340390913503A0913603B091D1
:104960003703B7FF03C00F96A11DB11DC4E0B59575
:10497000A79597958795CA95D1F7209141043091D5
:104980004204281B390B64E0213036071CF020E07C
:1049900034E006C07CEF2030370714F420E03CEF11
:1049A00080913103909132038091310390913203D1
:1049B00097FF03C0909581959F4FA901F3E0440FA5
:1049C000551FFA95E1F78D5B9240C4F08091310359
:1049D000909132039C01E4E0220F331FEA95E1F746
:1049E000281B390B240F351F37FF02C0215F3F4FB3
:1049F00074E0359527957A95E1F717C080913103DA
:104A0000909132039C0165E0220F331F6A95E1F714
:104A1000281B390B240F351F37FF02C0215E3F4F83
:104A200045E0359527954A95E1F730933203209379
:104A3000310380915C0390915D03A0915E03B0917E
:104A40005F03B7FF03C00196A11DB11DB595A795E2
:104A50009795879580935C0390935D03A0935E0385
:104A6000B0935F0388E08093600302C010924B0311
:104A700082E080934A0380914A0380937C00809176
:104A80004B03882319F08FEC80937A00FF91EF910C
:104A9000DF91CF91BF91AF919F918F917F916F9156
:104AA0005F914F913F912F911F910F91FF90EF9048
:104AB0000F900FBE0F901F90189590E2EBEEF7E06D
:104AC0008FE49193815087FFFCCF08959091630309
:104AD000903540F4E92FFF27E551F84F80839F5F21
:104AE000909363030895A0E0B0E0E9E7F5E20C9449
:104AF000399D2091610320FF0AC0809162038823C1
:104B000011F0815002C0809128018093620321FF3F
:104B10000CC09091620380912801981719F41092AB
:104B2000620303C09F5F90936203822F992780FFE7
:104B300004C081FF02C0109262030E945D25809133
:104B40006203282F332706E615E2C0919805D0911D
:104B500099058A3098F481E1809363033F932F9302
:104B600084EB94E09F938F931F930F93FE0109951D
:104B70002DB73EB72A5F3F4F2DBF12C080E1809313
:104B800063033F932F9389EB94E09F938F931F933D
:104B90000F93FE0109954DB75EB74A5F5F4F4DBF5A
:104BA00020916203822F9927AA27BB27FC014297F5
:104BB00010F00C940E2EE85AFF4F06E615E2C09155
:104BC0009805D09199050C94669D109263038EEB25
:104BD00094E09F938F9356E6E52E55E2F52E1F93B2
:104BE0000F93FE01099584E1809363030F900F906A
:104BF0000F900F9082E690E09F938F9382E090E079
:104C00009F938F939F938F93809103016AE00E94FB
:104C1000BF9C892F99279F938F93809103010E94B6
:104C2000BF9C99279F938F938EEC94E09F938F93D3
:104C30001F930F93E0919805F0919905099588E2EB
:104C4000809363038DB79EB70E968DBF8EEB98E071
:104C50009F938F938091010199279F938F9386EE65
:104C600094E09F938F931F930F93E0919805F09199
:104C7000990509958091B2059927EDB7FEB7389649
:104C8000EDBFEC01C071D07084FF0AC08CE380934B
:104C9000630384EF94E09F938F931F930F9353C705
:104CA00090912805992351F18CE380936303892F18
:104CB00099279F938F9381E095E09F938F93FF9225
:104CC000EF92E0919805F09199050995DF93CF93C4
:104CD0009091280581E1989FC0011124855D954F31
:104CE0009F938F93FF92EF92E0919805F091990531
:104CF00009952DB73EB7245F3F4F77C49091B1051A
:104D0000992371F08CE380936303892F99279F93F4
:104D10008F9389E095E09F938F93FF92EF9204C465
:104D2000909169039923B9F08CE380936303892FF1
:104D300099279F938F9380E295E09F938F93FF92A3
:104D4000EF92E0919805F091990509958DB79EB77E
:104D500006968DBF6CC780913C0190913D010697EE
:104D600030F48CE38093630386E395E0E8C690918A
:104D7000F80A9E3108F05BC78CE380936303892FA8
:104D800099279F938F9383E495E00AC11092630360
:104D90008091410490914204A0914304B091440455
:104DA000BC01CD0125E030E040E050E00E94149DC0
:104DB0003F932F9387E595E09F938F931F930F93D6
:104DC000FE01099584E1809363032DB73EB72A5F06
:104DD0003F4F2DBF80913D0490913E04A0913F0430
:104DE000B0914004BC01CD0125E030E040E050E04E
:104DF0000E94149D3F932F9384E695E09F938F9399
:104E00001F930F93E0919805F0919905099588E219
:104E1000809363034DB75EB74A5F5F4F4DBF80918C
:104E20001C0190911D019F938F9381E795E09F93C3
:104E30008F931F930F93E0919805F0919905099531
:104E40008CE3809363038DB79EB706968DBF87B5BD
:104E500099279F938F938EE795E09F938F931F934E
:104E60000F93E0919805F09199050995EDB7FEB77C
:104E70003696EDBF80910604882309F4D8C689E3ED
:104E8000809363038BE895E09F938F931F930F9319
:104E9000E0919805F091990509958DE4809363035D
:104EA0000F900F900F900F908091150199279F936D
:104EB0008F938FE895E08CC31092630382E995E0AD
:104EC0009F938F9346E6E42E45E2F42E1F930F93B3
:104ED000FE01099584E1809363030F900F900F907A
:104EE0000F908091A1049091A204A091A304B0918D
:104EF000A404B7FF04C081509C4FAF4FBF4F3AE0AE
:104F0000B595A795979587953A95D1F7BF93AF93A8
:104F10009F938F938FE995E09F938F93FF92EF92EA
:104F2000E0919805F0919905099588E280936303D3
:104F30004DB75EB7485F5F4F4DBF80919904909128
:104F40009A04A0919B04B0919C04B7FF04C08150C7
:104F50009C4FAF4FBF4F2AE0B595A7959795879582
:104F60002A95D1F7BF93AF939F938F938EEA95E0E5
:104F70009F938F93FF92EF92E0919805F09199059E
:104F800009958CE3809363038DB79EB708968DBF18
:104F900080910E0A90910F0A9F938F938DEB95E06D
:104FA0009F938F93FF92EF92E0919805F09199056E
:104FB0000995EDB7FEB73696D8C391E0F92EC1E05A
:104FC000D0E006E719E09F2D969584E1989FC001F7
:104FD000112480936303F801828193819F938F93BF
:104FE0002196DF93CF932197808191819F938F9317
:104FF000DF93CF938CEC95E09F938F9386E695E2B9
:105000009F938F93E0919805F091990509952DB79D
:105010003EB7245F3F4F2DBF32E0F30E22960C5F68
:105020001F4F48E04F1578F602C610926303809137
:105030003E08E82FFF27EE0FFF1FEC58F64F808148
:1050400091819F938F9380913D08E82FFF27EE0F6A
:10505000FF1FEC58F64F808191819F938F938EEDC7
:1050600095E09F938F931F930F93FE01099584E121
:10507000809363038DB79EB708968DBF80914008DB
:10508000E82FFF27EE0FFF1FEC58F64F808191812C
:105090009F938F9380913F08E82FFF27EE0FFF1F0C
:1050A000EC58F64F8081918181589F4F9F938F9349
:1050B0008EEE95E09F938F931F930F93E091980549
:1050C000F0919905099588E280936303EDB7FEB7E7
:1050D0003896EDBF80914208E82FFF27EE0FFF1FA3
:1050E000EC58F64F8081918181589F4F9F938F9309
:1050F00080914108E82FFF27EE0FFF1FEC58F64F75
:105100008081918181589F4F9F938F938EEF95E07F
:105110009F938F931F930F93E0919805F0919905BA
:1051200009958CE3809363032DB73EB7285F3F4F0B
:105130002DBF80914408E82FFF27EE0FFF1FEC588A
:10514000F64F8081918181589F4F9F938F938091DB
:105150004308E82FFF27EE0FFF1FEC58F64F808122
:10516000918181589F4F9F938F938EE096E09F93FC
:105170008F931F930F93E0919805F09199050995EE
:105180004DB75EB7485F5F4FD8C1109263038EE1A1
:1051900096E09F938F9386E6E82E85E2F82E1F9384
:1051A0000F93FE01099584E1809363030F900F90A4
:1051B0000F900F908091B7049091B8049C0197FFD5
:1051C00002C0215F3F4F207F821B930B97FD01960A
:1051D000959587959F938F938091B7049091B8048C
:1051E00097FD0F96B4E095958795BA95E1F79F9353
:1051F0008F932091B7043091B80437FF02C0295F24
:105200003F4FA3E035952795AA95E1F7809142039A
:1052100090914303821B930B9F938F938CE296E0B4
:105220009F938F93FF92EF92E0919805F0919905EB
:10523000099588E2809363038DB79EB70A968DBF68
:105240008091B5049091B6049C0197FF02C0215F44
:105250003F4F207F821B930B97FD01969595879575
:105260009F938F938091B5049091B60497FD0F960C
:10527000E4E095958795EA95E1F79F938F932091C8
:10528000B5043091B60437FF02C0295F3F4F73E089
:10529000359527957A95E1F78091400390914103E8
:1052A000821B930B9F938F938EE396E09F938F9334
:1052B000FF92EF92E0919805F091990509958CE3A2
:1052C00080936303EDB7FEB73A96EDBF8091B304C8
:1052D0009091B40497FD0196959587959F938F9330
:1052E0008091B3049091B40420913E0330913F0328
:1052F000821B930B9F938F9380E596E09F938F93F0
:10530000FF92EF92E0919805F091990509952DB7DC
:105310003EB7285F3F4F69C1109263038FE596E067
:105320009F938F931F930F93FE01099584E18093C0
:1053300063030F900F900F900F908091AD049091A8
:10534000AE049F938F9380913A0390913B039F9378
:105350008F938CE696E09F938F931F930F93E0912A
:105360009805F0919905099588E2809363034DB7FC
:105370005EB7485F5F4F4DBF8091AB049091AC0426
:105380009F938F9380913C0390913D039F938F93C4
:105390008BE796E09F938F931F930F93E09198056F
:1053A000F091990509958CE3809363038DB79EB7BF
:1053B00008968DBF8091A7049091A8049F938F9326
:1053C00080913803909139039F938F938AE896E0F8
:1053D0009F938F931F930F93C0C11092630380918B
:1053E0002601909127016AE070E00E94DF9C9F9364
:1053F0008F9380912601909127016AE070E00E94CE
:10540000DF9C7F936F9389E996E09F938F931F931F
:105410000F93FE01099584E1809363032DB73EB796
:10542000285F3F4F2DBF8091F20A9091F30A6AE006
:1054300070E00E94CB9C9F938F938091F20A909191
:10544000F30A6AE070E00E94CB9C7F936F938DEA31
:1054500096E09F938F931F930F93E0919805F0919F
:105460009905099588E2809363034DB75EB7485F5D
:105470005F4F4DBF8091F40A9091F50A9F938F93EF
:1054800081EC96E09F938F931F930F93E091980583
:10549000F091990509958CE3809363038DB79EB7CE
:1054A00006968DBF8091F60A9091F70A9F938F938D
:1054B00081ED96E09F938F931F930F9375CD10927C
:1054C000630383EE96E09F938F931F930F93FE01E8
:1054D000099588E2809363030F900F900F900F90CF
:1054E0008091470499279F938F938CEE96E09F932A
:1054F0008F931F930F93E0919805F091990509956B
:105500008CE3809363032DB73EB72A5F3F4F2DBFD7
:1055100080917309992701979F938F938CEF96E061
:105520009F938F931F930F93E0919805F0919905A6
:1055300009954DB75EB74A5F5F4F4DBF78C3109274
:1055400063038CE097E09F938F931F930F93FE016B
:10555000099584E1809363030F900F900F900F9053
:1055600080919001909191019F938F9384E197E0B6
:105570009F938F931F930F93E0919805F091990556
:10558000099588E2809363038DB79EB706968DBF19
:1055900080910E0A90910F0A9F938F9382E297E079
:1055A0009F938F931F930F93E0919805F091990526
:1055B00009958CE380936303EDB7FEB73696EDBF94
:1055C00080915F04909160049F938F9380E397E0B4
:1055D0009F938F931F930F93E0919805F0919905F6
:1055E00009952DB73EB72A5F3F4F2DBF20C358E422
:1055F000C52E54E0D52E20E030E0E90143E0F42E42
:10560000C0936303F60181916F0199279F938F9354
:1056100089010F5F1F4F1F930F938EE397E09F93B6
:105620008F9386E695E29F938F93E0919805F09192
:10563000990509952DB73EB7285F3F4F2DBFFA94C6
:1056400064969801F7FEDCCFF2C29CE4C92E94E088
:10565000D92EC0E0D0E08E0183E0F82E00936303E2
:10566000F60181916F0199279F938F932596DF9380
:10567000CF938BE497E09F938F9386E695E29F9379
:105680008F93E0919805F091990509952DB73EB754
:10569000285F3F4F2DBFFA940C5E1F4F2497F7FEF3
:1056A000DDCFC5C21092630388E597E09F938F9387
:1056B000B6E6EB2EB5E2FB2E1F930F93FE01099584
:1056C00084E1809363030F900F900F900F9080916F
:1056D0006F0199279F938F9380E697E09F938F9315
:1056E0001F930F93E0919805F0919905099588E231
:1056F000809363034DB75EB74A5F5F4F4DBF8091A4
:1057000014039091150397FD0396959587959595AC
:1057100087959F938F938EE697E09F938F93FF9249
:10572000EF92E0919805F091990509958CE38093AB
:1057300063038DB79EB706968DBF80916C0899273D
:105740009F938F9380916B0899279F938F938CE7FA
:1057500097E09F938F93FF92EF92E0919805F091DD
:1057600099050995EDB7FEB73896EDBF60C2109266
:1057700063038AE897E09F938F93F6E6CF2EF5E2D6
:10578000DF2E1F930F93FE0109950F900F900F903E
:105790000F90C3E1D9E000E010E0E2E0FE2E802FA0
:1057A0008C5E809363038B8D99278F7790709F9386
:1057B0008F938B8999278F7790709F938F938B8589
:1057C00099278F7790709F938F938B8199278F77ED
:1057D00090709F938F938AE997E09F938F93DF92C6
:1057E000CF92E0919805F091990509952DB73EB7B4
:1057F000245F3F4F2DBFFA940C5E1F4FA096F7FE1B
:10580000CECF15C2109263038BEA97E09F938F93DC
:1058100076E6C72E75E2D72E1F930F93FE010995EA
:105820000F900F900F900F90C3E1D9E000E010E0CF
:1058300062E0F62E802F8C5E809363038F8D992714
:1058400087FD90959F938F938F89992787FD9095DA
:105850009F938F938F85992787FD90959F938F9323
:105860008F81992787FD90959F938F938AEB97E07F
:105870009F938F93DF92CF92E0919805F0919905D5
:1058800009954DB75EB7445F5F4F4DBFFA940C5E0C
:105890001F4FA096F7FECECFCAC1109263038BECC8
:1058A00097E09F938F9356E6C52E55E2D52E1F9312
:1058B0000F93FE01099587E4809363030F900F9087
:1058C0000F900F9086ED97E09F938F931F930F9308
:1058D000E0919805F09199050995FF240F900F909C
:1058E0000F900F90C0E0D0E08E01802F8C5E8093EF
:1058F00063038C2F8D5F0E94AA7A9F938F938C2FC6
:105900008E5F0E94AA7A9F938F938C2F8F5F0E9445
:10591000AA7A9F938F938C2F0E94AA7A9F938F933A
:1059200080EE97E09F938F93DF92CF92E09198055E
:10593000F091990509959E012C5F3F4F80913B089E
:105940009927EDB7FEB73C96EDBF281739070CF045
:105950006EC1F3940C5E1F4FE901F2E0FF1528F6CB
:1059600066C11092630381EF97E09F938F9346E6A1
:10597000E42E45E2F42E1F930F93FE01099584E176
:10598000809363030F900F900F900F9080912E09DA
:10599000881F8827881F97E0899FC00111248D9652
:1059A0009F938F9380912609881F8827881F96E0F0
:1059B000899FC00111248D969F938F9380911E091A
:1059C000881F8827881F95E0899FC00111248D9624
:1059D0009F938F9380911609881F8827881F992786
:1059E000880F991F880F991F8D969F938F9380E042
:1059F00098E09F938F931F930F93E0919805F091F8
:105A00009905099588E2809363032DB73EB7245F1B
:105A10003F4F2DBF80914E09881F8827881F9BE02C
:105A2000899FC00111248D969F938F938091460981
:105A3000881F8827881F9AE0899FC00111248D96AE
:105A40009F938F9380913E09881F8827881F99E034
:105A5000899FC00111248D969F938F938091360961
:105A6000881F8827881F992723E0880F991F2A9568
:105A7000E1F78D969F938F9384E198E09F938F93A6
:105A80001F930F93E0919805F091990509958CE388
:105A9000809363034DB75EB7445F5F4F4DBF809106
:105AA0005609881F8827881F9CE0899FC001112400
:105AB0008D969F938F9388E298E09F938F931F9387
:105AC0000F93E0919805F0919905099580915E09F1
:105AD000EDB7FEB73696EDBF87FF12C080E4809326
:105AE000630389E398E09F938F931F930F93E09153
:105AF0009805F091990509950F900F900F900F90D0
:105B00008091660987FF12C084E4809363038CE36D
:105B100098E09F938F93FF92EF92E0919805F09118
:105B2000990509950F900F900F900F9080916E0935
:105B300087FF7DC088E4809363038FE398E09F93A1
:105B40008F93FF92EF92E0919805F0919905099556
:105B50000F900F900F900F906AC01092630382E431
:105B600098E09F938F931F930F93FE01099584E113
:105B7000809363030F900F900F900F908091EA0233
:105B80009091EB029F938F9380E598E09F938F9382
:105B90001F930F93E0919805F0919905099588E27C
:105BA000809363032DB73EB72A5F3F4F2DBF80918F
:105BB000EC029091ED029F938F938DE598E09F9377
:105BC0008F931F930F93E0919805F0919905099594
:105BD00089E4809363034DB75EB74A5F5F4F4DBF63
:105BE0008AE698E09F938F931F930F93E091980517
:105BF000F09199050995809161030F900F900F9096
:105C00000F9083FF14C01092ED021092EC0260E03E
:105C100070E08EE090E00E944D3009C08091280134
:105C2000281719F421502093280110926203109232
:105C30006103E8E0CDB7DEB70C94559DF999FECF2E
:105C400092BD81BDF89A80B599270895F999FECF44
:105C50001FBA92BD81BD60BD0FB6F894FA9AF99A49
:105C60000FBE08954AEA20E030E02617370740F4D7
:105C7000FC018191480F2F5F3F4F26173707C8F36C
:105C8000842F99270895EAEA40E050E04617570725
:105C900078F49C01F999FECF32BD21BDF89A80B508
:105CA000E80F4F5F5F4F2F5F3F4F4617570790F347
:105CB0008E2F9927089581E080933F0882E080939A
:105CC0003E0883E080933D0884E08093400885E0AF
:105CD0008093410886E08093420887E080934308E0
:105CE00088E08093440889E0809345088AE08093A7
:105CF00046088BE0809347088CE08093480808951D
:105D000081E680933C088CE0E0EBF8E011928A9504
:105D1000E9F780910301843150F08AE080935C08B8
:105D2000109280088BE1809358088EE40AC083E0CB
:105D300080935C0880E2809380088EE1809358080D
:105D400085E580937D0880937E0880E280937F08BC
:105D50001092AC088AE68093490882E78093AE08E7
:105D600080E58093AF0886E0809363081092A008D6
:105D700010929D0838E03093560886EE80935708BD
:105D800080E48093590885E080934C082EE12093AD
:105D90004A0890910604992399F084E180934D0874
:105DA00088E280934B0820934F0881E0809350084D
:105DB000109251088FE7809352082093A30810C0D7
:105DC0008FE080934D0820934B0890934F083093B9
:105DD000500884E180935108909352089093A3084F
:105DE0008FE080934E081092A8088CE08093A90859
:105DF0001092650810926608109267081092680861
:105E000010928208109283081092840810928508DC
:105E100090E89093690842E340936A0872E07093B7
:105E2000AD0888E180936B0886EE80936C0883E070
:105E3000809371085DE750937408509375085093F0
:105E4000760890936D0865E560936E0886E480930C
:105E50006F088CED809370088CE380937208109229
:105E600073089AEA909386088CEC809388081092C5
:105E70008A0890938B0898E29093870890938908FA
:105E800010928C08409377082AE520937808409375
:105E9000790836E030938D0884E680938E088093ED
:105EA0008F082093900888E7809391089093950835
:105EB0008BE48093920860939308809394083093C6
:105EC000960888E080939708409398088AE2809328
:105ED000990885EF80939A088CE880939B087093CB
:105EE0009C0810929E0810929F0881E2809360089F
:105EF00081E480936108209362081092A1081092B7
:105F0000A20886E98093A40850937A0884E38093DA
:105F10007B081092A5081092A6081092A70810926C
:105F2000AA088FE18093AB0808950E94802E8AE032
:105F30008093530880E18093540826E0209355080D
:105F40009AE590935A0888E780935B0890935D08E0
:105F500080935E0820935F0880E2809364088CE35E
:105F600080937C088BE48093810886E491E6A3E724
:105F7000B4E78093B0089093B108A093B208B093AF
:105F8000B30860E870E08CE398E00E94322E8093C2
:105F9000BC080895CF93DF930E94802E88E0809301
:105FA000530830E13093540826E02093550894E6D6
:105FB00090935A0888E780935B0890935D088093DC
:105FC0005E0820935F083093640886E480937C0821
:105FD00080938108A0EBB8E085E0E9E2F1E0ED0113
:105FE000019009928A95E1F760E870E0CD0184574D
:105FF00090400E94322E8093BC08DF91CF9108958B
:106000000E94802E26E0209353088AE08093540853
:1060100084E08093550894E690935A0888E780932B
:106020005B0890935D0880935E0820935F0880E191
:106030008093640886E480937C088093810885E4DB
:1060400091E6A3E7B9E78093B0089093B108A093D5
:10605000B208B093B30860E870E08CE398E00E9467
:10606000322E8093BC080895F999FECF92BD81BD70
:10607000F89A80B599270895F999FECF1FBA92BD75
:1060800081BD60BD0FB6F894FA9AF99A0FBE0895D3
:106090006EE17EE20E942E9B089546E25EE20E943F
:1060A000689B0895EF92FF920F931F93CF93C82F91
:1060B0008150853008F0C3E081E8C89F8001112439
:1060C00083EEE82E8FEFF82EE00EF11E60E870E010
:1060D000C7010E94432E682F98012D593F4F8FB35F
:1060E0009927AC014270507081FDF9CF32BD21BDBE
:1060F000F89A80B5861711F0CA0123C08FB399278B
:106100009C012270307081FDF9CFF2BCE1BCF89A9D
:1061100080B5813611F0C90114C081E8C89FC00163
:1061200011244D972EE13EE241E850E0BC018CE3A2
:1061300098E00E94099B0E940D760E94229581E0C2
:1061400090E0CF911F910F91FF90EF900895282F2D
:10615000863010F025E003C0882309F421E0209365
:106160000101F999FECF1FBA82E090E092BD81BD96
:1061700020BD0FB6F894FA9AF99A0FBE0895CF93FE
:10618000C82F80913C08813609F051C0C63010F00C
:10619000C5E003C0CC2309F44AC00E94E99980916C
:1061A000AF0882FF07C080916108843618F080E54F
:1061B0008093610860E870E08CE398E00E94322EE2
:1061C0008093BC0881E8C89FC001112426E23EE20A
:1061D00041E850E06CE378E04D970E94469B26E250
:1061E0003EE24CE050E06DE378E080E590E00E9414
:1061F000469B6CE070E08DE398E00E94322E282FE1
:10620000F999FECF1FBA8CE590E092BD81BD20BD0B
:106210000FB6F894FA9AF99A0FBE8C2F0E94A73005
:106220000E940D760E94229581E090E002C080E0FD
:1062300090E0CF9108956DE470E088EE93E00E94C5
:10624000432E482F8FB399279C012270307081FD17
:10625000F9CF85E394E092BD81BDF89A80B58417AB
:1062600079F48FB399279C012270307081FDF9CFAA
:1062700088EE93E092BD81BDF89A80B5813011F02F
:10628000C90108952EE13EE24EE450E068EE73E06D
:106290008DEB98E00E94099B81E090E00895809149
:1062A000BD088130A9F46DE470E08DEB98E00E94A8
:1062B000322E80930A0926E23EE24EE450E06DEB76
:1062C00078E088EE93E00E94469B81E090E008959C
:1062D00080E090E00895CF93DF9381E08093BD0844
:1062E000EDEBF8E08FE0158616861786108A815050
:1062F000349687FFF8CF80E48093CA088093CB0858
:106300001092CC088093CD088093CE0890EC9093A7
:10631000CF081092D0088093D1088093D2081092B1
:10632000D3089093D4089093D5088093D608109200
:10633000D7088093D8089093D908AEEBB8E08CE0EA
:10634000EFE2F1E0ED01019009928A95E1F76DE449
:1063500070E0CD0101970E94322E80930A09DF91EF
:10636000CF910895F999FECF82E090E092BD81BD72
:10637000F89A80B5282F863078F023E0322FF999EB
:10638000FECF1FBA82E090E092BD81BD30BD0FB656
:10639000F894FA9AF99A0FBE20930101822F992757
:1063A00008951F93CF93C82F162F863010F0C5E0A5
:1063B00003C0882309F4C1E08C2F9927823091050E
:1063C00041F08330910544F4019731F40E94952FF8
:1063D00005C00E94CA2F02C00E9400301123E1F0C4
:1063E0006CE070E080E590E00E94432E282FF99940
:1063F000FECF8CE590E092BD81BDF89A80B5821702
:1064000059F42EE13EE24CE050E060E570E08DE3AF
:1064100098E00E94099B02C00E945B2E8C2F0E9474
:10642000BF30CF911F910895DF92EF92FF920F93AB
:106430001F93CF93FF24DF2CEF2C81E190E00E948B
:10644000343090910301981791F1963169F481E10C
:1064500090E00E943430853139F44C9905C06F2D9D
:1064600081E090E00E943C306091030181E190E086
:106470000E943C3088E190E028E00FB6F894A8959F
:10648000809360000FBE2093600082E798E09F93A6
:106490008F938DE096E19F938F93E0919805F09113
:1064A000990509950F900F900F900F90FFCF81E005
:1064B00090E00E943430813611F031E0E32E6CE040
:1064C00070E080E590E00E94432EC82FF999FECF3E
:1064D0008CE590E092BD81BDF89A80B58C1711F4DF
:1064E00021E0D22EC1E001E010E0EE2029F48C2F53
:1064F0000E9452308823B9F591E0F92E1F930F9333
:106500008AE998E09F938F938DE096E19F938F9314
:10651000E0919805F091990509952DB73EB72A5F4E
:106520003F4F2DBF0130110521F00230110521F040
:1065300006C00E94952F05C00E94CA2F02C00E946B
:106540000030DD2059F02EE13EE24CE050E060E505
:1065500070E08DE398E00E94099B02C00E945B2ED0
:106560008C2F0E94BF30CF5F0F5F1F4FC63008F4E3
:10657000BCCFFF2019F083E00E94A7300E94B23107
:10658000C82F0E9452308C2F99279F938F9380ECB5
:1065900098E09F938F930DE016E11F930F93E09186
:1065A0009805F0919905099581E090E00E943430BA
:1065B0002DB73EB72A5F3F4F2DBF8F3F21F00E947E
:1065C0001B31882399F489ED98E09F938F931F9353
:1065D0000F93E0919805F091990509950E946B3110
:1065E0000E944F310F900F900F900F90EE2029F0E6
:1065F00061E681E090E00E943C3010923B0890E020
:10660000EAECF8E0CFE08081349618160CF49F5F36
:10661000C150C7FFF8CF90933B08892F99279F93CC
:106620008F938EEB98E09F938F938AEF98E09F93E0
:106630008F931F930F93E0919805F0919905099519
:106640000E9492098DB79EB708968DBFCF911F917A
:106650000F91FF90EF90DF900895982F2FB7F89447
:106660003998389A88B1836088B98091B9008C7F55
:106670008093B9008AE28093B80010926E03109262
:106680006C0310926B03992379F0E3E1F9E08BE05E
:10669000108211821282138214821582168217824E
:1066A0008150389687FFF4CF78942FBF08951092C9
:1066B0006E0384E98093BC0080E88093BC00109254
:1066C000BD001092BA001092BB001092B900109257
:1066D000B80010926A0380E00E942D331092BB0034
:1066E00085E88093BC008091680382608093680392
:1066F00008951F920F920FB60F9211242F933F937C
:106700004F935F938F939F93EF93FF9380916E03CB
:10671000282F3327442755278F5F80936E03F90175
:106720002731310508F00DC3E659FF4F0C94669DE3
:1067300081E080936A0309C080916C038C3090F4EF
:1067400080916C038F5F80936C0380916C03E82FC2
:10675000FF27EE0FFF1FEE0FFF1FE354F74F858556
:10676000181654F780916C038C3070F01092670308
:106770001092660310926C0385E080936E03809103
:106780006B03880F8D5A04C080916C03880F8E5A5A
:106790008093BB0085E8CAC280916C03E82FFF2775
:1067A00023E0EE0FFF1F2A95E1F7ED5EF64F8181A2
:1067B0008093BB0085E88093BC0080916C03E82F38
:1067C000FF2793E0EE0FFF1F9A95E1F7ED5EF64F7E
:1067D000808180FF92C080916C03E82FFF2783E0C7
:1067E000EE0FFF1F8A95E1F7ED5EF64F8281882359
:1067F00029F080913B08873008F4B9C28091660384
:1068000090916703892B09F0B2C280916403909143
:106810006503892B09F0ABC270C080916C0321E045
:1068200030E002C0220F331F8A95E2F780916403A3
:106830009091650328233923232B79F080916C03F1
:10684000E82FFF27EE0FFF1FEE0FFF1FEE0FFF1FBA
:10685000ED5EF64F80E184830DC080916C03E82FDC
:10686000FF27EE0FFF1FEE0FFF1FEE0FFF1FED5E66
:10687000F64F148280916C03E82FFF27EE0FFF1F65
:10688000EE0FFF1FEE0FFF1FED5EF64F8481282FE6
:106890003327220F331F220F331F220F331F809104
:1068A0006C03E82FFF2753E0EE0FFF1F5A95E1F727
:1068B000ED5EF64F82818770822B8093BB0085E866
:1068C0008093BC0020916C0381E090E002C0880FAF
:1068D000991F2A95E2F7209166033091670382237E
:1068E0009323892B51F08BE099E09093720380936E
:1068F000710388E0809373033AC284E0D4C1E091CD
:106900007103F091720381918093BB0085E88093BD
:10691000BC00F0937203E093710380917303815084
:1069200080937303882309F422C283E0BCC1809161
:10693000B900803349F580916F03882329F4809151
:106940006C038F5F80936F0380916C03E82FFF27A8
:1069500043E0EE0FFF1F4A95E1F7ED5EF64F8381AE
:1069600099278F7790708F37910574F480916C031D
:10697000E82FFF2733E0EE0FFF1F3A95E1F7ED5EBA
:10698000F64F83818F5F838310926E0384E9809337
:10699000BC008AE090E090933D0180933C0180919F
:1069A0006C038F5F80936C0310926E03B9C180916A
:1069B000B9008034C1F180916B03E82FFF2723E0F9
:1069C000EE0FFF1F2A95E1F7ED5EF64F83818F777B
:1069D000838380916B038F5F80936B0380916B0344
:1069E0008C30A0F010926B03109265031092640338
:1069F000809170038F5F809370038C3038F0109219
:106A00007003809168038D7F809368038091680391
:106A100081608093680310926E0384E98093BC00C8
:106A200010926A0383C080916B03E82FFF2793E0E5
:106A3000EE0FFF1F9A95E1F7ED5EF64F83818068B8
:106A4000838380916B03E82FFF2783E0EE0FFF1F06
:106A50008A95E1F7ED5EF64F808180FF40C080911E
:106A60006B03E82FFF27EE0FFF1FEE0FFF1FEE0F48
:106A7000FF1FED5EF64F848199270097D1F0409774
:106A800009F04BC08BE099E09093720380937103FF
:106A900088E08093730380916B03E82FFF27EE0F4C
:106AA000FF1FEE0FFF1FEE0FFF1FED5EF64F14826C
:106AB00034C080916B039927E3E0880F991FEA9512
:106AC000E1F7885E964F90937203809371039091E3
:106AD0006B03809170039817E9F483E01CC08091E8
:106AE0006B039927880F991F880F991F880F991F8B
:106AF000885E964F90937203809371038091680330
:106B000081FD06C090916B0380917003981711F47A
:106B100082E001C081E08093730380917303813030
:106B200011F485E801C085EC8093BC0080916F036F
:106B30008093690310926F031AC1E0917103F09181
:106B400072038091BB0080838091710390917203E6
:106B50000196909372038093710380917303815027
:106B600080937303823010F085EC9AC0813011F469
:106B700085E896C08091680381FF6AC080910E0409
:106B800080FD66C080916B03E82FFF27EE0FFF1F8B
:106B9000EE0FFF1FEE0FFF1FED5EF64F8681992768
:106BA0008C7F9070883F910579F480916B03E82F7A
:106BB000FF2753E0EE0FFF1F5A95E1F7ED5EF64F0A
:106BC0008081816080830CC080916B03E82FFF2758
:106BD00043E0EE0FFF1F4A95E1F7ED5EF64F10829E
:106BE00080916B03E82FFF2733E0EE0FFF1F3A95EC
:106BF000E1F7ED5EF64F8681883F71F480916B037B
:106C0000E82FFF2723E0EE0FFF1F2A95E1F7ED5E47
:106C1000F64F808186601BC080916B03E82FFF27B1
:106C200093E0EE0FFF1F9A95E1F7ED5EF64F868138
:106C3000893F71F480916B03E82FFF2783E0EE0F0B
:106C4000FF1F8A95E1F7ED5EF64F808184608083B7
:106C500080916B038F5F80936B0380916B038C300B
:106C6000A0F010926B031092650310926403809160
:106C700070038F5F809370038C3038F01092700334
:106C8000809168038D7F8093680310926E0384E97E
:106C90008093BC008091680381608093680365C025
:106CA0008093BC0086E080936E0361C088E970CD5C
:106CB00080916D03880F805F6BCD80916D03992764
:106CC0008130910561F0823091051CF4892B21F00F
:106CD0004EC0029739F04BC080911B0159CD809175
:106CE0001A0156CD8091190153CD80E851CD1092F3
:106CF0006E0384E98093BC0010926A038AE090E0FE
:106D000090933D0180933C0180916D03823088F423
:106D100080916D038F5F80936D0382E180936E039A
:106D2000809168038E7F8093680385EA8093BC001E
:106D30001EC010926D038091680381608093680388
:106D400016C010926E0384E98093BC0080916803A2
:106D50008160809368038AE090E090933D01809386
:106D60003C0110926C0310926B0310926A03FF9126
:106D7000EF919F918F915F914F913F912F910F9044
:106D80000FBE0F901F9018951F93CF93DF93182F6E
:106D900080914604882321F48091F902882319F018
:106DA00081E090E09AC01D3008F095C01123B1F049
:106DB000E12FFF2743E0EE0FFF1F4A95E1F7ED5E5D
:106DC000F64F35978081359688230CF084C038972C
:106DD000808180FD03C083E090E07FC080910B093B
:106DE00099278B709070029719F084E090E075C03D
:106DF00067E070E08BE099E00E94322E90911209DA
:106E0000891719F085E090E068C080ED97E00E9456
:106E1000DF19EC018091680380FD05C0CE010E945E
:106E2000E8198823B9F3112319F48FEF90E00BC010
:106E3000212F33272150304081E090E002C0880F9D
:106E4000991F2A95E2F79093670380936603A1E068
:106E5000B0E0E3E1F9E040E050E06BE0CD01042E6A
:106E600002C0880F991F0A94E2F7209166033091BF
:106E7000670382239323892B11F0118212826150C0
:106E80004F5F5F4F389667FFE9CF10926C03109207
:106E90006E03809168038E7F8093680385EA8093F8
:106EA000BC008091680380FD05C0CE010E94E819F6
:106EB0008823B9F38091660390916703892B29F0A9
:106EC000CE010E94E819882311F380916603909106
:106ED0006703009711F082E090E0DF91CF911F915E
:106EE00008950F931F93CF93DF93982F80914604BB
:106EF000882321F48091F902882319F081E090E041
:106F000095C09D30A0F4992319F486E090E08EC0DE
:106F1000C92FDD27FE0153E0EE0FFF1F5A95E1F761
:106F2000ED5EF64F35978081359687FD03C082E090
:106F300090E07CC03897808180FD03C083E090E0C2
:106F400075C080ED97E00E94DF198C018091680385
:106F500080FD05C0C8010E94E8198823B9F3219774
:106F600021E030E0C90102C0880F991FCA95E2F7FD
:106F70009093650380936403D901E3E1F9E040E075
:106F800050E06BE0CD01042E02C0880F991F0A94D7
:106F9000E2F7209164033091650382239323892BC8
:106FA00011F01182128261504F5F5F4F389667FF78
:106FB000E9CF10926B0310920B09109212091092F4
:106FC0006E03809168038E7F8093680385EA8093C7
:106FD000BC008091680380FD05C0C8010E94E819CB
:106FE0008823B9F38091640390916503892B29F07C
:106FF000C8010E94E819882311F380910B09992791
:107000008B709070029719F084E090E00FC067E0F9
:1070100070E08BE099E00E94322E9091120989175E
:1070200019F085E090E002C080E090E0DF91CF9120
:107030001F910F910895CF93DF9380E021E83FEFF8
:10704000CAEBD9E0E4E7F9E0DF01853020F41196DE
:107050001C921E9202C031832083198218822296CC
:107060008F5F12963296833280F38FE790E0909391
:10707000B3098093B20981E89FEF9093B10980939F
:10708000B0091092B5091092B4091092B40410928C
:10709000B3041092B6041092B5041092B804109282
:1070A000B704DF91CF9108951F920F920FB60F9200
:1070B00011240F931F932F933F934F935F936F93DD
:1070C0007F938F939F93AF93BF93CF93DF93EF9370
:1070D000FF938091AE0882FDC2C04091860050911E
:1070E00087008091750390917603481B590B80911E
:1070F0008600909187009093760380937503CA0170
:107100008D549440A0917703B0917803835F9A41A6
:1071100058F48091770380937309149714F01092B8
:10712000400181E090E096C0A131B1050CF0F7C1BB
:10713000CA018B5F9040845B914008F086C08091CB
:107140003E0190913F01481B590BE091A508EE23A9
:1071500051F0FF27EE0FFF1FEC58F64F8081918111
:1071600084369105ECF4FD01EA0FFB1FEC58F64F55
:1071700080819181FA01E81BF90BCF01F7FF03C071
:10718000909581959F4F06975CF480914704883CC9
:1071900020F480914704865F01C088EC8093470407
:1071A000FD01EA0FFB1FEC58F64F808191819C0195
:1071B000220F331F280F391F240F351F37FF02C03E
:1071C0002D5F3F4FE901D595C795D595C795CA0164
:1071D00001968C179D0714F4219706C0415050402A
:1071E000C417D5070CF4219680914704833CE0F046
:1071F0008D010A0F1B1FF801EC58F64F8081918119
:107200009E01281B390BC90163E070E00E94DF9CDE
:10721000CB01880F991F860F971F0654164FD80170
:1072200011969C938E9307C0AA0FBB1FA654B64F0E
:1072300011961C921E92E0917703F0917803EE0F65
:10724000FF1FEC58F64FD183C08380917703909154
:1072500078030196909378038093770360C14091FF
:107260008600509187008091790390917A03481BA2
:10727000590B809186009091870090937A038093B8
:107280007903CA018D54944060910304835F9A414D
:1072900008F07AC06093740380917403843008F41A
:1072A00053C09091730980917403981709F04CC0F2
:1072B000509104045B3008F43FC0109240011092DA
:1072C000030440E05F31C0F0E42FFF27EE0FFF1F03
:1072D0009F0121543C4FDF01AC58B64F8D919C91DA
:1072E000D9018D939C93DF01A654B64F8D919C914B
:1072F000EF51FC4F91838083E42FFF27EE0FFF1F98
:107300009F012C58364FDF01A558BC4F8D919C91A1
:10731000D90111969C938E93DF01A356BC4F8D919A
:107320009C91E654F64F91838083842F8F5F482F82
:10733000813140F280930304809104048F3FB9F0BF
:107340008F5F8093040413C080910404853620F07D
:107350008AE08093040402C0109204048091030127
:107360008A3011F0843110F0289A01C0289881E009
:107370008093030480914604882309F0D0C0809153
:10738000740380937309CBC0613108F0A0C0CA01B7
:107390008B5F9040845B914008F090C080913E01EB
:1073A00090913F01481B590BE62FFF27EE0FFF1F5F
:1073B000E558FC4F80819181FA01E81BF90BCF0160
:1073C00005960B9720F5E091A508EE2351F0FF27D5
:1073D000EE0FFF1FEC58F64F8081918184369105A6
:1073E000B4F4809104048A3120F080914704865FD0
:1073F00005C08B3028F0809147048E5F809347044E
:1074000080914704893C18F088EC80934704E62F6C
:10741000FF27EE0FFF1FE558FC4F808191819C01F3
:10742000220F331F280F391F240F351F37FF02C0CB
:107430002D5F3F4FE901D595C795D595C795CA01F1
:1074400001968C179D0714F4219706C041505040B7
:10745000C417D5070CF42196809147048E3BD8F0D1
:10746000E62FFF27EE0FFF1FDF01A558BC4F8D91C0
:107470009C919E01281B390BC90163E070E00E94BA
:10748000DF9CCB01880F991F860F971FE356FC4F97
:107490009183808308C0E62FFF27EE0FFF1FE3567E
:1074A000FC4F1182108280910304E82FFF27EE0F1A
:1074B000FF1FE558FC4FD183C08309C080910301B1
:1074C0008A3011F0843110F0289A01C028988091F8
:1074D0000304843120F48F5F8093030420C084313F
:1074E000F1F4809103018A3011F0843110F0289A70
:1074F00001C028988EE18093030420E1CAEBD9E013
:10750000AFEBB3E0E4E7F9E08D919D919183808347
:107510003296198218822296215027FFF5CFFF91CB
:10752000EF91DF91CF91BF91AF919F918F917F911B
:107530006F915F914F913F912F911F910F910F90FC
:107540000FBE0F901F9018958091800A9091810A2C
:1075500090939807809397078091820A9091830A6D
:1075600090939A07809399078091560A9091570AB1
:1075700097FD0396959587959595879590939C078C
:1075800080939B078091660A9091670A97FD039606
:10759000959587959595879590939E0780939D07E0
:1075A0008091B3049091B40420913E0330913F0345
:1075B000821B930B9093A00780939F0780914104B7
:1075C00090914204A0914304B0914404BC01CD01C8
:1075D0002AE030E040E050E00E94149D3093A20782
:1075E0002093A1078091DC079091DD079093A40779
:1075F0008093A30780919001909191019093A807A7
:107600008093A70780912601909127019093AA0764
:107610008093A9078091470499279093AC078093A2
:10762000AB0780910E0A90910F0A9093AE0780935A
:10763000AD078091140999279093B0078093AF0705
:1076400080911C0999279093B2078093B10780918C
:10765000240999279093B4078093B30780912C094C
:1076600099279093B6078093B50780911403909162
:1076700015039093C0078093BF0780912B049091CE
:107680002C049093C2078093C1078091F20A9091D5
:10769000F30A9093C4078093C3078091F60A9091F0
:1076A000F70A9093C6078093C50780913D04909197
:1076B0003E04A0913F04B0914004BC01CD012AE0FA
:1076C00030E040E050E00E94149D3093C8072093C2
:1076D000C70780915F04909160049093CE078093D8
:1076E000CD078091F80A99279093D2078093D1070C
:1076F0008091190590911A059093D4078093D30730
:1077000080911705909118059093D6078093D5071F
:107710008091B105882321F48091B205882321F05E
:1077200080919607816003C0809196078E7F809339
:1077300096070895EF92FF921F93CF93DF93182F30
:107740007B0180914604882391F5809103018C3060
:1077500010F0893111F4299801C0299A11501F3F66
:10776000E9F0F0921C03E0921B03E70180911B03F8
:1077700090911C03892B11F4209781F380911F03B2
:107780008823A1F310921F0380911B0390911C0387
:10779000892B09F421970E94FF99E8CF809103017A
:1077A0008C3010F0893111F4299A01C02998DF91A9
:1077B000CF911F91FF90EF900895CF93DF93809129
:1077C00003018D3011F40E94381F10927A008091CD
:1077D0004203909143039093190A8093180A809171
:1077E00040039091410390930A0A8093090A809183
:1077F0003E0390913F0390935C0A80935B0A209133
:107800003A0330913B03C901880F991F880F991FD4
:10781000820F931F820F931F9093570A8093560AEB
:1078200020913C0330913D03C901880F991F880FB7
:10783000991F820F931F820F931F9093670A809363
:10784000660A8FEC80937A00A8E4B4E0C1E4D8E043
:1078500097E08991E82FFF27EE0FFF1FEC58F64FB6
:107860000190F081E02DE158FF4F1E161F061CF01D
:10787000E0E0F0E005C0EF3FF10514F0EFEFF0E0DD
:107880008C91282F3327E217F30714F4815004C09A
:107890002E173F0714F48F5F8C939150119697FF2A
:1078A000D8CF80917D089927AA27BB27BC01CD019D
:1078B00024EC39E040E050E00E94A09CDC01CB01C8
:1078C0008093880190938901A0938A01B0938B01E2
:1078D00080917E089927AA27BB27BC01CD010E9471
:1078E000A09CDC01CB018093840190938501A0933F
:1078F0008601B0938701DF91CF910895A0E0B0E0B9
:10790000E4E8FCE30C94339D782E91E0692ECC24BE
:10791000DD2456014601E6011092B105D092AE0475
:10792000C092AD04D092AC04C092AB04D092A80433
:10793000C092A7041092A604D092B804C092B704D3
:10794000D092B604C092B504D092B404C092B304ED
:1079500010926A0110926901109233030E94DD3B7C
:1079600084E690E00E94011A0E94DD3B8091490864
:1079700080FF14C080911C0190911D01875B934092
:1079800058F480911C0190911D018E5E924020F070
:1079900080913303882311F00E94981E00911C01EE
:1079A00010911D0187B58B5F87BD87B5809588BD18
:1079B0008FE1E82E8AE090E00E94011A80913E0358
:1079C00090913F03C80ED91E8091420390914303CA
:1079D000A80EB91E8091400390914103880E991E14
:1079E0008091DC079091DD07C80FD91FEA94E7FE6C
:1079F000E1CF80911C0190911D01825F934080F442
:107A000080911C0190911D01459750F080911C01BF
:107A100090911D01081B190B10931701009316017B
:107A200087B5855087BD87B5809588BD9501205F56
:107A30003F4F36952795369527953093B804209378
:107A4000B704C4014096969587959695879590932F
:107A5000B6048093B50440E150E0C40ED51EB5E0F5
:107A6000D694C794BA95E1F7D092B404C092B30407
:107A7000C40FD51FA5E0D695C795AA95E1F7D09379
:107A8000A804C093A7049093B2048093B1043093E8
:107A9000B0042093AF0452E07516C9F58091560AE0
:107AA0009091570A97FF03C0909581959F4F6CE086
:107AB00070E00E94DF9C9B017093AE046093AD0464
:107AC0008091660A9091670A97FF03C0909581950F
:107AD0009F4F6CE070E00E94DF9C7093AC04609359
:107AE000AB04B90184E090E00E944D306091AB049A
:107AF0007091AC0486E090E00E944D306091A70444
:107B00007091A80488E090E00E944D304FC084E05E
:107B100090E00E9448309093AE048093AD0486E0DC
:107B200090E00E9448309C019093AC048093AB0499
:107B30008091AD049091AE048150984018F421508A
:107B40003840A0F18BE199E09F938F938DE096E10F
:107B50009F938F93E0919805F091990509958091F5
:107B6000560A9091570A97FF03C0909581959F4FB1
:107B70006CE070E00E94DF9C7093AE046093AD04F3
:107B80008091660A9091670A97FF03C0909581954E
:107B90009F4F6CE070E00E94DF9C7093AC04609398
:107BA000AB0466240F900F900F900F9012BC11BC85
:107BB0001092190A1092180A10920A0A1092090AD1
:107BC00010925C0A10925B0A88EC90E00E94011A05
:107BD00080913A0390913B039C01220F331F220FA7
:107BE000331F280F391F280F391F3093570A20934E
:107BF000560A80913C0390913D038C01000F111FA8
:107C0000000F111F080F191F080F191F1093670A83
:107C10000093660A80915808C82EDD24EE24FF24C4
:107C2000442737FD4095542FC701B6010E94A09C00
:107C30004B015C016093A1047093A2048093A304A0
:107C40009093A4049801442737FD4095542FC70111
:107C5000B6010E94A09CDC01CB0180939904909313
:107C60009A04A0939B04B0939C0480928104909208
:107C70008204A0928304B092840480937904909348
:107C80007A04A0937B04B0937C0410927104109248
:107C90007204109273041092740400919001109178
:107CA00091011093600400935F0484E690E0909348
:107CB0008D0180938C0182E390E090931C0380936C
:107CC0001B0380917D089927AA27BB27BC01CD0102
:107CD00024EC39E040E050E00E94A09CDC01CB01A4
:107CE0008856954CAF4FBF4F809388019093890180
:107CF000A0938A01B0938B0180917E089927AA27CF
:107D0000BB27BC01CD010E94A09CDC01CB018856A1
:107D1000954CAF4FBF4F8093840190938501A09302
:107D20008601B09387011092470110924601C80165
:107D3000AA2797FDA095BA2F2091420130914301C7
:107D40004091440150914501BC01CD010E94A09C8D
:107D5000DC01CB018093620A9093630AA093640ACA
:107D6000B093650A10925C0410925B040E940D7639
:107D7000772029F080910E04846080930E048FEFA9
:107D80008093E20A1092E30A80E28093E40AC8E456
:107D9000D4E0A1E4B8E077E0E72E8D91E82FFF274B
:107DA000EE0FFF1FEC58F64F808191818158899327
:107DB000EA94E7FEF2CF84E68093470480911903AA
:107DC000882311F0579A17C08091AD08992780FF3A
:107DD00005C082FF03C080EE9EE202C080E091E118
:107DE00090930A018093090181E0809311010E9420
:107DF000A21A0E94A21A8091A1049091A204A091BB
:107E0000A304B091A404E0904201F09043010091DA
:107E1000440110914501BC01CD01A80197010E94C8
:107E2000149D59016A018091990490919A04A0913E
:107E30009B04B0919C04BC01CD01A80197010E9454
:107E4000149DB901C5010E94758D8C010E94837A31
:107E50009C019093230A8093220A8091A704909119
:107E6000A804AA2797FDA095BA2F6DE0880F991F47
:107E7000AA1FBB1F6A95D1F78050904FAF43B04007
:107E8000442737FD4095542FBC01CD010E94149D1D
:107E9000C90180509E4F9093A8048093A704053198
:107EA00011050CF06624772079F080910604882370
:107EB00059F0C90181599040C39730F08091B105C4
:107EC00080628093B10566248091B7049091B804D4
:107ED00080569940815C9B4228F08091B105816079
:107EE0008093B1058091B5049091B6048056994075
:107EF000815C9B4228F08091B10582608093B1053E
:107F00008091B3049091B4048C529140895795406C
:107F100028F08091B10584608093B1058091AD0413
:107F20009091AE048C529140835C914028F08091F6
:107F3000B10588608093B1058091AB049091AC0449
:107F40008C529140835C914028F08091B105806112
:107F50008093B1058091A7049091A804805092402D
:107F60008355914028F08091B10580628093B105DE
:107F70008091B1058111662486E480937F010E947F
:107F8000229582E00E94879680911E0190911F01A8
:107F9000A0912001B09121018093DE079093DF072B
:107FA000A093E007B093E1071092320310923103DF
:107FB0001092340310923503109236031092370357
:107FC000109261041092620410926304109264048F
:107FD0001092D0071092CF070E94601E862D99271D
:107FE000EEE0CDB7DEB70C944F9DA3E1B0E0EBEF30
:107FF000FFE30C942F9D8091B3049091B4042091E1
:108000003E0330913F03821B930B90935C0A809355
:108010005B0A809148039091490397FD07969C0164
:1080200053E0359527955A95E1F73093190A209337
:10803000180A809146039091470397FD079643E005
:10804000959587954A95E1F790930A0A8093090AD6
:108050003093250A2093240A90931C0A80931B0ACC
:108060008091560A9091570AAC01440F551F480F52
:10807000591F20913A0330913B03C901880F991F82
:10808000880F991F820F931F820F931F480F591F4C
:1080900057FF02C04D5F5F4F5595479555954795E2
:1080A0005093570A4093560A8091660A9091670A46
:1080B000AC01440F551F480F591F20913C033091CC
:1080C0003D03C901880F991F880F991F820F931FC5
:1080D000820F931F480F591F57FF02C04D5F5F4F1C
:1080E00055954795559547955093670A4093660A6D
:1080F00020913A0330913B03C901880F991F880FE3
:10810000991F820F931F820F931F9C01442737FDF5
:108110004095542F8091910490919204A0919304E2
:10812000B0919404820F931FA41FB51F80939104F4
:1081300090939204A0939304B093940420913C03F1
:1081400030913D03C901880F991F880F991F820F35
:10815000931F820F931F9C01442737FD4095542F96
:1081600080918D0490918E04A0918F04B091900421
:10817000820F931FA41FB51F80938D0490938E04CC
:10818000A0938F04B093900480912E0A90912F0AAF
:1081900020913A0330913B03820F931F90932F0A53
:1081A00080932E0A80915E0A90915F0A20913C0391
:1081B00030913D03820F931F90935F0A80935E0A74
:1081C0008091A9049091AA0401969093AA048093A7
:1081D000A9048091DC079091DD072091A7043091DC
:1081E000A804821B930B9C01442737FD4095542F14
:1081F0008091890490918A04A0918B04B0918C04A1
:10820000820F931FA41FB51F8093890490938A0443
:10821000A0938B04B0938C048FEC80937A0010921F
:1082200018012091790430917A0440917B04509197
:108230007C0429873A874B875C8729543B46414019
:1082400050402CF028E43BE641E050E00DC0898529
:108250009A85AB85BC85885B9449AE4FBF4F4CF483
:1082600028EB34E94EEF5FEF2D833E834F83588731
:1082700008C089859A85AB85BC858D839E83AF8335
:10828000B8872091810430918204409183045091F9
:1082900084042D873E874F87588B29543B464140A5
:1082A00050402CF028E43BE641E050E00DC08D85C5
:1082B0009E85AF85B889885B9449AE4FBF4F4CF41B
:1082C00028EB34E94EEF5FEF29833A834B835C83DD
:1082D00008C08D859E85AF85B88989839A83AB83D5
:1082E000BC83A0915B0AB0915C0ABB8BAA8BFD0199
:1082F000CF01AA2797FDA095BA2FA0907104B09046
:108300007204C0907304D0907404A80EB91ECA1EE3
:10831000DB1EA0927104B0927204C0927304D092DA
:108320007404E090620AF090630A0091640A10916C
:10833000650AE80EF91E0A1F1B1FE092620AF092FE
:10834000630A0093640A1093650AF0912A04F98B7A
:10835000FF2309F098C180912904882309F093C173
:108360008091520A86FF8FC18091090A90910A0A72
:10837000AA2797FDA095BA2FBC01CD0129813A818A
:108380004B815C810E94A09C9B01AC0197FF04C0C3
:108390002150384F4F4F5F4F6BE0559547953795BC
:1083A00027956A95D1F780916901682E77248824F2
:1083B0009924CA01B901A40193010E94A09CDC0187
:1083C000CB018093C3049093C404A093C504B093DD
:1083D000C604B7FF04C08150904FAF4FBF4F1C0180
:1083E0002D013CE055944794379427943A95D1F762
:1083F0002092C3043092C4044092C5045092C60433
:108400008091180A9091190AAA2797FDA095BA2F72
:10841000BC01CD012D813E814F8158850E94A09CD9
:1084200097FF04C06150784F8F4F9F4F2BE0959579
:108430008795779567952A95D1F7A40193010E94B6
:10844000A09CDC01CB018093C7049093C804A09347
:10845000C904B093CA04B7FF04C08150904FAF4F16
:10846000BF4F9C01AD018CE05595479537952795F9
:108470008A95D1F72093C7043093C8044093C90468
:108480005093CA048091C3049091C4049093010A4C
:108490008093000A8091C7049091C8049093050AC4
:1084A0008093040A22193309440955092093C7040B
:1084B0003093C8044093C9045093CA04E20EF31EDB
:1084C000041F151FE092620AF092630A0093640A87
:1084D0001093650A809168018823B1F457FF04C0A6
:1084E0002F5F3F4F4F4F5F4F5595479537952795D6
:1084F000A21AB30AC40AD50AA0927104B0927204F7
:10850000C0927304D09274042A893B8979010027B0
:10851000F7FC0095102F8091C7049091C804A0919A
:10852000C904B091CA04E80EF91E0A1F1B1FC80136
:10853000B70129813A814B815C810E94A09C9B01FB
:10854000AC0197FF04C02150384F4F4F5F4FBBE045
:108550005595479537952795BA95D1F780916A013A
:10856000A82EBB24CC24DD24CA01B901A6019501A3
:108570000E94A09CDC01CB018093BB049093BC04BF
:10858000A093BD04B093BE04B7FF04C08150904FC8
:10859000AF4FBF4F3C014D01ACE095948794779469
:1085A0006794AA95D1F76092BB047092BC04809244
:1085B000BD049092BE04C801B7012D813E814F8158
:1085C00058850E94A09C97FF04C06150784F8F4F40
:1085D0009F4FFBE09595879577956795FA95D1F72D
:1085E000A60195010E94A09CDC01CB018093BF04F1
:1085F0009093C004A093C104B093C204B7FF04C019
:108600008150904FAF4FBF4FAC01BD01ECE075956D
:10861000679557954795EA95D1F74093BF045093D6
:10862000C0046093C1047093C2042A893B8937FF58
:1086300003C0309521953F4F21343105E4F1D40139
:10864000C30197FE07C0B095A095909581959F4F67
:10865000AF4FBF4F81389105A105B10584F4DB010F
:10866000CA0177FF07C0B095A095909581959F4F5F
:10867000AF4FBF4F81389105A105B105E4F081E00E
:1086800080935D0418C01092050A1092040A10929B
:10869000010A1092000A1092BF041092C0041092B6
:1086A000C1041092C2041092BB041092BC04109238
:1086B000BD041092BE048091BF049091C004A091AB
:1086C000C104B091C204BC01CD0124E630E040E019
:1086D00050E00E94149DE090BB04F090BC04E21AAC
:1086E000F30AF092170AE092160A8091BB04909167
:1086F000BC04A091BD04B091BE04BC01CD0124E630
:1087000030E040E050E00E94149DDA01C901209160
:10871000BF043091C0048C01021B130B10930C0A90
:1087200000930B0A8091420190914301A091440172
:10873000B0914501BC01CD0128E631E040E050E0B8
:108740000E94A09C2091620A3091630A4091640AC1
:108750005091650A261737074807590764F0261B0A
:10876000370B480B590B2093620A3093630A4093EE
:10877000640A5093650A2091620A3091630A40911D
:10878000640A5091650A57FF0CC0260F371F481F17
:10879000591F2093620A3093630A4093640A5093EE
:1087A000650A6091090A70910A0A6E0D7F1D9B018E
:1087B000442737FD4095542F80917504909176049D
:1087C000A0917704B0917804820F931FA41FB51F66
:1087D0008093750490937604A0937704B093780403
:1087E00080912F0490913004681B790BCB01AA274C
:1087F00097FDA095BA2F29853A854B855C85820F18
:10880000931FA41FB51F8093790490937A04A093BB
:108810007B04B0937C04C0908401D0908501E090EB
:108820008601F0908701C816D906EA06FB06C4F453
:1088300088EA91E6A0E0B0E08C199D09AE09BF0975
:108840008093790490937A04A0937B04B0937C0482
:108850008093750490937604A0937704B093780482
:1088600022273327A9012C193D094E095F09809160
:10887000790490917A04A0917B04B0917C048217D2
:108880009307A407B507B4F4D701C601885A9146E7
:10889000A040B0408093790490937A04A0937B0425
:1088A000B0937C048093750490937604A09377042E
:1088B000B09378046091180A7091190A600F711FC3
:1088C0009B01442737FD4095542F80917D04909162
:1088D0007E04A0917F04B0918004820F931FA41F97
:1088E000B51F80937D0490937E04A0937F04B09382
:1088F000800480912D0490912E04681B790BCB018C
:10890000AA2797FDA095BA2F2D853E854F855889BA
:10891000820F931FA41FB51F80938104909382043C
:10892000A0938304B0938404E0908801F0908901BF
:1089300000918A0110918B01E816F9060A071B07BE
:10894000C4F488EA91E6A0E0B0E08E199F09A00B7C
:10895000B10B8093810490938204A0938304B0931D
:10896000840480937D0490937E04A0937F04B0934D
:10897000800422273327A9012E193F09400B510BF0
:108980008091810490918204A0918304B091840429
:1089900082179307A407B507B4F4D801C701885A12
:1089A0009146A040B0408093810490938204A093AC
:1089B0008304B093840480937D0490937E04A093F9
:1089C0007F04B09380048091710490917204A0910F
:1089D0007304B09174048093850490938604A093EB
:1089E0008704B09388048091810490918204A091BF
:1089F0008304B09184048093A1049093A204A09373
:108A0000A304B093A4048091790490917A04A09176
:108A10007B04B0917C048093990490939A04A09372
:108A20009B04B0939C0480917D0490917E04A0915E
:108A30007F04B091800480939D0490939E04A09342
:108A40009F04B093A0048091750490917604A09146
:108A50007704B09178048093950490939604A09342
:108A60009704B0939804809124019091250197FD7B
:108A7000079633E0959587953A95E1F79093190A13
:108A80008093180A809122019091230197FD079607
:108A900023E0959587952A95E1F790930A0A8093AC
:108AA000090A80914203909143030F9734F488E1BF
:108AB0009CEF9093190A8093180A80914203909139
:108AC0004303079734F480E398EF9093190A809357
:108AD000180A209103012A30A9F480914203909151
:108AE0004303835F934034F088EE93E09093190A38
:108AF0008093180A80914203909143038A5F9340C8
:108B0000DCF014C08091420390914303815D974053
:108B100034F088EE93E09093190A8093180A8091BC
:108B2000420390914303805E974034F080ED97E0DC
:108B30009093190A8093180A809140039091410301
:108B40000F9734F488E19CEF90930A0A8093090A06
:108B50008091400390914103079734F480E398EFAC
:108B600090930A0A8093090A2A30A9F4809140035D
:108B700090914103835F934034F088EE93E09093AB
:108B80000A0A8093090A80914003909141038A5F09
:108B90009340DCF014C08091400390914103815DCB
:108BA000974034F088EE93E090930A0A8093090A84
:108BB0008091400390914103805E974034F080EDB6
:108BC00097E090930A0A8093090A609177016623DF
:108BD00009F4AFC040912401509125018091CB044C
:108BE0009091CC04481B590B5093D2044093D1046C
:108BF0002091240130912501280F391F37FF02C031
:108C00002F5F3F4F359527953093CC042093CB04AD
:108C1000413851051CF080E890E005C040585F4F96
:108C200034F480E89FEF9093D2048093D104409174
:108C30002201509123018091CD049091CE04481BD4
:108C4000590B5093D0044093CF04209122013091CE
:108C50002301280F391F37FF02C02F5F3F4F359583
:108C600027953093CE042093CD04413851051CF054
:108C700080E890E005C040585F4F34F480E89FEFF3
:108C80009093D0048093CF04462F55278091D10430
:108C90009091D204849FB001859F700D949F700DB8
:108CA00011249B0177FF02C0215F3F4FB4E035954F
:108CB0002795BA95E1F78091180A9091190A820FC9
:108CC000931F9093190A8093180A8091CF04909172
:108CD000D004849FD001859FB00D949FB00D1124C6
:108CE000AD019D01B7FF02C0215F3F4FA4E0359564
:108CF0002795AA95E1F78091090A90910A0A820FB7
:108D0000931F90930A0A8093090A809124019091FD
:108D10002501860F971F9093250180932401809150
:108D2000220190912301840F951F9093230180933A
:108D3000220100911B0A10911C0A8091000A909157
:108D4000010A101611065CF59C0197FF04C022274A
:108D50003327281B390BC901AA2797FDA095BA2FE5
:108D600020916801332744275527BC01CD010E947B
:108D7000A09C9B01AC0197FF04C0215C3F4F4F4F6B
:108D80005F4FF6E05595479537952795FA95D1F7BA
:108D90008091160A9091170A820F931F27C097FFA0
:108DA00003C0909581959F4FAA2797FDA095BA2F54
:108DB00020916801332744275527BC01CD010E942B
:108DC000A09C9B01AC0197FF04C0215C3F4F4F4F1B
:108DD0005F4FE6E05595479537952795EA95D1F78A
:108DE0008091160A9091170A821B930B9093170A91
:108DF0008093160AE090240AF090250A8091040AD4
:108E00009091050A1E141F045CF59C0197FF04C095
:108E100022273327281B390BC901AA2797FDA095C4
:108E2000BA2F20916801332744275527BC01CD0173
:108E30000E94A09C9B01AC0197FF04C0215C3F4FA6
:108E40004F4F5F4F76E055954795379527957A9523
:108E5000D1F780910B0A90910C0A820F931F27C0C3
:108E600097FF03C0909581959F4FAA2797FDA095E6
:108E7000BA2F20916801332744275527BC01CD0123
:108E80000E94A09C9B01AC0197FF04C0215C3F4F56
:108E90004F4F5F4F66E055954795379527956A95F3
:108EA000D1F780910B0A90910C0A821B930B90933F
:108EB0000C0A80930B0A8091520A87FF44C0B9893B
:108EC000BB2309F040C0809129048823E1F5E1E04B
:108ED000EE16E1E0FE064CF08091180A9091190A16
:108EE0008E0D9F1D805091400DC0F0E0EF16FFEFFA
:108EF000FF0664F48091180A9091190A8E0D9F1D47
:108F000080509F4F9093190A8093180A21E00130F6
:108F100012074CF08091090A90910A0A800F911F64
:108F2000805091400CC03FEF0030130764F48091F3
:108F3000090A90910A0A800F911F80509F4F9093C9
:108F40000A0A8093090AE2E1CD5E0C944B9D809160
:108F50004604882329F580910E048C7F80930E04AB
:108F600080910D048F7D80930D04A6EBB5E0E3E1C5
:108F7000F9E09BE08091F902882309F48C938D91AC
:108F8000818312829150389697FFF4CF8091F90235
:108F9000882359F08091F90281508093F90205C02D
:108FA00080910E04816080930E0480916A0388236F
:108FB00019F010926A03089580936C0380936E03F6
:108FC000809168038E7F8093680385EA8093BC005C
:108FD0000895882319F480E090E00895E82FFF2792
:108FE000EE0FFF1FEC58F64F8081918181589F4F03
:108FF0008F3F910521F01CF08FEF90E004C097FFA8
:1090000002C080E090E099270895CF93DF93A8E411
:10901000B4E0C1E4D8E057E08991E82FFF27EE0FD4
:10902000FF1FEC58F64F0190F081E02DE158FF4F03
:10903000EF3FF10521F01CF0EFEFF0E004C0F7FF87
:1090400002C0E0E0F0E0893111F4EC931BC04C91D8
:10905000242F3327E217F307A9F0CF01821B930BCC
:1090600097FD03969595879595958795242F280FBD
:109070002C93822F9927E817F90714F4215001C087
:109080002F5F2C935150119657FFC6CF80914B08FC
:10909000883F38F0EFEFF0E0E81BF109E85BFB4FA9
:1090A000808180937C0180917C01882329F0843623
:1090B00018F084E680937C0180914D08883F38F059
:1090C000EFEFF0E0E81BF109E85BFB4F8081809354
:1090D0007B0180917B01882329F0843618F084E697
:1090E00080937B0180915A08883F38F0EFEFF0E0E1
:1090F000E81BF109E85BFB4F80818093760180914A
:1091000076018B3010F48AE002C08F3F11F4809317
:10911000760180918708883F38F0EFEFF0E0E81B98
:10912000F109E85BFB4F80818093300A8091300A1F
:10913000863010F485E002C08F3F11F48093300A2E
:1091400080918908883F38F0EFEFF0E0E81BF109E3
:10915000E85BFB4F80818093590A8091590A8630E1
:1091600010F485E002C08F3F11F48093590A80917A
:109170007408873F19F4429905C006C0863F31F450
:10918000439B02C08CE815C086E413C0883F38F0CA
:10919000EFEFF0E0E81BF109E85BFB4F8081809383
:1091A0002D0A80912D0A893110F488E102C08F3F89
:1091B00011F480932D0A80917508873F19F4429924
:1091C00005C006C0863F31F4439B02C08CE815C041
:1091D00086E413C0883F38F0EFEFF0E0E81BF109B8
:1091E000E85BFB4F80818093060A8091060A8931F3
:1091F00010F488E102C08F3F11F48093060A809139
:109200007608883F38F0EFEFF0E0E81BF109E85B03
:10921000FB4F80818093360A8091360A893110F4A1
:1092200088E102C08F3F11F48093360A80914C0888
:109230000E94E9478093240480914F08883F38F0CA
:10924000EFEFF0E0E81BF109E85BFB4F80818093D2
:109250007A0180915108883F38F0EFEFF0E0E81B89
:10926000F109E85BFB4F8081809378018091590878
:10927000883F38F0EFEFF0E0E81BF109E85BFB4FC7
:1092800080818093790180915B08883F38F0EFEF0F
:10929000F0E0E81BF109E85BFB4F808180937501EA
:1092A00080915C08883F38F0EFEFF0E0E81BF109AF
:1092B000E85BFB4F80818093770180915D08883F58
:1092C00038F0EFEFF0E0E81BF109E85BFB4F80813D
:1092D0008093740180915E08883F38F0EFEFF0E0F2
:1092E000E81BF109E85BFB4F80818093730180915B
:1092F0006408883F38F0EFEFF0E0E81BF109E85B25
:10930000FB4F80818093710180916508883F38F020
:10931000EFEFF0E0E81BF109E85BFB4F8081809301
:10932000230480916608883F38F0EFEFF0E0E81BF7
:10933000F109E85BFB4F80818093220480916708EC
:10934000883F38F0EFEFF0E0E81BF109E85BFB4FF6
:1093500080818093210480916808883F38F0EFEF86
:10936000F0E0E81BF109E85BFB4F8081809320046B
:1093700080918208883F38F0EFEFF0E0E81BF109B8
:10938000E85BFB4F808180931F0480918308883FB6
:1093900038F0EFEFF0E0E81BF109E85BFB4F80816C
:1093A00080931E0480918408883F38F0EFEFF0E04E
:1093B000E81BF109E85BFB4F808180931D048091DD
:1093C0008508883F38F0EFEFF0E0E81BF109E85B33
:1093D000FB4F808180931C0480916908883F38F09E
:1093E000EFEFF0E0E81BF109E85BFB4F8081809331
:1093F0006F0180916D08883F38F0EFEFF0E0E81BD7
:10940000F109E85BFB4F808180936E0180916A08CF
:10941000883F38F0EFEFF0E0E81BF109E85BFB4F25
:10942000808180936D0180916E08883F38F0EFEF66
:10943000F0E0E81BF109E85BFB4F808180936C0151
:1094400080917708883F38F0EFEFF0E0E81BF109F2
:10945000E85BFB4F808180936B0180917A08883FA5
:1094600038F0EFEFF0E0E81BF109E85BFB4F80819B
:1094700080936A0180917B08883F38F0EFEFF0E03D
:10948000E81BF109E85BFB4F8081809369018091C3
:109490007C08883F38F0EFEFF0E0E81BF109E85B6B
:1094A000FB4F8081809368018091A408883F38F049
:1094B000EFEFF0E0E81BF109E85BFB4F8081809360
:1094C000150A90912305992321F08091150A981788
:1094D00020F08091150A882311F49093150A809149
:1094E00049088093520A8091AE088093350A809192
:1094F0008108883F38F0EFEFF0E0E81BF109E85B06
:10950000FB4F80818093670180919D08883F38F0F0
:10951000EFEFF0E0E81BF109E85BFB4F80818093FF
:10952000690A80917101282F33272F5F3F4F8CE309
:1095300098E2B9010E94DF9C70937E0160937D01E7
:109540008091570880935A0A8091560880931D0A8B
:10955000E0919F08EE2309F449C081E080931B0449
:10956000FF27EE0FFF1FEC58F64F80819181805C42
:109570009F4F14F410921B0480917F0120911B04D3
:10958000821721F18330F8F43091AA01222351F09F
:109590008CED95E090931C0380931B03332369F4B7
:1095A0008EE209C088EC90E090931C0380931B032B
:1095B000332319F487E18093AA0185E08093310475
:1095C00020937F0103C0815080937F018091A90A7D
:1095D0009091AA0A97FF0FC080911B04882359F02D
:1095E0008091B10580688093B10505C0E0931B04AC
:1095F0008AE080937F018091A90A9091AA0A97FF3F
:109600001DC0809146048823C9F080911B048823E3
:10961000A9F080910B0190910C018F5F9F4F71F425
:1096200088E99AE390931C0380931B0380E094EAFB
:1096300090930C0180930B0110921B0480911B04EA
:10964000882321F080910D04816003C080910D0476
:109650008E7F80930D04DF91CF910895A8E1B0E053
:10966000E4E3FBE40C942F9D0E94F53F80910E04EF
:10967000992784719070892B91F58091AF0882FFB2
:1096800027C080912B0490912C040097F1F002E008
:1096900088359007D4F49C0197FF02C02D5F3F4F9F
:1096A0003595279535952795809161089927289FAD
:1096B000A001299F500D389F500D1124CA0164E666
:1096C00070E00E94DF9CCB0106C08DE290E003C0F9
:1096D00080916108992790930C0480930B0420914A
:1096E000090430910A0455E72033350759F41092E4
:1096F00052041092510480911D0A992790930C04F2
:1097000080930B0460915104709152047A836983B1
:1097100080911D0A99270A966817790714F49A838D
:10972000898380914704843608F06AC080910D04D3
:1097300082FD66C08091E7049091E804009731F0C3
:1097400001979093E8048093E7040BC010924604BD
:109750009093100480930F0480910E048D7E80936B
:109760000E04809103018A3011F0843110F0289AA0
:1097700001C0289880910F0490911004895E934055
:10978000E0F18091F80A8536C0F180910B04909148
:109790000C049A83898380910E04806180930E0467
:1097A00080913D08A82FBB27AA0FBB1FFD01E654DF
:1097B000F64F1182108280913E08282F3327220F06
:1097C000331FC9018654964FFC0111821082AC5898
:1097D000B64F11961C921E922C58364FD9011196F5
:1097E0001C921E9280914008E82FFF27EE0FFF1F6A
:1097F000EC58F64F11821082B4C510924604B1C5E0
:10980000809147048D3808F482C59091A808992367
:1098100009F445C08091A908882309F440C0E92FC4
:10982000FF27EE0FFF1FEC58F64F80819181C39701
:10983000BCF080919401823361F480910D0485FF26
:1098400008C080910D04806480930D0480E38093B0
:10985000AA0180910D048F7780930D0486E917C0CB
:10986000808191818E5C9F4FACF480919401863908
:1098700041F480910D04806880930D048FE2809301
:10988000AA0180910D048F7B80930D0482E3809365
:10989000940105C080910D048F7380930D04809115
:1098A0000E048F7E80930E049091620882E3989F4D
:1098B000C00111249093E8048093E704E981FA81C0
:1098C000B9978CF080914604882369F080910F0449
:1098D00090911004FFEF8F3F9F0729F0019690931E
:1098E000100480930F0440910F04509110044F3FD7
:1098F000510509F048F51092690410926A0410921B
:109900006B0410926C04109265041092660410921D
:109910006704109268041092D3041092D404109239
:10992000D5041092D6041092710410927204109211
:1099300073041092740480910D04806280930D046E
:1099400084E68093940135C180910E0482608093F7
:109950000E0480910D0485FF98C0809124059927FD
:109960009C012470307082FD04C080910D0486FF3C
:109970002AC0809141018D3331F5809106048823FE
:1099800011F180E58093360484EF91E0A0E0B0E02F
:109990008093370490933804A0933904B0933A0429
:1099A00080933D0490933E04A0933F04B093400401
:1099B00088EE93E09093930180939201232B19F00A
:1099C0008DE08093AA018091270390912803A091B4
:1099D0002903B0912A0387399105A105B1058CF4BB
:1099E0008091410490914204A0914304B0914404B9
:1099F000825A9E4FAF4FBF4F24F08091520A80FD94
:109A000021C088EE93E0909393018093920180911E
:109A10000D0486FF0FC0109236048CE291E0A0E0A6
:109A2000B0E080933D0490933E04A0933F04B09334
:109A3000400403C080E38093AA0180910D048F71DC
:109A400080930D041092690410926A0410926B04C2
:109A500010926C04109265041092660410926704D0
:109A600010926804109271041092720410927304A0
:109A700010927404495E534008F49BC088EE93E052
:109A80009093100480930F0494C080910D0487FF7D
:109A90001AC080914101863711F08D33A1F4809175
:109AA0000604882381F08091A9088093360480EE13
:109AB00091EBAFEFBFEF8093370490933804A093FE
:109AC0003904B0933A04209192013091930143E01C
:109AD000283E340708F048C02F5F3F4F3093930172
:109AE000209392011092690410926A0410926B0400
:109AF00010926C0410926504109266041092670430
:109B000010926804109271041092720410927304FF
:109B1000109274048091270390912803A091290347
:109B2000B0912A038C529140A040B04080933D04F4
:109B300090933E04A0933F04B0934004285E3340CA
:109B4000C1F580910D0487FF34C0809141018B32B3
:109B500081F180910D048F7780930D0480910D0425
:109B6000806280930D0425C080910604882309F14A
:109B700080914101863711F08D32D9F480914104F2
:109B800090914204A0914304B0914404885E9340B4
:109B9000A040B04074F48091DC079091DD078D5AAD
:109BA00093403CF010929301109292018EE08093CA
:109BB000AA0180913F08E82FFF27EE0FFF1FEC5806
:109BC000F64F80819181813591050CF454C120912B
:109BD0004604222309F04FC180914008E82FFF2757
:109BE000EE0FFF1FEC58F64F808191818C34910568
:109BF0000CF411C18091E9048F5F8093E904893CE2
:109C000008F439C12093E9041092100410920F0453
:109C100030913D08E32FFF27EE0FFF1FEC58F64F62
:109C20008081918187349105B4F480913E08E82FBA
:109C3000FF27EE0FFF1FEC58F64F808191810190B6
:109C4000F081E02DF7FF03C0F095E195FF4FE73479
:109C5000F1050CF478C041E020913E08A22FBB270B
:109C6000AA0FBB1FAC58B64F8D919C9111978734AA
:109C7000910544F0E32FFF27EE0FFF1FEC58F64F3E
:109C8000808191818D919C918734910574F08091B0
:109C90003D08E82FFF27EE0FFF1FEC58F64F80819D
:109CA0009181873491050CF042E0E22FFF27EE0FFF
:109CB000FF1FEC58F64F808191818634910574F432
:109CC00080913D08E82FFF27EE0FFF1FEC58F64F5D
:109CD00080819181873491050CF043E0E22FFF27CA
:109CE000EE0FFF1FEC58F64F808191818A5B9F4FEA
:109CF00074F480913D08E82FFF27EE0FFF1FEC580A
:109D0000F64F80819181873491050CF044E0E22F79
:109D1000FF27EE0FFF1FEC58F64F808191818A5B81
:109D20009F4F74F480913D08E82FFF27EE0FFF1F2F
:109D3000EC58F64F80819181863491050CF445E012
:109D4000842F0E94A73080913E08E82FFF27EE0F56
:109D5000FF1FEC58F64F808191810190F081E02D3A
:109D6000F7FF03C0F095E195FF4F7E97CCF480910B
:109D70003D08E82FFF27EE0FFF1FEC58F64F8081BC
:109D800091818A5B9F4F64F481E08093CC051092AF
:109D9000320488EE93E090931C0380931B036BC006
:109DA000809101010E94523080E00E94D20980918E
:109DB00063080E944F988091520A80FF10C08091E2
:109DC0001C0190911D01875B934038F480911C0128
:109DD00090911D018E5E924010F40E94981E81E0C9
:109DE0000E947E3C982F8093320421E02093190337
:109DF000579A8091B105882311F087E006C0992316
:109E000019F42093AA0103C088E18093AA0185E098
:109E100080934E0527C080819181855B9F4F4CF5D3
:109E20008091E9048F5F8093E904893C20F12093BD
:109E300046042093E9041092100410920F0482E06B
:109E40000E947E3C982F809332048091B105882334
:109E500011F087E005C0992311F481E001C088E189
:109E60008093AA0168E770E0809101010E949A3B0B
:109E700002C02093E90480913F08E82FFF27EE0FEE
:109E8000FF1FEC58F64F808191818C599F4F0CF049
:109E900037C22091A008E22FFF27EF77F070EE0F76
:109EA000FF1FE654F64F80819181069714F084E6F7
:109EB00006C0808191818B5F9F4F1CF48CE9809359
:109EC000EC0480914604E0914008882309F063C1C6
:109ED000FF27EE0FFF1FEC58F64F808191818C59C0
:109EE0009F4F9CF48091AF0883FD0BC0E22FFF27AA
:109EF000EE0FFF1FEC58F64F80819181855B9F4FDD
:109F0000DCF08091A0088823B9F08091AF0883FF2E
:109F10003FC18091A008E82FFF27EE0FFF1FEC58EC
:109F2000F64F80819181875F9F4F0CF431C1809102
:109F3000EC04843609F02CC180913204882329F086
:109F400080910E04886080930E0480911E01909190
:109F50001F01A0912001B09121018093DE07909311
:109F6000DF07A093E007B093E10710922703109258
:109F700028031092290310922A0310924104109290
:109F8000420410924304109244041092340310923D
:109F90003503109236031092370380913D08E82F65
:109FA000FF27EE0FFF1FEC58F64F808191818D59EE
:109FB0009F4FACF480913E08E82FFF27EE0FFF1F64
:109FC000EC58F64F808191810190F081E02DF7FFF0
:109FD00003C0F095E195FF4FE436F10534F480912C
:109FE000A008882311F48093EA048091EA048F5F2B
:109FF0008093EA048E3F08F466C180915B0A9091D9
:10A000005C0A97FF03C0909581959F4F8197B4F4A8
:10A010008091180A9091190A97FF03C09095819535
:10A020009F4F45975CF48091090A90910A0A97FF27
:10A0300003C0909581959F4F459714F0109232047C
:10A040001092EA048091B105882309F094C08091B0
:10A050003204882309F48FC080912805882309F0F1
:10A060008AC081E090E09093100480930F0481E017
:10A07000809346041092D3041092D4041092D50415
:10A080001092D6041092710410927204109273040C
:10A090001092740410926D0410926E0410926F046A
:10A0A0001092700480915808E82EFF240027112791
:10A0B0008091560A9091570A9C01442737FD40959C
:10A0C000542FC801B7010E94A09CDC01CB018093F2
:10A0D000810490938204A0938304B09384048091BC
:10A0E000660A9091670A9C01442737FD4095542FDA
:10A0F000C801B7010E94A09CDC01CB0180937904C8
:10A1000090937A04A0937B04B0937C048091A10483
:10A110009091A204A091A304B091A40480937D0423
:10A1200090937E04A0937F04B0938004809199045F
:10A1300090919A04A0919B04B0919C048093750423
:10A1400090937604A0937704B093780410926904F6
:10A1500010926A0410926B0410926C0410926504C1
:10A1600010926604109267041092680484E680934B
:10A17000310484E39AC08CED95E090931C038093A6
:10A180001B0380913204882309F09DC081E08DC0BB
:10A190001092EA0498C0FF27EE0FFF1FEC58F64F0D
:10A1A00080819181853691059CF08091AF0883FD77
:10A1B0000BC0E22FFF27EE0FFF1FEC58F64F8081F8
:10A1C0009181855B9F4FDCF08091A0088823B9F0D6
:10A1D0008091AF0883FF75C08091A008E82FFF270A
:10A1E000EE0FFF1FEC58F64F808191818E5C9F4FE0
:10A1F0000CF067C08091EC048C3909F062C080914A
:10A200003D08E82FFF27EE0FFF1FEC58F64F808127
:10A2100091818D599F4FACF480913E08E82FFF2724
:10A22000EE0FFF1FEC58F64F808191810190F08175
:10A23000E02DF7FF03C0F095E195FF4FE436F105FF
:10A240003CF48091A008882319F48093EB0418C093
:10A250001092690410926A0410926B0410926C04BC
:10A2600010926504109266041092670410926804BC
:10A2700010925804109257041092560410925504EC
:10A280008091EB048F5F8093EB048B3F88F01092FA
:10A2900046041092EB041092100410920F04809167
:10A2A0000D048F7180930D0486E28093AA010BC088
:10A2B000843649F48CEA9DE090931C0380931B0341
:10A2C00002C01092EB042091090430910A04F3E0DB
:10A2D000283E3F0708F045C080913103909132033A
:10A2E0008B569F4F1CF02F5F3F4F05C02115310546
:10A2F000C1F12150304030930A042093090431C049
:10A300001092EC0410920A04109209042AC02E5EE6
:10A31000324038F18091710A9091720A80599140CF
:10A3200000F58091410490914204A0914304B091C2
:10A3300044048C5D9540A040B0409CF480E395E7D8
:10A3400090930A048093090480910F049091100463
:10A350008A5E934030F089EE93E0909310048093EE
:10A360000F04809140018150809340018091400111
:10A370008F3F21F080910E0484FFDFC30E940548C7
:10A38000B09053088091F5049091F6049C01220F3F
:10A39000331F280F391FC0903D08AC2DBB27AA0FD3
:10A3A000BB1FFD01EC58F64F4B2D55278081918145
:10A3B000849FB001859F700D949F700D1124260F0E
:10A3C000371F37FF02C02D5F3F4FB9017595679565
:10A3D00075956795A654B64F80915408082F11279C
:10A3E0008D919C91809FD001819FB00D909FB00D69
:10A3F00011246A0F7B1F7093F6046093F50480911B
:10A40000F7049091F8049C01220F331F280F391F85
:10A41000D0903E08AD2DBB27AA0FBB1FFD01EC5805
:10A42000F64F80819181849FF001859FF00D949F6C
:10A43000F00D11242E0F3F1F37FF02C02D5F3F4F3D
:10A44000A9015595479555954795A654B64F8D91B9
:10A450009C91809F7001819FF00C909FF00C1124C3
:10A460004E0D5F1D5093F8044093F70480911B0438
:10A47000882309F448C0CB0177FD0396DC01B5952C
:10A48000A795B595A795CA0157FD0396FC01F595CB
:10A49000E795F595E7958091A501682F772767FDEA
:10A4A00070956A9F90016B9F300D7A9F300D11243B
:10A4B00080912A05482F552747FD50954E9FC00192
:10A4C0004F9F900D5E9F900D1124280F391F37FF6D
:10A4D00002C0295F3F4F03E0359527950A95E1F7C4
:10A4E00030935804209357046E9F90016F9F300D56
:10A4F0007E9F300D11244A9FC0014B9F900D5A9FA3
:10A50000900D11243FC080919E08E82FFF27E85B43
:10A51000FE4F86818093A501908190932A05A82FF4
:10A52000BB27A7FDB095A69F9001A79F300DB69FB2
:10A53000300D1124E92FFF27E7FDF095E49FC001BE
:10A54000E59F900DF49F900D1124280F391F37FFC0
:10A5500002C0295F3F4F13E0359527951A95E1F723
:10A560003093580420935704A49F9001A59F300D69
:10A57000B49F300D1124E69FC001E79F900DF69F18
:10A58000900D1124281B390B37FF02C0295F3F4F64
:10A5900043E0359527954A95E1F73093560420938B
:10A5A000550480914008E82FFF27EE0FFF1FEC585D
:10A5B000F64F80819181909581959F4F909354049F
:10A5C000809353048530910514F0049705C00FEF74
:10A5D0008C3F900734F40496909354048093530472
:10A5E00004C0109254041092530480910904909175
:10A5F0000A048150924078F1809157049091580458
:10A6000097FD079623E0959587952A95E1F7909316
:10A61000580480935704809155049091560497FDF7
:10A62000079603E0959587950A95E1F79093560470
:10A63000809355041092690410926A0410926B047E
:10A6400010926C04109265041092660410926704D4
:10A650001092680443C080911605882309F43EC017
:10A66000282F3327809157049091580497FD07961F
:10A6700013E0959587951A95E1F7289FA001299FEA
:10A68000500D389F500D1124CA0157FD0F96B4E0AC
:10A6900095958795BA95E1F7909358048093570460
:10A6A000809155049091560497FD0796A3E09595E7
:10A6B0008795AA95E1F7289FB001299F700D389FD3
:10A6C000700D1124CB0177FD0F96F4E095958795D9
:10A6D000FA95E1F7909356048093550480905704BF
:10A6E000909058048091190590911A05881A990A3A
:10A6F000909258048092570400915504109156048A
:10A700008091170590911805081B190B109356049A
:10A710000093550480913F08E82FFF27EE0FFF1F9D
:10A72000EC58F64FE080F1808FE790E0E80EF91EDC
:10A73000F0925204E0925104809176019927AA2761
:10A7400097FDA095BA2FBC01CD010E94149CDC019D
:10A75000CB0120E030E040E251E4BC01CD010E9499
:10A76000829BDC01CB01BC01CD010E94E69BDC0198
:10A77000CB018093600A809175018093370A8091A4
:10A7800074019927AA2797FDA095BA2FBC01CD0186
:10A790000E94149CDC01CB0120E030E040E251E457
:10A7A000BC01CD010E94829BDC01CB01BC01CD012B
:10A7B0000E94E69BDC01CB018093100A809173011B
:10A7C0008093260A8091D80580FF59C08091690A3C
:10A7D000813808F454C08091D105992787FD909560
:10A7E0002B2D3327829FD001839FB00D929FB00DF8
:10A7F00011248A0E9B1E90925804809257048091D7
:10A80000D205992787FD9095829FF001839FF00DD7
:10A81000929FF00D11240E0F1F1F109356040093EA
:10A8200055048091D305282F332727FD309580913B
:10A83000530490915404820F931F90935404809377
:10A8400053048091D505282F332727FD309580911B
:10A850004E089927289F8001299F100D389F100DC1
:10A86000112410934701009346018091D405992744
:10A870008E159F0524F49093520480935104809187
:10A8800051049091520497FF04C010925204109208
:10A8900051048091520A82FF02C01092370A4091FF
:10A8A000570450915804CA0157FD03969C013595F1
:10A8B00027953595279537FF03C0309521953F4F54
:10A8C000809113049091140482179307B4F4CA0181
:10A8D00057FF03C0909581959F4F97FD03969595DF
:10A8E00087959595879590931404809313048536E6
:10A8F000910544F084E690E001C001979093140420
:10A90000809313044091550450915604CA0157FD99
:10A9100003969C01359527953595279537FF03C0FC
:10A92000309521953F4F8091110490911204821728
:10A930009307B4F4CA0157FF03C0909581959F4FC8
:10A9400097FD039695958795959587959093120415
:10A95000809311048536910544F084E690E001C0AF
:10A960000197909312048093110480910E0484FF48
:10A9700008C0109214041092130410921204109242
:10A980001104ED2DFF27EE0FFF1FEC58F64F4091FD
:10A990007808242F3327808191812817390744F4C0
:10A9A0008091AC0882FF04C081E08093280413C02A
:10A9B000ED2DFF27EE0FFF1FEC58F64F842F992740
:10A9C00020917908821B910920813181281739074C
:10A9D00014F41092280440913E08E42FFF27EE0F54
:10A9E000FF1FEC58F64F50917808852F99272227A2
:10A9F0003327281B390B808191818217930744F4F8
:10AA00008091AC0883FF04C081E08093270416C0C6
:10AA100080912704882391F0E42FFF27EE0FFF1F7A
:10AA2000EC58F64F809179089927851B9109208170
:10AA300031818217930714F410922704EC2DFF271D
:10AA4000EE0FFF1FEC58F64F40917808242F332764
:10AA5000808191812817390744F48091AC0880FFE8
:10AA600004C081E08093250417C0809125048823C9
:10AA700099F0EC2DFF27EE0FFF1FEC58F64F842FB7
:10AA8000992720917908821B91092081318128170B
:10AA9000390714F41092250440913D08E42FFF2754
:10AAA000EE0FFF1FEC58F64F50917808852F99272D
:10AAB00022273327281B390B808191818217930726
:10AAC00044F48091AC0881FF04C081E080932604A7
:10AAD00016C080912604882391F0E42FFF27EE0F03
:10AAE000FF1FEC58F64F809179089927851B910933
:10AAF000208131818217930714F4109226048091EB
:10AB00002804882319F480912704811181E080931F
:10AB1000290480912504882321F480912604882328
:10AB200051F081E080932A041092290410922804A5
:10AB30001092270402C080932A048091290488235C
:10AB400021F480912A04882369F08091770899275D
:10AB500029813A818217930714F49A83898381E0CB
:10AB600080935D0480910D0499279C0124703070BE
:10AB700082FF2DC08091190590911A0590958195BD
:10AB80009F4F90935804809357048091170590919C
:10AB90001805909581959F4F909356048093550486
:10ABA000809182019091830190935204809351048B
:10ABB0008091520A8B778B668093520A8091350A76
:10ABC0008C7B8093350A88EC809324041EC080918E
:10ABD0000E0484FF1AC0309354042093530430931E
:10ABE00058042093570430935604209355049AE553
:10ABF0009093600A88E78093370A9093100A8093B5
:10AC0000260A1092290410922A048091290A909110
:10AC10002A0AA0912B0AB0912C0A2091A10430910C
:10AC2000A2044091A3045091A404820F931FA41F77
:10AC3000B51F8093290A90932A0AA0932B0AB093F8
:10AC40002C0A8091310A9091320AA091330AB09176
:10AC5000340AE0909904F0909A0400919B041091BA
:10AC60009C04EB82FC820D831E838E0D9F1DA01F12
:10AC7000B11F8093310A9093320AA093330AB093A4
:10AC8000340A80911E0A90911F0AA091200AB09167
:10AC9000210AE0909D04F0909E0400919F04109181
:10ACA000A004EF82F88609871A878E0D9F1DA01FCA
:10ACB000B11F80931E0A90931F0AA093200AB0939D
:10ACC000210A8091110A9091120AA091130AB09161
:10ACD000140AE0909504F090960400919704109166
:10ACE0009804EB86FC860D871E878E0D9F1DA01F86
:10ACF000B11F8093110A9093120AA093130AB09384
:10AD0000140AF0902A04FF86FF2029F48091290478
:10AD1000882309F460C0109291041092920410925A
:10AD200093041092940410928D0410928E04109249
:10AD30008F04109290041092290A10922A0A1092FD
:10AD40002B0A10922C0A1092310A1092320A109299
:10AD5000330A1092340A10921E0A10921F0A10929F
:10AD6000200A1092210A1092110A1092120A1092CF
:10AD7000130A1092140A8091810490918204A09188
:10AD80008304B091840480937D0490937E04A09307
:10AD90007F04B09380048091790490917A04A0910B
:10ADA0007B04B0917C048093750490937604A09307
:10ADB0007704B09378041092300310922F0310920E
:10ADC0002E0410922D041092300410922F040F853F
:10ADD000002309F0D0C180912904882309F0CBC158
:10ADE0008091DC079091DD07815092402CF4809196
:10ADF0004604882309F4BFC19090E20AA090580845
:10AE00002090560A3090570A4090660A5090670A80
:10AE100019140CF0BBC0BB24CC24DD24CA01B90139
:10AE2000A60195010E94149D79018A018091AB0AC7
:10AE30009091AC0A281A390AC101AA2797FDA0955A
:10AE4000BA2FE81AF90A0A0B1B0B6B817C818D81E2
:10AE50009E81A60195010E94149D59016A0180916D
:10AE6000AD0A9091AE0A481A590AC201AA2797FD65
:10AE7000A095BA2FA81AB90ACA0ADB0A292C3324CA
:10AE800027FC3094432C532CC801B701A201910137
:10AE90000E94A09C97FF04C061507E4F8F4F9F4F30
:10AEA0003B014C0109E095948794779467940A9547
:10AEB000D1F7C601B501A20191010E94A09C97FFA4
:10AEC00004C061507E4F8F4F9F4F5B016C0119E0B2
:10AED000D594C794B794A7941A95D1F78091130489
:10AEE00090911404813491053CF480911104909167
:10AEF000120481349105D4F0D401C30197FE03C03C
:10AF00000196A11DB11D3C014D0195948794779444
:10AF10006794D601C501D7FE03C00196A11DB11DDE
:10AF20005C016D01D594C794B794A7948091E40A0D
:10AF3000282F332727FD3095432F532F261537050C
:10AF40004805590514F439014A01992787FD909560
:10AF5000909581959F4FAA2797FDA095BA2F6816C7
:10AF600079068A069B0614F43C014D012A153B051F
:10AF70004C055D0514F459016A01A816B906CA0604
:10AF8000DB060CF0D0C05C016D01CDC0EA2CFF24C3
:10AF900000271127CA01B901A80197010E94149D39
:10AFA00039014A01C101AA2797FDA095BA2F681A55
:10AFB000790A8A0A9B0A6B817C818D819E81A80116
:10AFC00097010E94149D59016A01C201AA2797FDA9
:10AFD000A095BA2FA81AB90ACA0ADB0AD401C3017C
:10AFE00097FE03C00F96A11DB11D3C014D01F4E079
:10AFF0009594879477946794FA95D1F7D601C50113
:10B00000D7FE03C00F96A11DB11D5C016D01E4E0E8
:10B01000D594C794B794A794EA95D1F78091130477
:10B0200090911404813491053CF480911104909125
:10B03000120481349105A4F0C401B30123E030E08F
:10B0400040E050E00E94149D39014A01C601B5015B
:10B0500023E030E040E050E00E94149D59016A0175
:10B0600080914008E82FFF27EE0FFF1FEC58F64FA6
:10B07000808191810190F081E02DF7FF03C0F09570
:10B08000E195FF4F7A97A4F0C401B30123E030E0CB
:10B0900040E050E00E94149D39014A01C601B5010B
:10B0A00023E030E040E050E00E94149D59016A0125
:10B0B00089E180938E0121E262167104810491047A
:10B0C0002CF070E2672E712C812C912C30EE6316DF
:10B0D0003FEF73063FEF83063FEF930644F460EEC5
:10B0E000662E6FEF762E6FEF862E6FEF962E41E273
:10B0F000A416B104C104D1042CF050E2A52EB12C49
:10B10000C12CD12C50EEA5165FEFB5065FEFC5063A
:10B110005FEFD50644F440EEA42E4FEFB42E4FEF70
:10B12000C42E4FEFD42E8091810490918204A0917F
:10B130008304B091840486199709A809B9098093FA
:10B14000810490938204A0938304B093840480913B
:10B15000790490917A04A0917B04B0917C048A19BF
:10B160009B09AC09BD098093790490937A04A0935C
:10B170007B04B0937C0480912F03909130038F3F28
:10B18000910509F008F4C4C56F85662309F04EC522
:10B1900080912904882309F049C580915D048823A2
:10B1A00009F044C570918008788B772309F43EC577
:10B1B0008091290A90912A0AA0912B0AB0912C0A19
:10B1C000B7FF04C081509F4FAF4FBF4FE92EFA2EFB
:10B1D0000B2F112707FD1A95E092290AF0922A0AEF
:10B1E00000932B0A10932C0A8091310A9091320A15
:10B1F000A091330AB091340AB7FF04C081509F4F29
:10B20000AF4FBF4F892F9A2FAB2FBB27A7FDBA9502
:10B21000898B9A8BAB8BBC8B8093310A9093320ACB
:10B22000A093330AB093340A80915808A82EBB2407
:10B23000CC24DD2420919104309192044091930418
:10B2400050919404C601B5010E94A09C97FF04C0D0
:10B2500061507F4F8F4F9F4F672E782E892E9924F4
:10B2600087FC9A9460929104709292048092930465
:10B270009092940420918D0430918E0440918F041B
:10B2800050919004C601B5010E94A09C97FF04C094
:10B2900061507F4F8F4F9F4F272E382E492E5524B8
:10B2A00047FC5A9420928D0430928E0440928F0471
:10B2B000509290048091890490918A04A0918B040B
:10B2C000B0918C04B7FF04C081509F4FAF4FBF4F68
:10B2D000892F9A2FAB2FBB27A7FDBA95809389049E
:10B2E00090938A04A0938B04B0938C04D801C70177
:10B2F00086199709A809B9098093DF049093E0049F
:10B30000A093E104B093E20420917F08E22EFF2491
:10B3100000271127BC01CD01A80197010E94149DAF
:10B3200059016A012093ED043093EE044093EF0439
:10B330005093F00489899A89AB89BC898219930951
:10B34000A409B5098093E3049093E404A093E50471
:10B35000B093E604BC01CD01A80197010E94149DA1
:10B360002093F1043093F2044093F3045093F404D7
:10B37000D601C501D7FE04C081509F4FAF4FBF4FCC
:10B38000892F9A2FAB2FBB27A7FDBA9590932E0438
:10B3900080932D0457FF04C021503F4F4F4F5F4F04
:10B3A000BB2757FDBA95A52F942F832F9093300478
:10B3B00080932F048091130490911404813491059B
:10B3C000DCF4809111049091120481349105A4F46D
:10B3D00080914008E82FFF27EE0FFF1FEC58F64F33
:10B3E000808191810190F081E02DF7FF03C0F095FD
:10B3F000E195FF4F7A97E4F08091E20A8F3FC1F424
:10B4000080912D0490912E0497FD01969595879536
:10B4100090932E0480932D0480912F0490913004FA
:10B4200097FD0196959587959093300480932F040E
:10B4300080911E0A90911F0AA091200AB091210AC2
:10B44000B7FF04C081509F4FAF4FBF4F892F9A2F36
:10B45000AB2FBB27A7FDBA9580931E0A90931F0AB6
:10B46000A093200AB093210A8091110A9091120AA8
:10B47000A091130AB091140AB7FF04C081509F4FE6
:10B48000AF4FBF4F892F9A2FAB2FBB27A7FDBA9580
:10B490008093110A9093120AA093130AB093140A8E
:10B4A0008091A1049091A204A091A304B091A4045E
:10B4B0002F81388549855A85281B390B4A0B5B0B30
:10B4C0002093D7043093D8044093D9045093DA04DE
:10B4D0008091990490919A04A0919B04B0919C044E
:10B4E000EB84FC840D851E85E81AF90A0A0B1B0BF8
:10B4F000E092DB04F092DC040093DD041093DE04A0
:10B500002093DF043093E0044093E1045093E2047D
:10B51000E092E304F092E4040093E5041093E6045F
:10B5200080917D0490917E04A0917F04B09180046D
:10B53000821B930BA40BB50B80937D0490937E0428
:10B54000A0937F04B0938004809175049091760459
:10B55000A0917704B09178048E199F09A00BB10BCC
:10B560008093750490937604A0937704B093780445
:10B5700088898823E1F020915B0430915C042138B4
:10B5800031054CF08091B3049091B40401969093EE
:10B59000B4048093B30420583F4F4CF48091B3041B
:10B5A0009091B40401979093B4048093B3041092E3
:10B5B0005C0410925B0481E090E09093FA04809325
:10B5C000F904E090DF04F090E0040091E1041091B0
:10B5D000E204D801C70117FF07C088279927DC01BB
:10B5E0008E199F09A00BB10B81509240A040B04032
:10B5F00034F084E090E09093FA048093F904809111
:10B60000FF0490910005A0910105B09102052091E1
:10B61000290A30912A0A40912B0A50912C0A821B48
:10B62000930BA40BB50B815E914BAF4FBF4F8F5364
:10B630009C49A040B04028F08091E30A89310CF485
:10B64000FFC021E0E21620E1F20620E0020720E040
:10B6500012070CF473C08091FB04882309F46AC0BC
:10B66000D801C70117FF07C088279927DC018E1969
:10B670009F09A00BB10B9C01AD01B7FF04C0215085
:10B680003E4F4F4F5F4FF9E05595479537952795BA
:10B69000FA95D1F78091F9049091FA04820F931FE3
:10B6A0009093FA048093F904D801C70117FF03C0EF
:10B6B0000796A11DB11DE3E0B595A79597958795D0
:10B6C000EA95D1F78093ED049093EE04A093EF04F4
:10B6D000B093F00489589341A040B04064F088E8EA
:10B6E00093E1A0E0B0E08093ED049093EE04A0938A
:10B6F000EF04B093F0042091ED043091EE044091FA
:10B70000EF045091F00457FF04C021503F4F4F4FBA
:10B710005F4F232F342F452F552747FD5A95809192
:10B720002D0490912E04820F931F90932E048093EA
:10B730002D0406C081E08093FB0402C01092FB043C
:10B7400040E0E41640EFF4064FEF04074FEF140714
:10B750000CF073C08091FC04882309F46AC0D801FE
:10B76000C70117FF07C088279927DC018E199F0999
:10B77000A00BB10B9C01AD01B7FF04C021503E4F9F
:10B780004F4F5F4F69E055954795379527956A95D7
:10B79000D1F78091F9049091FA04820F931F90934E
:10B7A000FA048093F904D801C70117FF03C0079674
:10B7B000A11DB11D23E0B595A795979587952A956D
:10B7C000D1F78093ED049093EE04A093EF04B0932F
:10B7D000F00488579C4EAF4FBF4F64F488E79CEE4F
:10B7E000AFEFBFEF8093ED049093EE04A093EF04CE
:10B7F000B093F0042091ED043091EE044091EF04F9
:10B800005091F00457FF04C021503F4F4F4F5F4FFE
:10B81000232F342F452F552747FD5A9580912D040E
:10B8200090912E04820F931F90932E0480932D04E9
:10B8300011C081E08093FC040DC01092FC040AC08A
:10B840001092FA041092F90484E690E090938D012E
:10B8500080938C016889262F33278091F904909179
:10B86000FA042817390724F43093FA042093F904D2
:10B870001091E30A112379F0212F332727FD30950A
:10B880008091F9049091FA042817390724F4309331
:10B89000FA042093F9044091DF045091E004609190
:10B8A000E1047091E204413851056105710574F0BD
:10B8B0008091B7049091B8042091F9043091FA0472
:10B8C000820F931F9093B8048093B70440585F4F42
:10B8D0006F4F7F4F74F48091B7049091B80420911A
:10B8E000F9043091FA04821B930B9093B80480936F
:10B8F000B70481E090E09093FA048093F904C0903B
:10B90000E304D090E404E090E504F090E604D7016D
:10B91000C601F7FE07C088279927DC018C199D090D
:10B92000AE09BF0981509240A040B04034F084E09D
:10B9300090E09093FA048093F9048091030590912C
:10B940000405A0910505B09106052091310A3091BA
:10B95000320A4091330A5091340A821B930BA40B94
:10B96000B50B815E914BAF4FBF4F8F539C49A040A9
:10B97000B04018F019310CF4FFC001E0C01600E12E
:10B98000D00600E0E00600E0F0060CF473C0809101
:10B99000FD04882309F46AC0D701C601F7FE07C079
:10B9A00088279927DC018C199D09AE09BF099C01E4
:10B9B000AD01B7FF04C021503E4F4F4F5F4F09E02C
:10B9C00055954795379527950A95D1F78091F904B4
:10B9D0009091FA04820F931F9093FA048093F904D4
:10B9E000D701C601F7FE03C00796A11DB11D13E0E4
:10B9F000B595A795979587951A95D1F78093F104FA
:10BA00009093F204A093F304B093F4048958934103
:10BA1000A040B04064F088E893E1A0E0B0E08093FB
:10BA2000F1049093F204A093F304B093F4042091F2
:10BA3000F1043091F2044091F3045091F40457FF63
:10BA400004C021503F4F4F4F5F4F232F342F452FBE
:10BA5000552747FD5A9580912F0490913004820F0D
:10BA6000931F9093300480932F0406C081E080934D
:10BA7000FD0402C01092FD0420E0C21620EFD206A1
:10BA80002FEFE2062FEFF2060CF073C08091FE0458
:10BA9000882309F46AC0D701C601F7FE07C08827CA
:10BAA0009927DC018C199D09AE09BF099C01AD01E4
:10BAB000B7FF04C021503E4F4F4F5F4FE9E055950F
:10BAC000479537952795EA95D1F78091F90490919C
:10BAD000FA04820F931F9093FA048093F904D7011C
:10BAE000C601F7FE03C00796A11DB11D73E0B59511
:10BAF000A795979587957A95D1F78093F1049093C0
:10BB0000F204A093F304B093F40488579C4EAF4F13
:10BB1000BF4F64F488E79CEEAFEFBFEF8093F10472
:10BB20009093F204A093F304B093F4042091F104F1
:10BB30003091F2044091F3045091F40457FF04C093
:10BB400021503F4F4F4F5F4F232F342F452F552705
:10BB500047FD5A9580912F0490913004820F931FD6
:10BB60009093300480932F0411C081E08093FE04F1
:10BB70000DC01092FE040AC01092FA041092F9044B
:10BB800084E690E090938D0180938C014889242F66
:10BB900033278091F9049091FA042817390724F487
:10BBA0003093FA042093F9048091E30A882379F012
:10BBB000282F332727FD30958091F9049091FA04BE
:10BBC0002817390724F43093FA042093F90440919C
:10BBD000E3045091E4046091E5047091E604413877
:10BBE00051056105710574F08091B5049091B6041A
:10BBF0002091F9043091FA04820F931F9093B604B8
:10BC00008093B50440585F4F6F4F7F4FCCF48091C5
:10BC1000B5049091B6042091F9043091FA04821B86
:10BC2000930B9093B6048093B5040AC0109230042D
:10BC300010922F0410922E0410922D0410925D0485
:10BC40008091370A882341F41092300410922F0417
:10BC500010922E0410922D048091290A90912A0AA4
:10BC6000A0912B0AB0912C0A8093FF0490930005B9
:10BC7000A0930105B09302058091310A9091320A98
:10BC8000A091330AB091340A809303059093040580
:10BC9000A0930505B09306051092910410929204AA
:10BCA000109293041092940410928D0410928E04BA
:10BCB00010928F04109290041092890410928A04BA
:10BCC00010928B0410928C041092290A10922A0A66
:10BCD00010922B0A10922C0A1092310A1092320AFA
:10BCE0001092330A1092340A10921E0A10921F0A00
:10BCF0001092200A1092210A1092110A1092120A30
:10BD00001092130A1092140A1092300310922F030B
:10BD1000E0905304F0905404C701F7FE04C0882754
:10BD200099278E199F0904973CF08091520A84FD4F
:10BD300003C082E38093310410915508A12EBB24E7
:10BD4000CC24DD24B701882777FD8095982F9701B3
:10BD5000F7FE04C0222733272E193F09442737FD59
:10BD60004095542F0E94A09C9B01AC01C601B501D7
:10BD70000E94A09C97FF04C061507E4F8F4F9F4F41
:10BD800059E095958795779567955A95D1F79B01D9
:10BD9000812F99278E9DD0018F9DB00D9E9DB00D56
:10BDA0001124CD01B7FD03969595879595958795B7
:10BDB000280F391F8091090490910A048150924004
:10BDC00010F020E030E08091330490913404280F8B
:10BDD000391F442737FD4095542F2093D3043093C7
:10BDE000D4044093D5045093D6048091710490916B
:10BDF0007204A0917304B0917404821B930BA40B82
:10BE0000B50B8093710490937204A0937304B09364
:10BE100074048155934CA040B04064F080E593ECED
:10BE2000A0E0B0E08093710490937204A093730437
:10BE3000B09374048091710490917204A091730482
:10BE4000B0917404805B9C43AF4FBF4F64F480EBB0
:10BE50009CE3AFEFBFEF8093710490937204A093C3
:10BE60007304B0937404009190011091910117FD37
:10BE7000FCC08091520A83FFF8C080918F018150ED
:10BE800080938F01882309F0F4C08DE080938F01A7
:10BE90008091A1049091A204A091A304B091A40464
:10BEA000B7FF04C081509E4FAF4FBF4F39E0B595EB
:10BEB000A795979587953A95D1F77C0197FF04C090
:10BEC000F094E194F108F3948091990490919A048C
:10BED000A0919B04B0919C04B7FF04C081509E4F79
:10BEE000AF4FBF4F29E0B595A795979587952A95B0
:10BEF000D1F79C0197FF03C0309521953F4FE21683
:10BF0000F3060CF47901B701F7FE02C0695F7F4FB9
:10BF10002B0183E0559447948A95E1F722E030E0C5
:10BF2000420E531E6090620A7090630A8090640A09
:10BF30009090650A20914201309143014091440163
:10BF400050914501C401B3010E94149D59016A0139
:10BF500030930F0A20930E0A021B130BC801845E54
:10BF60009D4F68E671E00E94DF9C9C01245B30409D
:10BF700080918C0190918D01009731F00197909301
:10BF80008D0180938C011BC049E1E416F104BCF4DF
:10BF900080915B0490915C04820F931F90935C04EA
:10BFA00080935B0480913104882349F08150809311
:10BFB0003104882321F4B0926004A0925F04809140
:10BFC0008C0190918D01892BF9F480918E01992734
:10BFD000289FB001299F700D389F700D1124CB014F
:10BFE000B2010E94DF9CCB01AA2797FDA095BA2F32
:10BFF000680E791E8A1E9B1E6092620A7092630A06
:10C000008092640A9092650A80913104882369F5D0
:10C0100080915F049091600420910E0A30910F0A84
:10C02000821B930B845E9D4F68E671E00E94DF9C4B
:10C030009C01245B30408091790186959927289F47
:10C04000D001299FB00D389FB00D11249D01B7FF7D
:10C0500002C0215F3F4F04E0359527950A95E1F72F
:10C06000309334042093330404C0109234041092AB
:10C07000330480915D04882381F01092650410924E
:10C08000660410926704109268041092690410927A
:10C090006A0410926B0410926C0480912A04882325
:10C0A000F1F48091370A282F3327442755278091B0
:10C0B000A1049091A204A091A304B091A404BC0196
:10C0C000CD010E94A09CDC01CB01BC01CD0128EF79
:10C0D0003AE240E050E00E94149D290102C044244D
:10C0E0005524809129048823F1F48091370A282F60
:10C0F0003327442755278091990490919A04A09161
:10C100009B04B0919C04BC01CD010E94A09CDC0169
:10C11000CB01BC01CD0128EF3AE240E050E00E94A3
:10C12000149D190102C02224332480910B0A90919E
:10C130000C0A893C91051CF088EC90E005C08853FE
:10C140009F4F34F488E39FEF90930C0A80930B0A7F
:10C150008091160A9091170A893C91051CF088EC91
:10C1600090E005C088539F4F34F488E39FEF90938D
:10C17000170A8093160A8091180A9091190AAA2723
:10C1800097FDA095BA2F2091600AA22EBB24CC2443
:10C19000DD24BC01CD01A60195010E94A09C9B015C
:10C1A000AC0180910B0A90910C0AAA2797FDA095EB
:10C1B000BA2F17E0880F991FAA1FBB1F1A95D1F736
:10C1C000280F391F4A1F5B1F57FF04C0215C3F4FD8
:10C1D0004F4F5F4FA6E05595479537952795AA9500
:10C1E000D1F78201020F131F1093190A0093180A46
:10C1F0008091090A90910A0AAA2797FDA095BA2F63
:10C20000BC01CD01A60195010E94A09C9B01AC013F
:10C210008091160A9091170AAA2797FDA095BA2F28
:10C22000F7E0880F991FAA1FBB1FFA95D1F7280FB7
:10C23000391F4A1F5B1F57FF04C0215C3F4F4F4F00
:10C240005F4FE6E05595479537952795EA95D1F7E5
:10C250007101E20EF31EF0920A0AE092090A80913F
:10C260005B0A90915C0A880F991FAA2797FDA095F9
:10C27000BA2F2091100A332744275527BC01CD013E
:10C280000E94A09C5B016C0197FF08C02FE330E087
:10C2900040E050E0A20EB31EC41ED51E76E0D59439
:10C2A000C794B794A7947A95D1F78091260A282F3E
:10C2B0003327442755278091850490918604A091C7
:10C2C0008704B0918804BC01CD010E94A09CDC01D0
:10C2D000CB01BC01CD0120EF35E540E050E00E94EC
:10C2E000149DB501620F731F70935C0A60935B0A23
:10C2F0000150104134F080E090E19093190A80934E
:10C30000180A8091180A9091190A8050904F34F4BD
:10C3100080E090EF9093190A8093180A51E0E51697
:10C3200050E1F50634F080E090E190930A0A8093A2
:10C33000090A8091090A90910A0A8050904F34F4BA
:10C3400080E090EF90930A0A8093090A615070414F
:10C3500034F080E090E190935C0A80935B0A8091D6
:10C360005B0A90915C0A8050904F34F480E090EF2B
:10C3700090935C0A80935B0A80910E0485FD16C041
:10C38000809102019927209126013091270109818E
:10C390001A81089F7001099FF00C189FF00C11245E
:10C3A000C701B9010E94CB9C7A83698380910705FC
:10C3B0008150809307058F3F09F047C080910805A1
:10C3C00090910905892B41F48091260190912701D4
:10C3D000909309058093080580912601909127018B
:10C3E00020910805309109052817390718F42F5FA7
:10C3F0003F4F09C080912601909127018217930732
:10C4000030F421503040309309052093080584E62C
:10C41000809307058091AB08282F332740910805AA
:10C42000509109054217530710F48AE00CC080911F
:10C430000001280F311D2417350738F480910504B9
:10C44000882319F081508093050480910504882386
:10C45000D1F08091370490913804A0913904B091C3
:10C460003A04B7FD10C08091A9088093360480EE8D
:10C4700091EBAFEFBFEF8093370490933804A09314
:10C480003904B0933A0480911A03882311F40E946E
:10C49000EF7029813A81220F331F220F331F3A8315
:10C4A00029838091520A80FD02C00C94CF6C809148
:10C4B0002904882311F00C94CF6C20912A042223A4
:10C4C00011F00C94CF6C8091B10599278F77907003
:10C4D000009711F00C94CF6C3C018091B9049091BD
:10C4E000BA04892B09F044C080911C0190911D0170
:10C4F0008959934058F087B58A3F20F480913303DF
:10C50000815011C081E0809315055EC080911C01AF
:10C5100090911D018436910530F587B58630F8F08D
:10C52000809133038F5F8093330395E089029001FC
:10C5300011248091E807821B87BD87B5809588BD4F
:10C540008CE291E090931C0380931B038EE591E0B5
:10C550009093BA048093B9040E94601E35C081E0B4
:10C560008093140531C020931405209315052CC029
:10C57000709232036092310380910604882321F087
:10C5800081E00E94879617C08091410490914204F7
:10C59000A0914304B091440454E0880F991FAA1F4E
:10C5A000BB1F5A95D1F78093340390933503A09322
:10C5B0003603B09337038091B9049091BA04019780
:10C5C0009093BA048093B9048091520A2091240474
:10C5D00081FF3CC0223348F58091950181508093C2
:10C5E00095018F3F09F052C08091AA01882339F448
:10C5F00080915E04882319F088E28093AA0110924A
:10C600005E048091410490914204A0914304B09152
:10C61000440480933D0490933E04A0933F04B09360
:10C62000400481E08093950131C0273478F18091F6
:10C63000AA01882339F480915E04882319F487E2E3
:10C640008093AA0188EC809395011DC080914601DA
:10C6500090914701820F911D20914E083327829FB0
:10C66000A001839F500D929F500D1124CA01AA274B
:10C6700097FDA095BA2F80933D0490933E04A0931C
:10C680003F04B093400481E080935E048091A10454
:10C690009091A204A091A304B091A404E09042015F
:10C6A000F09043010091440110914501BC01CD017E
:10C6B000A80197010E94149D59016A018091990473
:10C6C00090919A04A0919B04B0919C04BC01CD016F
:10C6D000A80197010E94149DB901C5010E94758DA2
:10C6E0009093230A8093220ACC9734F08CE390E055
:10C6F0009093230A8093220A8091220A9091230A20
:10C700000E94837A9093230A8093220A80E2809386
:10C71000410110923C0410923B0480915E048823F6
:10C7200009F4A1C780910E0499279C0120713070F3
:10C7300084FD99C780910D04826080930D047091EF
:10C74000350A872F992741E0842E912C882299223F
:10C7500080FD04C08091520A81FD10C0E980FA80FA
:10C7600030930B0520930A0530933C0420933B043F
:10C7700080910E04806C80930E0410C380910E048F
:10C7800081FFDFC20091820110918301C8010F96E1
:10C79000A0915104B0915204B88FAF8B8A179B07B8
:10C7A0000CF09AC080911405882309F095C08091FF
:10C7B0000E0487FF15C080910E048F7780930E04BE
:10C7C0008091270390912803A0912903B0912A0317
:10C7D00080933D0490933E04A0933F04B0934004A3
:10C7E000E090150AEE20D9F180913D0490913E042D
:10C7F000A0913F04B0914004BC01CD0124E630E09B
:10C8000040E050E00E94149DAE2CBB24CC24DD24DB
:10C81000A216B306C406D50614F590923C04809285
:10C820003B048091AA018823C1F480914104909136
:10C830004204A0914304B0914404BC01CD012FE512
:10C8400030E040E050E00E94149DA216B306C406FA
:10C85000D5061CF48AE18093AA018DE338C080914B
:10C860000C0590910D05459784F0809127039091D8
:10C870002803A0912903B0912A0380933D0490934B
:10C880003E04A0933F04B093400480910E04806462
:10C8900080930E042F89388D201B310B2F50304090
:10C8A00037FF03C0309521953F4F30933C042093D0
:10C8B0003B0480910504882349F0C90163E070E0DE
:10C8C0000E94DF9C70933C0460933B048BE2809356
:10C8D00041011092350437C1C8010F97EF89F88DD7
:10C8E000E817F907CCF5209115052223A9F58091C9
:10C8F0000E0486FF15C080910E048F7B80930E047A
:10C900008091270390912803A0912903B0912A03D5
:10C9100080933D0490933E04A0933F04B093400461
:10C9200080910E04806880930E048F89988D801BFF
:10C93000910B0F9697FF03C0909581959F4F90950F
:10C9400081959F4F90933C0480933B048DE28093AC
:10C95000410120933504F7C08DE38093410160913C
:10C960003604662371F120913704309138044091E8
:10C97000390450913A0480913D0490913E04A09175
:10C980003F04B091400482179307A407B507CCF485
:10C9900080910E04806480930E04862F99279093D3
:10C9A0003C0480933B048AE0809335048EE58093B9
:10C9B000410180910E0487FFC6C080910E048F77DD
:10C9C00033C0662309F443C0209137043091380402
:10C9D0004091390450913A0480913D0490913E0475
:10C9E000A0913F04B0914004281739074A075B071C
:10C9F00074F580910E04806880930E04862F992729
:10CA0000909581959F4F90933C0480933B0486EFD3
:10CA10008093350486E78093410180910E0486FF60
:10CA200092C080910E048F7B80930E048091270327
:10CA300090912803A0912903B0912A0380933D048B
:10CA400090933E04A0933F04B09340047CC0809137
:10CA50000E04807C09F477C080913504882309F0A6
:10CA60004CC08091270390912803A0912903B09195
:10CA70002A03885C9040A040B04020913D04309152
:10CA80003E0440913F045091400482179307A4074D
:10CA9000B5076CF08091270390912803A09129039A
:10CAA000B0912A03885C9040A040B0401DC08091A6
:10CAB000270390912803A0912903B0912A0388535A
:10CAC0009F4FAF4FBF4F281739074A075B07BCF08E
:10CAD0008091270390912803A0912903B0912A0304
:10CAE00088539F4FAF4FBF4F80933D0490933E04B8
:10CAF000A0933F04B093400402C01092350480918B
:10CB00000E048F7380930E0410920B0510920A0589
:10CB100071FF06C084EF91E090931C0380931B0388
:10CB200080914504882379F48091410490914204D6
:10CB3000A0914304B0914404C397A105B1051CF032
:10CB400081E08093450460910A0570910B05809106
:10CB50003B0490913C04680F791F70930B05609320
:10CB60000A05CB0177FF04C088279927861B970BFE
:10CB7000855F91400CF4CEC040913504442389F187
:10CB8000809137049091380420913D0430913E0407
:10CB9000821B930B0996439748F480913704909138
:10CBA0003804A0913904B0913A0412C0242F3327DD
:10CBB00027FD3095432F532F80913D0490913E04E3
:10CBC000A0913F04B0914004820F931FA41FB51F92
:10CBD00080933D0490933E04A0933F04B09340049F
:10CBE00024C020913D0430913E0440913F04509177
:10CBF000400480914E081616170644F463E00E9424
:10CC0000BF9C280F311D411D511D07C063E00E94CC
:10CC1000BF9C281B31094109510920933D043093E1
:10CC20003E0440933F045093400410920B05109231
:10CC30000A05E0904104F0904204009143041091F1
:10CC40004404D801C70180509440A040B0402091D6
:10CC50003D0430913E0440913F04509140048217BE
:10CC60009307A407B5075CF4D801C70180509C4F17
:10CC7000AF4FBF4F281739074A075B0744F080932F
:10CC80003D0490933E04A0933F04B09340048091F0
:10CC9000350A81FF06C084E690E090931C038093E0
:10CCA0001B03809152088823A9F5809136048823BC
:10CCB00089F540912B0450912C0457FF02C04D5F21
:10CCC0005F4F5595479555954795809126019091D1
:10CCD0002701209102013327489F7001499FF00CE2
:10CCE000589FF00C1124C701B9010E94DF9C70937A
:10CCF000830160938201663471051CF486E490E040
:10CD000005C06739710534F086E990E0909383019E
:10CD1000809382018091B9049091BA04892BD1F15A
:10CD20008091270390912803A0912903B0912A03B1
:10CD300080933D0490933E04A0933F04B09340043D
:10CD400029C08091410490914204A0914304B09184
:10CD5000440480599140A040B04080933D0490939A
:10CD60003E04A0933F04B09340048091520888236E
:10CD700011F0992702C088E790E090938301809397
:10CD8000820109811A8110932C0400932B048EE2F6
:10CD900080934101E0902B04F0902C0480912703B4
:10CDA00090912803A0912903B0912A0320913D047A
:10CDB00030913E0440913F045091400428173907B8
:10CDC0004A075B0724F08091350A80FD98C4809162
:10CDD00006046091B9047091BA04882309F07CC2FA
:10CDE000672B49F0E0902B04F0902C0410920D0575
:10CDF00010920C05E1C08091270390912803A09127
:10CE00002903B0912A03821B930BA40BB50B8093CB
:10CE1000D7049093D804A093D904B093DA04823055
:10CE200010E891071FEFA1071FEFB1072CF481E075
:10CE300090E8AFEFBFEF09C08F5F9F47A040B040C1
:10CE400064F08FEF9FE7A0E0B0E08093D704909369
:10CE5000D804A093D904B093DA048091D7049091B8
:10CE6000D80490930D0580930C0580917B01282FA9
:10CE70003327442755278091D7049091D804A09157
:10CE8000D904B091DA04BC01CD010E94A09C97FFA7
:10CE900004C0615E7F4F8F4F9F4F25E0959587952A
:10CEA000779567952A95D1F76093D7047093D80446
:10CEB0008093D9049093DA0465303EEF73073FEF17
:10CEC00083073FEF93072CF484E09EEFAFEFBFEFB3
:10CED00009C0605074408040904064F080E094E06D
:10CEE000A0E0B0E08093D7049093D804A093D90435
:10CEF000B093DA046090D7047090D8042091310385
:10CF00003091320337FF02C0295F3F4F03E0359570
:10CF100027950A95E1F75FEF223835071CF421E8E1
:10CF20003FEF05C02038310514F020E830E0C9019A
:10CF3000AA2797FDA095BA2F20917C01332744277B
:10CF40005527BC01CD010E94A09C97FF04C06D5FD6
:10CF50007F4F8F4F9F4F12E09595879577956795F7
:10CF60001A95D1F79B016FEF213036071CF420E0B2
:10CF70003FEF06C02F3F310519F014F020E031E0FB
:10CF800080910E04807C49F0C90137FD03969C0115
:10CF900035952795359527950DC08091350A80FFE9
:10CFA00009C0C90137FD07969C01A3E03595279577
:10CFB000AA95E1F7620E731E20917A01222309F4EB
:10CFC00054C06091610470916204809163049091F7
:10CFD000640497FF04C061587F4F8F4F9F4FF7E065
:10CFE0009595879577956795FA95D1F733274427D7
:10CFF00055270E94A09C97FF04C0615E7F4F8F4F12
:10D000009F4FE5E09595879577956795EA95D1F7D8
:10D010006093D7047093D8048093D9049093DA0472
:10D020006138AFEF7A07AFEF8A07AFEF9A072CF4BA
:10D0300080E89FEFAFEFBFEF0AC06F3F710581053A
:10D04000910569F064F080E091E0A0E0B0E08093A9
:10D05000D7049093D804A093D904B093DA048091B4
:10D06000D7049091D804680E791E80917801282FFA
:10D0700033278091E60A992787FD9095289FF00134
:10D08000299FF00D389FF00D11249F01F7FF02C07A
:10D0900021583F4F220F232F221F330BFFEF213840
:10D0A0003F071CF420E83FEF06C02F3F310519F081
:10D0B00014F020E031E0260D371DC901AA2797FDA5
:10D0C000A095BA2F00912B0410912C0498014427AD
:10D0D00037FD4095542FBC01CD010E94A09C97FFC5
:10D0E00004C061507E4F8F4F9F4F59E095958795B3
:10D0F000779567955A95D1F7E61AF70A80913B0420
:10D1000090913C04892B09F064C0101611060CF0B4
:10D1100060C020910C0530910D05C90137FF03C097
:10D12000309521953F4F2D33310540F480915904BE
:10D1300090915A048E159F0574F526C02C533040EB
:10D1400045E0369527954A95E1F72031310510F0F5
:10D150002FE030E04091590450915A0418161906F6
:10D16000E4F480E190E0821B930B489F9001499F7B
:10D17000300D589F300D1124B4E036952795BA959F
:10D18000E1F72E153F0520F58091800190918101F6
:10D19000E816F906F4F07C011CC0205F3F4F809137
:10D1A000800190918101829FB001839F700D929FB9
:10D1B000700D11249B01A4E036952795AA95E1F7FF
:10D1C0004E155F0514F07A0104C0E216F30608F06C
:10D1D0007901C701AA2797FDA095BA2FFDE0880F16
:10D1E000991FAA1FBB1FFA95D1F72091220A3091EF
:10D1F000230A442737FD4095542FBC01CD010E94DE
:10D20000149D2093DB043093DC044093DD045093A1
:10D21000DE04E090DB04F090DC0480910E05909138
:10D220000F059C01220F331F280F391F2E0D3F1DA4
:10D2300037FF02C02D5F3F4FA90155954795559582
:10D24000479550930F0540930E0580914A08282F6B
:10D250003327220F331F220F331F241735076CF497
:10D2600080915A0A282F3327220F331F220F331F92
:10D27000205530404217530724F030930F05209378
:10D280000E058091350A80FF14C080910E059091A3
:10D290000F05A981BA818A179B0724F0B0930F0567
:10D2A000A0930E05E0910E05F0910F05FA83E98336
:10D2B00026C229813A81201B310B37FF02C02D5F26
:10D2C0003F4F3595279535952795E0900E05F090C1
:10D2D0000F05E20EF31EC1C1672B49F0E0902B044D
:10D2E000F0902C0410920D0510920C0538C180911D
:10D2F000270390912803A0912903B0912A03821B50
:10D30000930BA40BB50B8093D7049093D804A093F0
:10D31000D904B093DA04823000E890070FEFA00739
:10D320000FEFB0072CF481E090E8AFEFBFEF09C03A
:10D330008F5F9F47A040B04064F08FEF9FE7A0E071
:10D34000B0E08093D7049093D804A093D904B0930D
:10D35000DA048091D7049091D80490930D058093BE
:10D360000C0580917B01282F332744275527809176
:10D37000D7049091D804A091D904B091DA04BC01EB
:10D38000CD010E94A09C97FF04C0615E7F4F8F4F2C
:10D390009F4F05E095958795779567950A95D1F705
:10D3A0006093D7047093D8048093D9049093DA04DF
:10D3B000653028EF72072FEF82072FEF92072CF4CA
:10D3C00084E098EFAFEFBFEF09C060507840804035
:10D3D000904064F080E098E0A0E0B0E08093D70453
:10D3E0009093D804A093D904B093DA046090D70442
:10D3F0007090D80480917A01282F332780913803C8
:10D4000090913903829FA001839F500D929F500DF0
:10D4100011249A0157FF02C021503F4F232F330F91
:10D42000330B8091310390913203820F931FAA270F
:10D4300097FDA095BA2F8093D7049093D804A0931A
:10D44000D904B093DA048091350420913B043091E3
:10D450003C04882331F0B3E0220F331FBA95E1F783
:10D460001BC080914E089927289FB001299F700DFD
:10D47000389F700D11249B01A3E0220F331FAA9542
:10D48000E1F7260F371F37FF02C0215E3F4FF5E05F
:10D4900035952795FA95E1F7309308042093070412
:10D4A00080910704909108049C01442737FD409522
:10D4B000542F8091D7049091D804A091D904B091B1
:10D4C000DA04821B930BA40BB50B8093D7049093C3
:10D4D000D804A093D904B093DA0420917C013327B7
:10D4E00044275527BC01CD010E94A09C97FF04C092
:10D4F000615E7F4F8F4F9F4FE5E0959587957795BC
:10D500006795EA95D1F76093D7047093D804809318
:10D51000D9049093DA046530A8EF7A07AFEF8A0751
:10D52000AFEF9A072CF484E098EFAFEFBFEF09C09C
:10D53000605078408040904064F080E098E0A0E047
:10D54000B0E08093D7049093D804A093D904B0930B
:10D55000DA048091D7049091D804680E791EE618F9
:10D56000F7088091590490915A048E159F053CF458
:10D570008091800190918101E816F9060CF07C0100
:10D58000C701AA2797FDA095BA2F5DE0880F991FC4
:10D59000AA1FBB1F5A95D1F72091220A3091230A66
:10D5A000442737FD4095542FBC01CD010E94149DA6
:10D5B0002093DB043093DC044093DD045093DE04BD
:10D5C000E090DB04F090DC0480910E0590910F0553
:10D5D0009C01220F331F280F391F2E0D3F1D37FFCF
:10D5E00002C02D5F3F4FA901559547955595479529
:10D5F00050930F0540930E0580914A08282F33273A
:10D60000220F331F220F331F241735076CF480912C
:10D610005A0A282F3327220F331F220F331F20557A
:10D6200030404217530724F030930F0520930E0526
:10D630008091350A20910E0530910F0580FF10C0B2
:10D64000E981FA812E173F0724F0F0930F05E0934C
:10D650000E05E0900E05F0900F05FA82E9824FC0AA
:10D660003A8329834CC080915208882301F5609148
:10D670002B0470912C0477FF02C06D5F7F4F75956E
:10D680006795759567954091260150912701809186
:10D690000201282F3327649FC001659F900D749F5E
:10D6A000900D1124B9010E94DF9CCB0101C0992784
:10D6B00090938301809382018091820190918301F4
:10D6C000873491051CF486E490E005C08639910505
:10D6D00034F086E990E09093830180938201098180
:10D6E0001A8110930F0500930E0580910E04806C33
:10D6F00080930E0480910D048D7F80930D048091A2
:10D700000E0499279C012270307081FF39C18091ED
:10D71000100590911105A0911205B0911305009785
:10D72000A105B10521F0809145048130B9F48091C3
:10D730002B0490912C04AA2797FDA095BA2F1EE0E8
:10D74000880F991FAA1FBB1F1A95D1F78093100548
:10D7500090931105A0931205B09313058091450491
:10D76000813019F482E08093450429813A8179015E
:10D770000027F7FC0095102F8091220A9091230A30
:10D780009C01442737FD4095542FC801B7010E94E2
:10D79000A09CDC01CB018093DB049093DC04A0937C
:10D7A000DD04B093DE04B7FF04C08150904EAF4F4C
:10D7B000BF4F7C018D01ADE015950795F794E79477
:10D7C000AA95D1F7E092DB04F092DC040093DD042B
:10D7D0001093DE0460910F04709110043FE0603AF2
:10D7E000730750F58091100590911105A0911205D5
:10D7F000B09113059C01AD01FAE056954795379518
:10D800002795FA95D1F7821B930BA40BB50BA801B2
:10D810009701E4E0220F331F441F551FEA95D1F70B
:10D82000820F931FA41FB51F8093100590931105BD
:10D83000A0931205B093130560547F4118F58091B1
:10D84000100590911105A0911205B09113059C014E
:10D85000AD016CE056954795379527956A95D1F7B8
:10D86000821B930BA40BB50BA8019701F2E0220FCA
:10D87000331F441F551FFA95D1F7820F931FA41F22
:10D88000B51F41C0809131039091320380913103E3
:10D890009091320397FF03C0909581959F4F8436F6
:10D8A0009105CCF58091270390912803A09129033D
:10D8B000B0912A039C0180913D0490913E04281B65
:10D8C000390B37FF03C0309521953F4F2F3F31056E
:10D8D00009F00CF58091100590911105A0911205A9
:10D8E000B09113059C01AD01EEE056954795379533
:10D8F0002795EA95D1F7821B930BA40BB50B8E0DE0
:10D900009F1DA01FB11F8093100590931105A09338
:10D910001205B09313058091100590911105A09107
:10D920001205B09113057EE0B695A795979587955A
:10D930007A95D1F790932C0480932B044091500852
:10D94000442399F055279C01BA010E94DF9CC9012C
:10D95000861B970B90935A0480935904260F371F08
:10D9600030938101209380011FC010925A041092BD
:10D9700059048FEF93E0909381018093800114C04C
:10D980001092450410921005109211051092120584
:10D990001092130530932C0420932B0405C0809122
:10D9A0000E04806C80930E048091240581FF37C0A3
:10D9B00089819A8197FD0396959587959595879589
:10D9C00020910B0430910C042817390760F48091E2
:10D9D0002B0490912C04892B31F0220F331F220F3E
:10D9E000331F3A8329838091270390912803A091C4
:10D9F0002903B0912A0380933D0490933E04A093A1
:10DA00003F04B093400488E99AE390931C03809309
:10DA10001B0380E09EE090930C0180930B01A0918A
:10DA20001D0A8A2F9927880F991F880F991F88969A
:10DA300069817A818617970714F09A8389832091E8
:10DA40005A0A822F9927880F991F880F991F80558E
:10DA50009040E981FA818E179F0714F49A83898395
:10DA600080916903882341F48091F80A8F3F21F463
:10DA700080912805882319F180910F04909110045A
:10DA80000297C097E0F4E980FA801E141F04BCF4EA
:10DA900081E090E09093100480930F040A2F1127E7
:10DAA000000F111F000F111F085D1F4F1A830983FC
:10DAB0008091F80A883218F489E08093AA0149819C
:10DAC0005A815093A6074093A5078091D304909163
:10DAD000D404A091D504B091D60412E0880F991F08
:10DAE000AA1FBB1F1A95D1F700915B0A10915C0A1F
:10DAF000081B190B413A51058CF0CA0157FD0196DC
:10DB000095958795801791070CF48C0190958195D8
:10DB10009F4F081719076CF48C010BC001351105D4
:10DB200014F000E510E05FEF003B150714F400EB84
:10DB30001FEF3327220F331F220F331FC9016981C3
:10DB40007A81861B970B801791070CF48C018981D1
:10DB50009A81821B930B081719070CF48C01809192
:10DB6000180A9091190A6091570470915804861B05
:10DB7000970B9093280A8093270AD090370A209118
:10DB8000690430916A0440916B0450916C04DD206B
:10DB900041F0461A570AC201AA2797FDA095BA2F4D
:10DBA00004C0AA2797FDA095BA2F280F391F4A1F36
:10DBB0005B1F2093690430936A0440936B04509375
:10DBC0006C048091690490916A04A0916B04B091F7
:10DBD0006C0481509A4FA040B04064F080E09AEF0E
:10DBE000A0E0B0E08093690490936A04A0936B0472
:10DBF000B0936C048091690490916A04A0916B04C5
:10DC0000B0916C0480509640AF4FBF4F64F480E0F9
:10DC100096E0AFEFBFEF8093690490936A04A093FE
:10DC20006B04B0936C04C0905F082091270A309178
:10DC3000280A78E0E72EEC1498F08C2D9927829F23
:10DC4000A001839F500D929F500D1124CA0157FDD2
:10DC500007967C0163E0F594E7946A95E1F712C0BA
:10DC60008C2D86959927829FB001839F700D929F7E
:10DC7000700D1124CB0177FD03967C01F594E79498
:10DC8000F594E794A0907D01B0907E019501442722
:10DC900037FD4095542F8091690490916A04A091BA
:10DCA0006B04B0916C04BC01CD010E94149DE20E86
:10DCB000F31E90906701692D77278827992798018F
:10DCC00017FF04C022273327201B310B37FF02C068
:10DCD0002F5F3F4F35952795A981BA812A0F3B1FAA
:10DCE000442737FD4095542F0E94A09C97FF04C005
:10DCF000615C7F4F8F4F9F4F26E095958795779575
:10DD000067952A95D1F79B016E157F050CF47B0171
:10DD1000309521953F4FE216F3060CF4790180917E
:10DD2000090A90910A0A6091550470915604861B65
:10DD3000970B9093080A8093070A2091650430910D
:10DD400066044091670450916804DD2041F0261A72
:10DD5000370AC101AA2797FDA095BA2F04C0AA27A8
:10DD600097FDA095BA2F280F391F4A1F5B1F2093DC
:10DD7000650430936604409367045093680480916F
:10DD8000650490916604A0916704B0916804815085
:10DD90009A4FA040B04064F080E09AEFA0E0B0E07D
:10DDA0008093650490936604A0936704B09368041D
:10DDB0008091650490916604A0916704B091680415
:10DDC00080509640AF4FBF4F64F480E096E0AFEFD5
:10DDD000BFEF8093650490936604A0936704B093AB
:10DDE00068042091070A3091080A48E04C1598F021
:10DDF0008C2D9927829FB001839F700D929F700D8B
:10DE00001124CB0177FD07966C0193E0D594C7945C
:10DE10009A95E1F712C0C6948C2D9927829FD00164
:10DE2000839FB00D929FB00D1124CD01B7FD0396D5
:10DE30006C01D594C794D594C7949501442737FDB8
:10DE40004095542F8091650490916604A0916704D9
:10DE5000B0916804BC01CD010E94149DC20ED31E76
:10DE6000692D772788279927980117FF04C0222753
:10DE70003327201B310B37FF02C02F5F3F4F3595F3
:10DE80002795E981FA812E0F3F1F442737FD4095E2
:10DE9000542F0E94A09C97FF04C0615C7F4F8F4F5E
:10DEA0009F4FA6E09595879577956795AA95D1F7A9
:10DEB0009B016C157D050CF46B01309521953F4F4E
:10DEC000C216D3060CF4690180911A03882311F459
:10DED0000E94EF7080911D0A282F33273E8B2D8BD7
:10DEE00080915A0A282E33245090A108F3E1AF2ED6
:10DEF000F9E0BF2EEAEC8E2EE8E09E2E7BE0472E66
:10DF000068E3662E6AE0762ED4012C9112160CF08E
:10DF10002FC1203429F4E981FA81F88FEF8B1FC0DB
:10DF200049815A81CA01AA2797FDA095BA2F3327A4
:10DF300027FD3095432F532FBC01CD010E94A09C9B
:10DF400097FF04C0615C7F4F8F4F9F4F56E09595C0
:10DF50008795779567955A95D1F7788F6F8BF401F0
:10DF60002181203439F42F89388D2E0D3F1D388FB3
:10DF70002F8B2AC0203C39F44F89588D4E195F09E8
:10DF8000588F4F8B21C0C701AA2797FDA095BA2FA4
:10DF9000332727FD3095432F532FBC01CD010E941D
:10DFA000A09C97FF04C0615C7F4F8F4F9F4F46E05E
:10DFB00095958795779567954A95D1F7AF89B88DEF
:10DFC000A60FB71FB88FAF8BF4012281203439F42C
:10DFD0002F89388D2C0D3D1D388F2F8B2AC0203C6A
:10DFE00039F44F89588D4C195D09588F4F8B21C0DA
:10DFF000C601AA2797FDA095BA2F332727FD309594
:10E00000432F532FBC01CD010E94A09C97FF04C059
:10E01000615C7F4F8F4F9F4F36E095958795779541
:10E0200067953A95D1F7AF89B88DA60FB71FB88F0E
:10E03000AF8BF4012381203439F42F89388D200FE0
:10E04000311F388F2F8B2AC0203C39F44F89588DCF
:10E05000401B510B588F4F8B21C0C801AA2797FD39
:10E06000A095BA2F332727FD3095432F532FBC019E
:10E07000CD010E94A09C97FF04C0615C7F4F8F4F31
:10E080009F4F26E095958795779567952A95D1F7C7
:10E09000AF89B88DA60FB71FB88FAF8BF501808100
:10E0A00081FD08C0D3018D919C91EF89F88D8E1769
:10E0B0009F0774F4D3018D919C91EF89F88D8E0F99
:10E0C0009F1F97FD019695958795988F8F8B1EC002
:10E0D000552049F42F89388D220F331F281B390B07
:10E0E000388F2F8B13C031E0351580F4252D332761
:10E0F0004F89588D841B950BB9010E94DF9CCB0181
:10E100006F89788D680F791F788F6F8B8D899E89C5
:10E11000880F991F880F991FAF89B88D8A179B07A1
:10E1200054F4C101880F991F880F991FEF89F88D4A
:10E13000E817F90714F0988F8F8B8F89988D97FDCA
:10E1400003969595879595958795F5018183880F19
:10E15000991F880F991F2F89388D281B390BC901EA
:10E16000880F8283EF89F88DD301ED93FC9303C070
:10E17000F501118212824A9422E030E0620E731E91
:10E1800044E050E0840E951E68E070E0A60EB71ED5
:10E1900047FEBACEE2E1C85E0C944B9D84B1806A22
:10E1A00084B93D9A82E58CBD1DBC459A81E080937F
:10E1B0006C0A8AEA80937D0A83E880937E0A8AE06B
:10E1C00080937F0A1092810A1092800A1092830A2B
:10E1D0001092820A1092E50A1092A10A08953091D5
:10E1E0006C0A332309F070C00DB407FE6DC083E0E4
:10E1F00080931A03459A2EB580912B05992781307B
:10E20000910589F0823091051CF4892B21F03EC0E4
:10E210000297B9F03BC03093A00A20932C05213817
:10E22000A9F581E008C0253549F480912C05820FBD
:10E2300080932C0582E080932B0528C030932B051A
:10E2400025C08091A00AE82FFF27EE53F54F2083C9
:10E250008F5F8093A00A90912C058032A0F029173F
:10E2600069F480E2A2ECBAE0E2EAFAE00D900192F1
:10E270008A95E1F781E08093A10A02C03093A10A58
:10E2800010922B0503C0920F90932C0520917C0ACD
:10E290002232A0F445980000000000000000E09148
:10E2A000750AF091760AE20FF11D80818EBD809192
:10E2B0009E0A9081890F80939E0A03C081E080931B
:10E2C0006C0A2F5F20937C0A0895EF92FF920F93C0
:10E2D0001F93809158089927880F991F880F991FBD
:10E2E0007C010027F7FC0095102F8091A1049091EC
:10E2F000A204A091A304B091A404BC01CD01A80183
:10E3000097010E94149D3093810A2093800A809186
:10E31000990490919A04A0919B04B0919C04BC0133
:10E32000CD01A80197010E94149D3093830A209388
:10E33000820A2091620A3091630A4091640A5091E6
:10E34000650ADA01C90173E0880F991FAA1FBB1F74
:10E350007A95D1F7820F931FA41FB51F820F931FC9
:10E36000A41FB51F20914201309143014091440107
:10E3700050914501BC01CD010E94149D3093890A42
:10E380002093880A8091B3049091B40420913E03B5
:10E3900030913F03821B930B90938F0A80938E0AD8
:10E3A000E091A904F091AA0480912E0A90912F0A7D
:10E3B000BF010E94DF9CCB019B01220F331F220F64
:10E3C000331F280F391F280F391F37FF02C02D5F59
:10E3D0003F4F35952795359527953093850A20939E
:10E3E000840A80915E0A90915F0ABF010E94DF9CBF
:10E3F0009B01220F331F220F331F260F371F260FBB
:10E40000371F37FF02C02D5F3F4F35952795359554
:10E4100027953093870A2093860A1092AA041092B7
:10E42000A90410922F0A10922E0A10925F0A1092DD
:10E430005E0A80917F0A9927AA27BB27FC013A9799
:10E44000E830F10508F031C2EF57FF4F0C94669D9C
:10E45000809123048093920A809122048093930AEE
:10E46000809121048093940A809120048093950ADE
:10E4700080911F048093960A80911E048093970ACE
:10E4800080911D048093980A80911C048093990ABE
:10E4900080910E0480939A0A80910E04837F80936A
:10E4A0000E048091010180939B0A80912601909136
:10E4B000270180939C0A80910D0480939D0A4299C4
:10E4C000F4C180910D04877F80930D04EEC180918B
:10E4D000F20A9091F30A9093930A8093920A8091A2
:10E4E000F60A9091F70A9093950A8093940A809186
:10E4F0008D080E94E9478093960A8091410180939C
:10E50000970A90912D059093980AE92FFF2713E021
:10E51000EE0FFF1F1A95E1F7ED5EF64F80818093B5
:10E52000990A868180939A0A838180939B0A8781C6
:10E5300080939C0A858180939D0A9F5F90932D050F
:10E54000E92FFF27EE0FFF1FEE0FFF1FE354F74FDA
:10E55000858518160CF4A9C1992309F4A6C1892F41
:10E56000992701966DE070E00E94DF9C9C01982F36
:10E57000E82FFF27EE0FFF1FEE0FFF1FE354F74FAB
:10E580008585181614F0222351F720932D058DC18F
:10E59000809102018093920A80918E088093930A61
:10E5A00080918F088093940A809190088093950AB7
:10E5B000809191088093960A809195088093970A9C
:10E5C000809196088093980A809197088093990A81
:10E5D00080919A0880939A0A8091980880939B0A68
:10E5E0008091990880939C0A80919B085CC18091DE
:10E5F0008C088093920A80916308863081F0809124
:10E60000E602823451F00E94FD7BE82FFF27E054A0
:10E61000FF4E84918093E60202C00E94FD7B8091B0
:10E620004F058093930A8091A9088093940A809162
:10E63000A2088093950A39C1F89480913F08E82F89
:10E64000FF27EE0FFF1FEC58F64F0190F081E02DF1
:10E65000E038F1051CF0EFE7F0E006C02FEFE138FD
:10E66000F20714F4E1E8FFEFE093920A809140088A
:10E67000E82FFF27EE0FFF1FEC58F64F0190F081B7
:10E68000E02DE038F1051CF0EFE7F0E006C07FEF89
:10E69000E138F70714F4E1E8FFEFE093930A809183
:10E6A0003E08E82FFF27EE0FFF1FEC58F64F0190B2
:10E6B000F081E02DE038F1051CF0EFE7F0E006C056
:10E6C0008FEFE138F80714F4E1E8FFEFE093940AE4
:10E6D00080913D08E82FFF27EE0FFF1FEC58F64F03
:10E6E0000190F081E02DE038F1051CF0EFE7F0E05B
:10E6F00006C02FEFE138F20714F4E1E8FFEF789459
:10E70000E093950A809148048093960A8091490489
:10E710008093970A80914A048093980A80914B04D1
:10E720008093990A80914C0480939A0A80914D04B9
:10E7300080939B0A80914E0480939C0A80914F04A1
:10E74000B2C08091CC05863018F01092CC0585E0DF
:10E750008093920A80919C088093930A809141044F
:10E7600090914204A0914304B0914404BC01CD01B6
:10E7700025E030E040E050E00E94149D3093950A7F
:10E780002093940A80913D0490913E04A0913F040F
:10E79000B0914004BC01CD0125E030E040E050E004
:10E7A0000E94149D3093970A2093960A80919208B4
:10E7B0008093980A809193088093990A8091940895
:10E7C00080939A0A8091470480939B0A80912E053A
:10E7D00080939C0A8091A5079091A60797FD0396C8
:10E7E00095958795959587955EC082E08093920A6E
:10E7F0008093930A81E08093940A89E38093950A39
:10E80000809103018093960A8091B1058093970AC5
:10E810009091B2059093980A8F778093B10590718B
:10E820009093B2058091AA088093990A8091520A28
:10E8300080939A0A8091350A80939B0A80919E0862
:10E8400080939C0A8091AF082EC0809171088093BC
:10E85000920A8091AD088093930A80916F01809312
:10E86000940A80916A088093950A80916B0880933E
:10E87000960A80916C088093970A80916E0180932C
:10E88000980A80916E088093990A80916F0880930E
:10E890009A0A8091700880939B0A8091F80A80936D
:10E8A0009C0A8091CF0780939D0A8091A10A8823BA
:10E8B00009F479C16091A20A8091A601681719F044
:10E8C0008AEF8093A4016093A60181E080938F0179
:10E8D0004091A30A5091A40ACA0181509E4F8F5FB4
:10E8E0009340B0F42091A50A3091A60AC901815045
:10E8F0009E4F8F5F934060F48091490885FF08C068
:10E9000050931A0540931905309318052093170565
:10E910008091A90A9091AA0A21E08936920724F4ED
:10E9200090939101809390012091B30A3091B40AA1
:10E9300080911B0390911C038217930740F48091F0
:10E94000EE02882321F430931C0320931B03862FAF
:10E9500099278936910509F4A5C08A36910544F4B2
:10E960008736910571F08836910509F462C023C19C
:10E970008A36910509F414C18B36910509F4E2C079
:10E980001AC18091B50A8093E20A8091B60A8093F9
:10E99000E40A8091B70A8093E30A8091B80A8093D1
:10E9A0008E018091B90A8093E60A8091BA0A809319
:10E9B000A5018091BB0A80932A058091BC0A8093AF
:10E9C000160580911B048823F9F02091BD0A30912F
:10E9D000BE0A37FD19C03093600420935F04909104
:10E9E0007308992389F08FE0989FC0011124281B98
:10E9F000390BC90188599E4F68E671E00E94DF9C7F
:10EA00009093600480935F0420912105309122054A
:10EA10008091BF0A9091C00A280F391F37FF02C0AA
:10EA20002F5F3F4F35952795309322052093210581
:10EA3000C2C08091B50A8093770A8091B60A80930C
:10EA4000780A8091B70A8093790A8091B80A8093F6
:10EA50007A0A8091B90A80937B0A809195079091F8
:10EA6000BA0A892B809395079091960793708091AD
:10EA7000BB0A8C70982B909396078091BC0A809368
:10EA800028058091BD0A809396018091BE0A8093EB
:10EA9000E50A8091BF0A809324058091C00A809383
:10EAA000230589C08091B50A80936D0A8091B60ACA
:10EAB00080936E0A8091B70A80936F0A8091B80A9A
:10EAC0008093700A8091B90A9091BA0A9093720A61
:10EAD0008093710A8091BB0A9091BC0A9093740A4A
:10EAE0008093730A8091BD0A992787FD9095909332
:10EAF000AF098093AE098091BE0A8093360480915D
:10EB0000BF0A9091C00A9C01442737FD4095542FBD
:10EB1000DA01C90163E0880F991FAA1FBB1F6A951C
:10EB2000D1F7820F931FA41FB51F820F931FA41F3D
:10EB3000B51F8093370490933804A0933904B093A1
:10EB40003A0439C08091B50A809327058091B60AAE
:10EB5000809326058091B70A809325059091B80A85
:10EB6000992349F08091AA01882319F081518330BB
:10EB700010F49093AA018091B90A8093570580916F
:10EB8000BA0A809356058091BB0A9091BC0A909373
:10EB90005405809353058091BD0A809355050BC0A1
:10EBA0000E94647C08C010921A05109219051092F8
:10EBB0001805109217051F910F91FF90EF9008957F
:10EBC00080916C0A882319F480E090E008954598BC
:10EBD0008DE79AE09093760A8093750A90912905C3
:10EBE000E92FFF27E956FE4F9F5F9093290580810B
:10EBF00080937F0A9D3010F01092290510926C0AC4
:10EC00000E94657181E080937C0A80917D0A8093E7
:10EC10009E0A8EBD81E090E0089587B18C6087B92F
:10EC2000429843981092300580E88093A801109292
:10EC30002F058093A70108958091AE099091AF09A7
:10EC400081589F4F39F08091AE099091AF0981585A
:10EC500080933A05809135058150809335058F3F2B
:10EC600009F052C18091860880933605809188080A
:10EC70008093370589E08093350580910E049927AC
:10EC800080739070892B21F48091B20580FF1DC0A4
:10EC900080918A08882351F080913805882319F4DF
:10ECA00084E08093300581E08093380580918B0863
:10ECB000882379F080913905882319F484E08093C2
:10ECC0002F0581E08093390504C010923805109219
:10ECD000390580913805882309F082C08091AC08FD
:10ECE000282F332724FF07C080914604882319F476
:10ECF00025FD8FC090C090918708983F48F0809183
:10ED0000300A8D3D28F08091360588236CF00AC0CA
:10ED1000983F78F08091300A853059F4809136051B
:10ED200087FF02C0429A01C0429881E08093A80107
:10ED300054C0809130058150809330058F3F09F099
:10ED40006BC08091AF0885FF2FC090913A05892F45
:10ED5000869580933005992361F490932E058091D8
:10ED6000360587FF02C0429A01C042981092A8015E
:10ED700053C081E080932E058091A80190913605C3
:10ED8000882349F480933A0580E48093A80199236D
:10ED90000CF43FC040C0982311F0429A01C0429841
:10EDA00086958093A80138C08091300A869580931B
:10EDB00030058091A801813021F410923A0580E459
:10EDC00001C086958093A8018091A8019091360595
:10EDD000892311F0429A01C0429810922E051CC05E
:10EDE000809130058150809330058F3FA9F489E0F0
:10EDF000809330058091A801813011F480E801C032
:10EE000086958093A8018091A80190918A08892312
:10EE100011F0429A01C0429880913905882309F087
:10EE200043C09091AC0897FF07C0809146048823A7
:10EE300019F496FD52C053C090918908983F48F04C
:10EE40008091590A8D3D28F08091370588236CF018
:10EE50000AC0983F78F08091590A853059F4809122
:10EE6000370587FF02C0439A01C0439881E0809331
:10EE7000A70136C080912F05815080932F058F3FC9
:10EE800079F58091590A869580932F058091A70185
:10EE9000813011F480E401C086958093A7018091B0
:10EEA000A7019091370517C080912F05815080935D
:10EEB0002F058F3FA9F489E080932F058091A7014A
:10EEC000813011F480E801C086958093A70180917C
:10EED000A70190918B08892311F0439A01C04398B0
:10EEE000429B05C080910D04886080930D04439B74
:10EEF00006C080910D04806180930D040895809177
:10EF00000D048F7E80930D0408950F931F93CF936C
:10EF1000DF93482FEB0180914704E42FFF27843BC8
:10EF2000D8F08F010E0F1F1FF801EC58F64F8081AB
:10EF300091819B01281B390BC90163E070E00E949D
:10EF4000DF9CCB01880F991F860F971F0654164F21
:10EF5000F8019183808306C0EE0FFF1FE654F64F41
:10EF600011821082E42FFF27EE0FFF1FEC58F64F9F
:10EF7000D183C083DF91CF911F910F9108954FB737
:10EF800024E130E0F8948091C9008F778093C90024
:10EF90008091C9008F7B8093C9008091C9008F7DCB
:10EFA0008093C900832F99278093CD002093CC00B4
:10EFB0008091C80082608093C80080E18093C9007E
:10EFC0008091CA008F778093CA008091CA008F7B9E
:10EFD0008093CA008091CA008F7D8093CA0080917F
:10EFE000CA008F7E8093CA008091CA00877F809379
:10EFF000CA008091C9008B7F8093C9008091CA00AC
:10F0000084608093CA008091CA0082608093CA00A5
:10F010008091C80087FF03C08091CE00F9CF809116
:10F02000C90080688093C9004FBF0895EF92FF9296
:10F030000F931F93CF93DF93482F00E010E0809150
:10F04000A901813061F41092A90184E480933D0507
:10F0500010923F0510923E051092400503C2809128
:10F060003D05882319F421E030E001C0980190911A
:10F070003E05992371F4232B11F081E010C084E444
:10F0800080933D0590933F0590933E0590934005F6
:10F09000D2C1913069F4232B09F0C3C182E080937F
:10F0A0003E0580913F058F5F80933F0583E0C1C19E
:10F0B0009230D1F4232B09F0B4C183E080933D0555
:10F0C0004093400590913F05923039F410924105EC
:10F0D00047FF03C081E08093410583E080933E05B4
:10F0E0009F5F90933F05A7C1933009F09AC1232BEE
:10F0F00009F097C190933D0582E080933E05809191
:10F100003F058F5F80933F0520914005822F99270F
:10F11000782F6627842F9927682B792B8091630895
:10F12000813051F47370CB018050924063E070E005
:10F130000E94DF9CEB0119C0823069F47770CB012B
:10F140008050944066E070E00E94DF9CEB012695C1
:10F15000269526950CC0EB01D370C856D140CE0140
:10F16000D7FD0196EC01D595C79526952695022FDA
:10F1700011270F7010700F5F1F4F0D30110508F031
:10F1800049C10230110519F404E010E005C0043053
:10F19000110511F402E010E0D801A00FB11FFD012C
:10F1A000EC58F64F808191819E01281B390BC901D3
:10F1B00037FF03C0909581959F4F069704F5E09126
:10F1C000A508EE2351F0FF27EE0FFF1FEC58F64F76
:10F1D000808191818436910594F480914704883C24
:10F1E00030F480914704865F8093470408C088EC20
:10F1F0008093470480916F008F7D80936F00AC589F
:10F20000B64F8D919C91BC01660F771F680F791FD7
:10F210006C0F7D1F77FF02C06D5F7F4F7B01F59400
:10F22000E794F594E794CE0101968E159F0524F49A
:10F230000894E108F10808C0CE010197E816F90624
:10F240001CF40894E11CF11C0630110509F0CEC035
:10F25000C536D1050CF4A5C090913C05E92FFF27D8
:10F26000E951F54FE081ED3729F480913B05809518
:10F2700080933B05963061F480913B05882311F023
:10F28000E338B9F0882309F088C0ED3791F085C0E4
:10F29000993009F082C080913B05882329F4809140
:10F2A000F00A833831F079C08091F00A8D3709F087
:10F2B00074C08091E80A8D3739F48091E90A833867
:10F2C00099F463E87FEF0DC0833871F48091E90A07
:10F2D000833819F460E070E004C08D3729F46DE7DD
:10F2E00070E085E00E9485778091EA0A992787FD82
:10F2F0009095BC0186E00E9485778091EB0A992762
:10F3000087FD9095BC018BE00E9485778091EC0A87
:10F31000992787FD9095BC018CE00E9485778091AC
:10F320003C058930D1F58091EE0A8D3749F4809102
:10F330008409909185090596BC0188E00E94857733
:10F340008091EF0A8D3749F4809184099091850965
:10F350000597BC0188E00E9485778091840990918F
:10F36000850983589F4F1CF483E89FEF09C0809163
:10F370008409909185098E37910534F08DE790E0EE
:10F3800090938509809384098091ED0A992787FDE0
:10F390009095BC018AE00E94857710923C051092FE
:10F3A0003B05CA30D1055CF480913C058F5F8093AA
:10F3B0003C05E82FFF27E951F54F83E880838091D2
:10F3C0003C058A3011F410923C058FEFCC39D807F8
:10F3D0006CF480913C05E82FFF27E951F54F8DE74C
:10F3E000808380913B05809580933B050530110516
:10F3F00018F4B701802F0BC00530110519F4BE01B8
:10F4000087E005C007301105B1F4BE0189E00E9414
:10F41000857711C00231110570F081E08093A90158
:10F420000AC081E08093A90110923F051092410526
:10F4300084E480933D0580913F05803198F0809170
:10F440004105882331F48091A901882311F4809328
:10F45000400110923F051092410510923E0584E450
:10F4600080933D05E6E0CDB7DEB70C94579DCF9372
:10F47000FC0197FF05C0CFEFF095E195FF4F01C06C
:10F48000C1E028E631E0CF01B9010E94DF9CFC0118
:10F490008B35910554F08B5590408A35910538F4A1
:10F4A00084EB90E08E1B9F0BFC0141E00DC0CF016F
:10F4B000855B90408A35910518F4E45BF04003C009
:10F4C0002E1B3F0BF9014FEFEE0FFF1FED5CF64FC8
:10F4D000259134918C2F992787FD9095289FB00115
:10F4E000299F700D389F700D1124842F992787FD57
:10F4F0009095689FA001699F500D789F500D112431
:10F50000CA01CF9108952AE530E0281B390BC901C3
:10F510000E94377A089508950895089508950895EA
:10F5200080E090E008951092F30A1092F20A10928F
:10F53000F70A1092F60A1092F50A1092F40A109245
:10F54000F80A82E390E00E94DF19909343058093CC
:10F5500042050895E82FFF2783E0EE0FFF1F8A95ED
:10F56000E1F7ED5EF64F95819F3F19F480E090E062
:10F570000895993C18F4892F99270895808182FF76
:10F5800007C08AE0989FC0011124885097400895D1
:10F59000892F99270895A0E0B0E0E1EDFAE70C94F7
:10F5A000389D80914205909143050E94E819882377
:10F5B00009F4C0C08091420590914305C296909392
:10F5C000430580934205C0E0D0E07E01BB247FEF7D
:10F5D000C72EDB2C03E119E0F801838187FF14C0FB
:10F5E000B3948581893C30F08D2D0E94AA7AC80F92
:10F5F000D91F02C0C80FD11DF8018181E80EF11C8E
:10F6000086818C1508F4C82ED394085F1F4FFBE049
:10F61000FD1510F7C092F80AEF2841F52091480532
:10F620003091490540914A0550914B05BB27A52FC4
:10F63000942F832F9093470580934605AA27BB27D5
:10F64000281B390B4A0B5B0BCE01AA27BB27280FBF
:10F65000391F4A1F5B1F209348053093490540938B
:10F660004A0550934B05C5E0D0E013C08091460594
:10F67000909147058C179D0718F4C81BD90B02C041
:10F68000C0E0D0E08B2D9927880F991FC80FD91F94
:10F690002596D093F30AC093F20ACF3FD10578F4B0
:10F6A00080912601909127018C9F90018D9F300DB4
:10F6B0009C9F300D1124C90164E670E013C0CE0197
:10F6C00096958795969587952091260130912701EB
:10F6D000289FA001299F500D389F500D1124CA0169
:10F6E00069E170E00E94CB9C7093F50A6093F40A84
:10F6F00080914405909145058C0F9D1F9093450581
:10F700008093440552E0813D9507A0F02091F60AD0
:10F710003091F70A2F5F3F4F805D9240E2E0813DDC
:10F720009E07C0F790934505809344053093F70AF0
:10F730002093F60AE9E0CDB7DEB70C94549D3091E2
:10F740005805E32FFF2783E0EE0FFF1F8A95E1F7AF
:10F75000ED5EF64F2781422F552747FD509580914A
:10F7600059059927841795072CF420935905309350
:10F770005B050AC0222341F080915A05992748175A
:10F78000590714F420935A05832F8F5F80935805EF
:10F790008C30D0F01092580580915A058F3F19F0A7
:10F7A0008093510502C010925105809159058093B4
:10F7B000520580915B05809350058FEF80935A0529
:10F7C0001092590510925B05089595E1899F802D4F
:10F7D00011240E941D9585EA9CE09F938F938FEEE4
:10F7E00094E99F938F93E0919805F091990509957D
:10F7F0000F900F900F900F900895CF93C0E040911D
:10F80000AA0140934F0580910E0485FF0CC08091A2
:10F810000504882331F080916308863011F4CEE02E
:10F8200029C0C0E127C0809128058823D1F0282F66
:10F830003327C90101968197A4F480914604882357
:10F8400041F4F901E20FF31FE651F64F849188234A
:10F8500041F4220F331F2751364FF901C491CC23B5
:10F8600049F48091AF0886FD03C01092AA0104C03C
:10F87000C42F02C0C0934F0580915C058C1771F4B2
:10F8800080915D0590915E050E94E819882319F426
:10F8900080E090E017C080EA9FE002C080ED97E032
:10F8A0000E94DF1990935E0580935D05CC2331F0B3
:10F8B0008091AA01C81711F41092AA01C0935C05A7
:10F8C0008C2F9927CF91089520E030E050E080916F
:10F8D000C00A992789389105B9F08A38910534F41E
:10F8E00081309105F1F00297F9F021C08D38910532
:10F8F000A1F08E38910524F48A38910541F017C0A3
:10F900008E38910539F013C021E53BE008C029E2AB
:10F910003CE005C029EF3AE002C025E23BE05CE2B2
:10F9200006C023EC32E002C026ED32E054E09091B4
:10F93000B50A40E08091B60A481770F4951760F454
:10F94000D901A90FB11DE42FFF27EE55F54F858989
:10F950008C939F5F4F5FEECF089520E335E7809152
:10F9600041018B3211F08D32F9F480914E08282F2D
:10F97000332780913B0490913C04829FA001839F98
:10F98000500D929F500D1124CA0163E070E00E9457
:10F99000DF9CCB019B01205D3A48C196C19708F0DE
:10F9A0003FC02EEF34E73CC0803229F580910E0431
:10F9B00081FF36C020914C0530914D05205D3A48BD
:10F9C00055E72133350748F085E72439380718F41F
:10F9D00020E335E702C02456304045E720333407A2
:10F9E000F8F454E72D3C350718F020E335E718C04C
:10F9F0002C593F4F15C08E3549F4909136048AE05A
:10FA0000989F90011124205D3A480AC0863741F43E
:10FA1000909136048AE0989FC0011124281B390B6D
:10FA2000C90108951F9399278A38910509F4A5C142
:10FA30008B38910524F48938910551F05EC38D38D7
:10FA4000910509F491C28E38910509F4EAC155C3B4
:10FA50000E94FD7B182F80932B0C80914104909184
:10FA60004204A0914304B0914404BC01CD0124E6BA
:10FA700030E040E050E00E94149DDA01C9018C5052
:10FA80009E4F9093570B8093560B112319F40E94AD
:10FA9000AD7C02C080E395E790935D0B80935C0B97
:10FAA00080915C0B90915D0B90935F0B80935E0B4C
:10FAB0009093610B8093600B2091560B3091570B04
:10FAC00080915A0B90915B0B2817390724F43093DF
:10FAD0005B0B20935A0B8091580B9091590B821716
:10FAE000930724F43093590B2093580B1092530B27
:10FAF00081E59BE09093700580936F0580914101B3
:10FB00008093770B80910D0480FF02C083E401C0D5
:10FB100080E28093780B20912805222311F1822F17
:10FB20006AE00E94BF9C805D8093620B822F0E94DE
:10FB3000BF9C892F805D8093630B8AE38093640B65
:10FB400081E1289FF0011124A5E6BBE0E55DF54FBA
:10FB50009FE084918D939150319697FFFACF80E288
:10FB600041C080910504882361F0A2E6BBE0E3E692
:10FB7000FCE094E184918D939150319697FFFACFF8
:10FB8000B9C280910E0485FF0CC0A2E6BBE0E9E794
:10FB9000FCE094E184918D939150319697FFFACFD8
:10FBA000A9C280914E05882301F1A2E6BBE0ECE5F5
:10FBB000FCE096E084918D939150319697FFFACFB7
:10FBC00080910101805D8093660BA9E6BBE0E0EBCC
:10FBD000F8E09BE081918D93915097FFFBCF80E2FD
:10FBE0008093740B8093750BB9C030915605332305
:10FBF00009F499C087E58093620B80E58093630BDD
:10FC000040E24093640B20915705822F6AE00E94E6
:10FC1000BF9C805D8093650B822F0E94BF9C892FC3
:10FC2000805D8093660B8FE28093670B832F0E9429
:10FC3000BF9C805D8093680B832F0E94BF9C892F9F
:10FC4000805D8093690B40936A0B2091530530913E
:10FC5000540583E0293E380780F0C90168EE73E05F
:10FC60000E94CB9CCB01805D80936B0BC90168EE39
:10FC700073E00E94CB9C9C0102C040936B0B253625
:10FC8000310580F0C90164E670E00E94CB9CCB0195
:10FC9000805D80936C0BC90164E670E00E94CB9C90
:10FCA0009C0103C080E280936C0BC9016AE070E0A4
:10FCB0000E94CB9CCB01805D80936D0BC9016AE0F3
:10FCC00070E00E94CB9C805D80936E0B8DE68093EC
:10FCD0006F0B80E28093700B20915505253660F004
:10FCE000822F64E60E94BF9C805D8093710B822FFF
:10FCF0000E94BF9C292F02C08093710B822F6AE063
:10FD00000E94BF9C805D8093720B822F0E94BF9CDB
:10FD1000892F805D8093730B83E78093740B80E25F
:10FD20008093750BE7C1809132048823D1F4A2E659
:10FD3000BBE0E1E9FCE090E184918D939150319634
:10FD400097FFFACF92E39093720B8EE28093730B3E
:10FD500080E38093740B9093750B82E68093760B0F
:10FD6000C9C1A2E6BBE0EFE8FCE094E184918D9389
:10FD70009150319697FFFACFBDC180914104909187
:10FD80004204A0914304B0914404BC01CD0124E697
:10FD900030E040E050E00E94149DDA01C9018C502F
:10FDA0009E4F90933F0C80933E0C80912B0C8823A8
:10FDB00019F40E94AD7C02C080E395E79093410C5A
:10FDC0008093400C88E78093420C80916E0A809368
:10FDD000430C80916D0A81FF02C084E407C08091CA
:10FDE0006F0A833011F480E201C081E28093440CF9
:10FDF00089E29CE09093700580936F058091960155
:10FE00008093500C8091440C8093520C8091730A23
:10FE10009091740A97FD0196959587958093450C6E
:10FE200069C10E949F7B8091410490914204A091FE
:10FE30004304B0914404BC01CD0124E630E040E02D
:10FE400050E00E94149DDA01C9018C509E4F90939E
:10FE5000140B8093130B80912601909127019093AE
:10FE60000E0B80930D0B80912601909127019093AA
:10FE7000100B80930F0B80910E0A90910F0A97FD43
:10FE80000196959587958093FF0A8093060B2091A4
:10FE9000730A3091740A37FF02C02F5F3F4F3595C8
:10FEA00027952093040B8091710A9091720A64E166
:10FEB00070E00E94CB9C6093050B20930B0B60932A
:10FEC0000C0B80912B0C882319F40E94AD7C02C08E
:10FED00080E395E790931C0B80931B0B88E780933E
:10FEE0001D0B80912601909127019093180B809310
:10FEF000170B809151058C5E8093110B80915205F8
:10FF00008C5E8093120B8091F60A9091F70A6AE05A
:10FF100070E00E94CB9C70931A0B6093190B809138
:10FF20002B0C8093FB0A8091F20A9091F30A909334
:10FF3000160B8093150B89EF9AE0909370058093D0
:10FF40006F052091E8023091E902C9016CE370E08D
:10FF50000E94CB9C6093200BC9016CE370E00E946F
:10FF6000CB9C8093210BC6C00E949F7B8091710A1D
:10FF70009091720A64E670E00E94CB9C70933B0BF8
:10FF800060933A0B80910E0A90910F0A97FD0196AB
:10FF90009595879580932B0B80919001909191017D
:10FFA00097FD01969595879580932C0B8091CF07AF
:10FFB00080932F0B8091730A9091740A97FD01969C
:10FFC000959587958093300B80910201482F552796
:10FFD0009A012E5F3F4F80912601909127012817AB
:10FFE000390784F48091260190912701841B950B99
:10FFF0009C01220F331F280F391F822F86508093B8
:020000021000EC
:10000000370B02C01092370B8091370B853618F0F2
:1000100084E68093370B8091280599279093390BBC
:100020008093380B8091410490914204A091430445
:10003000B0914404BC01CD0124E630E040E050E042
:100040000E94149DDA01C9018C509E4F90933D0B84
:1000500080933C0B80912601909127019093320B65
:100060008093310B80912601909127019093340B5E
:100070008093330B80912B0C882319F40E94AD7C64
:1000800002C080E395E790933F0B80933E0B8091F5
:100090002B0C88588093400B80912601909127016A
:1000A0009093440B8093430B809151058C5E809319
:1000B000350B809152058C5E8093360B8091F60A49
:1000C0009091F70A6AE070E00E94CB9C7093460B17
:1000D0006093450B1092270B8091F20A9091F30ADE
:1000E0009093420B8093410B85E29BE090937005C7
:1000F00080936F052CE230E002C020E030E0C901BF
:100100001F910895EF92FF920F931F93CF93DF9368
:1001100080914C0590914D059C0153E0220F331FB7
:100120005A95E1F7281B390B8091310390913203E6
:10013000280F391F37FF02C0295F3F4F43E0359535
:1001400027954A95E1F730934D0520934C05909102
:100150006005992309F026C380915F05282F332776
:10016000442755278F5F80935F05F90121313105C1
:1001700008F015C3E757FF4F0C94669D80910E045D
:1001800085FF2AC080E00E941D95809126019091F4
:1001900027016AE070E00E94DF9C9F938F9380911B
:1001A0002601909127016AE070E00E94DF9C7F9316
:1001B0006F938BEB9CE09F938F9380E195E99F93E6
:1001C0008F93E0919805F091990509952DB73EB769
:1001D000285F3F4F2DBF28C080E00E941D95809171
:1001E0002601909127016AE070E00E94DF9C9F93B6
:1001F0008F9380912601909127016AE070E00E9420
:10020000DF9C7F936F9388EC9CE09F938F938FEE9E
:1002100094E99F938F93E0919805F0919905099542
:100220008DB79EB708968DBF8091520A80FF3FC060
:1002300080915E048823E9F08AE00E941D958091F8
:10024000410199279F938F9380914104909142049B
:10025000A0914304B0914404BC01CD0124E630E0F8
:1002600040E050E00E94149D3F932F9385ED9CE069
:10027000C8C68AE00E941D95809141049091420475
:10028000A0914304B0914404BC01CD0124E630E0C8
:1002900040E050E00E94149D3F932F9381EE9CE03C
:1002A0009F938F938FEE94E99F938F93D1C78AE0AA
:1002B0000E941D958CEE9CE09F938F938FEE94E9A6
:1002C0000C94538A80910E0485FF2AC085E10E9418
:1002D0001D958091E8029091E9026CE370E00E9424
:1002E000CB9C9F938F938091E8029091E9026CE3FD
:1002F00070E00E94CB9C7F936F9386EF9CE09F936E
:100300008F9380E195E99F938F93E0919805F09109
:10031000990509952DB73EB7285F3F4F2DBF28C0DF
:1003200085E10E941D958091E8029091E9026CE3BD
:1003300070E00E94CB9C9F938F938091E8029091F4
:10034000E9026CE370E00E94CB9C7F936F9383E0A3
:100350009DE09F938F938FEE94E99F938F93E0910D
:100360009805F091990509958DB79EB708968DBFB0
:100370008FE10E941D9580E690E09F938F9380917E
:100380000E0A90910F0A9F938F9380E19DE09F93B7
:100390008F93CFEED4E9DF93CF93E0919805F0915E
:1003A0009905099580910D042DB73EB7285F3F4F01
:1003B0002DBF80FF06C089E20E941D958BE19DE064
:1003C0006FC389E20E941D958DE19DE0E2C6809198
:1003D0000E0485FF1BC08AE20E941D958091F60ADB
:1003E0009091F70A9F938F938FE19DE09F938F9356
:1003F00080E195E99F938F93E0919805F09199059D
:1004000009958DB79EB706968DBF1BC08AE20E94E4
:100410001D958091F60A9091F70A9F938F9387E23A
:100420009DE09F938F938FEE94E99F938F93E0913C
:100430009805F091990509952DB73EB72A5F3F4F72
:100440002DBF86E30E941D958091F20A9091F30AD8
:100450006AE070E00E94CB9C9F938F938091F20A98
:100460009091F30A6AE070E00E94CB9C7F936F93B7
:100470008FE29DE09F938F938FEE94E99F938F93EC
:10048000E0919805F091990509958DB79EB708966A
:10049000E7C689E00E941D958BE39DE09F938F93B3
:1004A0000FEE14E91F930F93E0919805F0919905D1
:1004B00009958EE10E941D950F900F900F900F905F
:1004C0008DE39DE09F938F931F930F93E091980589
:1004D000F0919905099583E30E941D950F900F9067
:1004E0000F900F908FE39DE09F938F931F930F9337
:1004F000E0919805F091990509958FE30E941D956B
:100500000F900F900F900F9081E49DE09F938F9339
:100510001F930F93E0919805F091990509958EE747
:100520000E941D950F900F900F900F9087E59DE012
:100530009F938F931F930F93B8C78091A401882333
:1005400009F462C08DE50E941D958DE69DE09F93A4
:100550008F93CFEED4E9DF93CF93E0919805F0919C
:100560009905099584E50E941D950F900F900F90B5
:100570000F9080916E0A99279F938F938FE69DE04D
:100580009F938F93DF93CF93E0919805F091990516
:1005900009958EE50E941D952DB73EB72A5F3F4F06
:1005A0002DBF8091710A9091720A6AE070E00E94FA
:1005B000CB9C7F936F9388E79DE09F938F93DF930E
:1005C000CF93E0919805F091990509958DB79EB765
:1005D00006968DBF80916F0A833081F480916D0AF9
:1005E00081FF06C08BE50E941D9582E89DE0D1C584
:1005F0008BE50E941D9585E89DE0CBC58BE50E94AB
:100600001D9588E89DE04BC784E0FCC38091A40160
:10061000882309F47AC0809162052FEEE22E24E946
:10062000F22E882309F44BC089E60E941D95809123
:10063000270599279F938F938BE89DE09F938F9336
:10064000FF92EF92E0919805F0919905099585E761
:100650000E941D952DB73EB72A5F3F4F2DBF809159
:10066000960199279F938F9300E610E01F930F93B5
:100670008091730A9091740A9F938F9386E99DE00D
:100680009F938F93FF92EF92E0919805F0919905D7
:10069000099582E70E941D958DB79EB70A968DBF7A
:1006A0008091250599279F938F931F930F93809196
:1006B000260599279F938F9382EA9DE091C689E64C
:1006C0000E941D958091960199279F938F9380E6B4
:1006D00090E09F938F938091730A9091740A9F93F7
:1006E0008F938091700A99279F938F9382EB9DE05F
:1006F0009F938F93FF92EF92E0919805F091990567
:1007000009958DB79EB70C96ABC585E07BC39091DC
:1007100028059923D1F080916C05882381F09132CE
:1007200070F487E00E94E57B83E90E941D9580912B
:10073000280599279F938F938BEC9DE0CDC383E988
:100740000E941D9586ED9DE0DCC380910E049FEE16
:10075000E92E94E9F92E85FF06C084E90E941D95D3
:100760008CED9DE003C483E90E941D958FEE9DE012
:10077000FDC380918E0C863059F4809162058823E8
:1007800019F010926205B8C681E080936205B4C684
:10079000883009F0B1C60E94229581E004C490938C
:1007A0005F05B2C6913009F009C480915F05282F1A
:1007B0003327442755278F5F80935F05F901213147
:1007C000310508F09CC6E656FF4F0C94669D80915B
:1007D0000E0485FF43C080E00E941D958091F60ABB
:1007E0009091F70A9F938F93809126019091270112
:1007F0006AE070E00E94DF9C9F938F9380912601B6
:10080000909127016AE070E00E94DF9C7F936F93D4
:100810008091E8029091E9026CE370E00E94CB9C29
:100820009F938F938091E8029091E9026CE370E0CE
:100830000E94CB9C7F936F9385E09EE09F938F9364
:1008400080E195E99F938F93E0919805F091990548
:1008500009952DB73EB7225F3F4FCFC580E00E947C
:100860001D958091F60A9091F70A9F938F9380913E
:100870002601909127016AE070E00E94DF9C9F931F
:100880008F9380912601909127016AE070E00E9489
:10089000DF9C7F936F938091E8029091E9026CE373
:1008A00070E00E94CB9C9F938F938091E80290917F
:1008B000E9026CE370E00E94CB9C7F936F9380E22F
:1008C0009EE0EBC285E10E941D9580E690E09F933B
:1008D0008F9380919001909191019F938F938BE3DF
:1008E0009EE09F938F93CFEED4E9DF93CF93E09177
:1008F0009805F091990509958091520A2DB73EB758
:10090000285F3F4F2DBF80FF51C080915E04882338
:1009100039F18FE10E941D9580914104909142042C
:10092000A0914304B0914404BC01CD0124E630E021
:1009300040E050E00E94149D3F932F9385E49EE099
:100940009F938F938FEF94E99F938F93E0919805F6
:10095000F091990509958DB79EB706968DBF38C061
:100960008FE10E941D958091410490914204A091D5
:100970004304B0914404BC01CD0124E630E040E0E2
:1009800050E00E94149D3F932F938EE49EE09F932E
:100990008F93DF93CF93E0919805F0919905099596
:1009A0002DB73EB72A5F3F4F2DBF12C08FE10E9487
:1009B0001D9587E59EE09F938F93DF93CF93E09102
:1009C0009805F091990509950F900F900F900F9051
:1009D00089E20E941D958091410199279F938F93F1
:1009E00081E69EE031C48091A4018823F9F08BE276
:1009F0000E941D958091960199279F938F938091D6
:100A0000710A9091720A6AE070E00E94CB9C7F9319
:100A10006F9380E690E09F938F938091730A9091FB
:100A2000740A9F938F9384E69EE068C182E0EAC1D6
:100A30008FE30E941D958091F40A9091F50A9F938F
:100A40008F938091F20A9091F30A6AE070E00E941D
:100A5000CB9C9F938F938091F20A9091F30A6AE066
:100A600070E00E94CB9C7F936F938BE79EE09F93F7
:100A70008F93CFEED4E9DF93CF93E0919805F09177
:100A80009905099580910D042DB73EB7265F3F4F1C
:100A90002DBF80FF0AC082E50E941D958FE89EE071
:100AA0009F938F938FEF94E9FEC482E50E941D957A
:100AB00082E99EE06EC38091A4010FEEE02E04E96E
:100AC000F02E882309F449C084E50E941D95809189
:100AD0006E0A99279F938F938091700A99279F930D
:100AE0008F9385E99EE09F938F93E701FF92EF92AA
:100AF000E0919805F091990509958DB79EB70896F4
:100B00008DBF80916F0A833051F484E60E941D9559
:100B100088EA9EE09F938F93FF92EF920BC084E64A
:100B20000E941D958EEA9EE09F938F9380E195E948
:100B30009F938F93E0919805F091990509950F90F7
:100B40000F900F900F9080916D0A81FFDDC484E6B5
:100B50000E941D9584EB9EE01CC384E50E941D95B8
:100B60008AEB9EE003C2809161051FEEE12E14E93D
:100B7000F12E882309F45BC089E60E941D9583E06D
:100B80000E94AA7A6AE070E00E94CB9C9F938F93A8
:100B900083E00E94AA7A6AE070E00E94CB9C7F9377
:100BA0006F9382E00E94AA7A6AE070E00E94CB9C78
:100BB0009F938F9382E00E94AA7A6AE070E00E947D
:100BC000CB9C7F936F9381E00E94AA7A6AE070E0E9
:100BD0000E94CB9C9F938F9381E00E94AA7A6AE047
:100BE00070E00E94CB9C7F936F9380E00E94AA7A72
:100BF0006AE070E00E94CB9C9F938F9380E00E94FC
:100C0000AA7A6AE070E00E94CB9C7F936F9380ED9C
:100C10009EE09F938F93FF92EF92E0919805F09161
:100C2000990509952DB73EB72C5E3F4FE6C389E67F
:100C30000E941D9580E690E09F938F9380913209EA
:100C4000992787FD90959F938F9380912A099927E3
:100C500087FD90959F938F9380912209992787FD17
:100C600090959F938F9380911A09992787FD90956E
:100C70009F938F938DEE9EE09F938F93FF92EF92C1
:100C8000E0919805F091990509958DB79EB70E965C
:100C9000E7C28091610590913B08882309F4AFC0B9
:100CA000943009F4AEC09630C9F58EE70E941D95C8
:100CB00085E00E94AA7A6AE070E00E94CB9C9F9334
:100CC0008F9385E00E94AA7A6AE070E00E94CB9C34
:100CD0007F936F9384E00E94AA7A6AE070E00E949A
:100CE000CB9C9F938F9384E00E94AA7A6AE070E085
:100CF0000E94CB9C7F936F9380E09FE09F938F93A4
:100D00008FEE94E99F938F93E0919805F091990568
:100D100009952DB73EB7245F3F4F6FC3973008F456
:100D2000F3C38EE70E941D9588E00E94AA7A6AE0CC
:100D300070E00E94CB9C9F938F9388E00E94AA7AD8
:100D40006AE070E00E94CB9C7F936F9387E00E94E3
:100D5000AA7A6AE070E00E94CB9C9F938F9387E011
:100D60000E94AA7A6AE070E00E94CB9C7F936F9306
:100D700086E00E94AA7A6AE070E00E94CB9C9F9372
:100D80008F9386E00E94AA7A6AE070E00E94CB9C72
:100D90007F936F9385E00E94AA7A6AE070E00E94D8
:100DA000CB9C9F938F9385E00E94AA7A6AE070E0C3
:100DB0000E94CB9C7F936F9384E00E94AA7A6AE0A2
:100DC00070E00E94CB9C9F938F9384E00E94AA7A4C
:100DD0006AE070E00E94CB9C7F936F938FE09FE06E
:100DE0009F938F938FEE94E99F938F93E091980553
:100DF000F091990509958DB79EB7489631C2943008
:100E000021F486E00E94E57B7FC39630F1F48EE703
:100E10000E941D9580E690E09F938F9380914209F8
:100E2000992787FD90959F938F9380913A099927F1
:100E300087FD90959F938F938CE29FE09F938F9374
:100E40008FEE94E99F938F93CFC2973008F45CC3E1
:100E50008EE70E941D9580E690E09F938F9380918E
:100E60005209992787FD90959F938F9380914A0906
:100E7000992787FD90959F938F9380914209992799
:100E800087FD90959F938F9380913A09992787FDCD
:100E900090959F938F938FE39FE09F938F938FEE17
:100EA00094E99F938F93ECCE90912805992309F4B0
:100EB0004AC080916C058823F9F09132E8F487E00C
:100EC0000E94E57B83E90E941D9580912805992762
:100ED0009F938F9382E59FE09F938F938FEF94E989
:100EE0009F938F93E0919805F091990509952DB7FF
:100EF0003EB72A5F3F4F81C283E90E941D958DE571
:100F00009FE09F938F930FEE14E91F930F93E0914F
:100F10009805F091990509951F921F9290912805C7
:100F200081E1989FC0011124855D954F9F938F9318
:100F30001F930F93E0919805F091990509958DB74E
:100F40009EB70A968DC180910E04CFEEEC2EC4E9B7
:100F5000FC2E85FF06C084E90E941D9583E69FE074
:100F600005C083E90E941D9586E79FE09F938F93BC
:100F7000FF92EF929AC280918E0C863079F4809124
:100F80006105882319F01092610503C081E0809308
:100F9000610585E00E94E57B86E0A3C2883031F4DC
:100FA0000E94229582E080936005A4C2813009F0FE
:100FB000A3C20E942295109260059CC2923009F053
:100FC000A1C280915F05282F3327442755278F5FC3
:100FD00080935F05F9012131310508F090C2E55594
:100FE000FF4F0C94669D80E00E941D9580EB98E079
:100FF0009F938F938091010199279F938F938CE802
:101000009FE09F938F938FEF94E99F938F93E0914D
:101010009805F091990509952DB73EB7285F3F4F88
:10102000ECC185E10E941D958EEB98E09F938F9314
:10103000809102016AE00E94BF9C892F99279F93AB
:101040008F93809102010E94BF9C99279F938F9359
:101050008BE99FE09F938F938FEE94E99F938F93FB
:10106000E0919805F0919905099569CF8AE20E946F
:101070001D958CEA9FE09F938F93CFEED4E9DF9389
:10108000CF93E0919805F091990509958091520AC6
:101090000F900F900F900F9080FF41C080914908F2
:1010A0009091240481FD0BC0892F99279F938F93E2
:1010B00081EB9FE09F938F93DF93CF9313CFE091CA
:1010C0009805F0919905933318F08BEB9FE002C0DF
:1010D00082EC9FE09F938F93DF93CF9309950F90BE
:1010E0000F900F900F908091350AE0919805F09144
:1010F00099059091240480FF0BC0892F99279F9315
:101100008F9389EC9FE09F938F93DF93CF93A4C03D
:10111000892F99279F938F938FEC9FE0C4C085ED13
:101120009FE037C08FE30E941D958EED9FE09F9357
:101130008F93CFEED4E9DF93CF93E0919805F091B0
:10114000990509950F900F900F900F9080919F082F
:10115000882319F482EE9FE01CC080911B04E0916B
:101160009805F0919905882319F08BEE9FE002C055
:1011700082EF9FE09F938F93DF93CF9309950F901A
:101180000F900F900F908091AE0886FFBDC189EF40
:101190009FE09F938F93DF93CF9387C184E50E9455
:1011A0001D9580E090E19F938F93CFEED4E9DF937C
:1011B000CF93E0919805F091990509958091520A95
:1011C0000F900F900F900F9085FD03C085E090E188
:1011D00008C080918D080E94E947823358F48EE060
:1011E00090E19F938F93DF93CF93E0919805F091D7
:1011F000990516C0843B18F085E190E1F2CF80910B
:10120000AE08E0919805F091990585FF03C08CE147
:1012100090E102C083E290E19F938F93DF93CF939D
:1012200009950F900F900F900F908091A30888233D
:1012300009F46AC18EE50E941D958091A308992743
:101240009F938F938AE290E19F938F93DF93CF9345
:10125000E0919805F091990509958DB79EB706968E
:101260008DBF52C189E60E941D9585E390E19F9351
:101270008F93CFEED4E9DF93CF93E0919805F0916F
:10128000990509950F900F900F900F908091A208EB
:10129000E0919805F0919905882351F099279F9343
:1012A0008F938FE390E19F938F93DF93CF931ECE25
:1012B00083E490E19F938F93DF93CF93FAC0809163
:1012C0006305BFEEEB2EB4E9FB2E882309F053C073
:1012D0008EE70E941D9580916F0199279F938F93B0
:1012E00080913E08E82FFF27EE0FFF1FEC58F64FC6
:1012F000808191819F938F9380913D08E82FFF27F4
:10130000EE0FFF1FEC58F64F808191819F938F93D2
:1013100089E490E19F938F93FF92EF92E09198057B
:10132000F0919905099583E90E941D958DB79EB7A7
:101330000A968DBF80914008E82FFF27EE0FFF1F10
:10134000EC58F64F808191819F938F9380913F0855
:10135000E82FFF27EE0FFF1FEC58F64F8081918199
:1013600081589F4F9F938F938DE590E19F938F932B
:10137000FF92EF924CCE8EE70E941D9580914A0419
:1013800099279F938F938091490499279F938F93D7
:101390008091480499279F938F938CE690E19F93C7
:1013A0008F93FF92EF92E0919805F091990509953E
:1013B00083E90E941D958DB79EB70A968DBF8091D7
:1013C0004D0499279F938F9380914C0499279F9365
:1013D0008F9380914B0499279F938F9380E890E19E
:1013E0009F938F93FF92EF92E0919805F09199056A
:1013F00009952DB73EB7265F3F4F2DBF85C0809121
:101400006C05882309F480C08EE70E941D958091A9
:10141000520A86FD11C084E990E19F938F9380E189
:1014200095E99F938F93E0919805F091990509951F
:101430000F900F900F900F908091AC0899278F70AC
:101440009070892B89F083EA90E19F938F9380E1DC
:1014500095E99F938F93E0919805F09199050995EF
:101460000F900F900F900F908091520A82FF11C041
:101470008DEA90E19F938F9380E195E99F938F93FD
:10148000E0919805F091990509950F900F900F90B4
:101490000F908091520A83FD37C082EB90E19F93B9
:1014A0008F9380E195E99F938F93E0919805F09158
:1014B000990509950F900F900F900F9025C00091FE
:1014C0008E0C063089F480916305882319F0109200
:1014D000630503C081E08093630586E00E94E57B9D
:1014E00087E00E94E57B08C0013031F40E9422951C
:1014F0000093600510925F0510928E0C05C010924B
:101500005F0502C010926005E6E0CDB7DEB70C942F
:10151000579D4FB728E130E0F8948091C9008F774C
:101520008093C9008091C9008F7B8093C90080910E
:10153000C9008F7D8093C900832F99278093CD00A8
:101540002093CC008091C80082608093C80080E125
:101550008093C9008091CA008F778093CA008091E0
:10156000CA008F7B8093CA008091CA008091CA0014
:101570008F7E8093CA008091CA0088608093CA00E1
:101580008091C9008B7F8093C9008091CA008460DC
:101590008093CA008091CA0082608093CA008091C3
:1015A000C80087FF03C08091CE00F9CF8091C900A9
:1015B00080688093C90080916C0C846080936C0C6F
:1015C0004FBF089590913D05992341F48F3031F438
:1015D0009093650580E580933D050895E09165054C
:1015E000EF5FE0936505E83121F481E080936405C5
:1015F0000895E93120F089E1809365050895FF277A
:10160000EB5AF34F80830895A0E0B0E0EAE0FBE8F6
:101610000C94379D91E0D92E82E0A82EBD2CE12CB0
:1016200001E0F02E80916C0C82FDB5C080916F00BE
:101630008F7D80936F00E091A508EE2351F0FF2786
:10164000EE0FFF1FEC58F64F808191818436910593
:101650005CF480914704883C20F4809147048C5EC0
:1016600001C088EC809347048091560C682F77273F
:10167000809166058150809366058F3F31F41CE7A9
:10168000C12E82E08093660502C0C4E2CC2E40E009
:101690004C1508F07EC0EA2DFF27EB5AF34F8081EE
:1016A0008D2111F06E297F298D2D9927880F991F83
:1016B000D82E882319F4B1E0DB2EAD0CEE0CFF1C04
:1016C00020E0E21628E0F20609F061C0A1E0EA2E6F
:1016D000F12CCB018050944065E070E00E94DF9CCB
:1016E000AB2DBB27FD01EA0FFB1FEC58F64F8081A5
:1016F00091819C01220F331F280F391F260F371F9E
:1017000037FF02C02D5F3F4FE901D595C795D595AD
:10171000C795CB0101968C179D0714F4219706C03D
:1017200061507040C617D7070CF42196809147048A
:10173000833CD8F08D010A0F1B1FF801EC58F64FBF
:1017400080819181FE01E81BF90BCF0163E070E01D
:101750000E94DF9CCB01880F991F860F971F0654AC
:10176000164FF8019183808307C0AA0FBB1FA654B0
:10177000B64F11961C921E92EB2DFF27EE0FFF1F06
:10178000EC58F64FD183C08360E070E0B3944F5FB4
:101790007FCF1092400110926405EAE0CDB7DEB72A
:1017A0000C94539D0895089540E050E080916705A2
:1017B000909168059C01220F331F280F391F8091DB
:1017C000310390913203280F391F37FF02C02D5F7C
:1017D0003F4F35952795359527953093680520938C
:1017E0006705809141018B32D9F480914E08282FF2
:1017F000332780913B0490913C04829FA001839FFA
:10180000500D929F500D1124CA0157FD4F96AC0107
:1018100025E0559547952A95E1F74B5F5F4F3DC011
:101820008D32D9F480914E08282F332780913B04C4
:1018300090913C04829FA001839F500D929F500D78
:101840001124CA0157FD4F96AC0195E05595479577
:101850009A95E1F74550504020C0803271F4809154
:101860000E0481FF1AC0C90137FD4F96AC0185E017
:10187000559547958A95E1F710C08E3529F48091EA
:101880003604482F552709C0863739F4809136042D
:10189000992744275527481B590BCA01AA2797FDAA
:1018A000A095BA2F80939D0290939E02A0939F02D1
:1018B000B093A00208950F931F930E949F7B809185
:1018C000260190912701AA2797FDA095BA2F809312
:1018D000CC019093CD01A093CE01B093CF01809124
:1018E000F20A9091F30AAA27BB278093DF01909315
:1018F000E001A093E101B093E2010AE010E08091E1
:10190000F60A9091F70AB8010E94CB9CCB01AA2756
:10191000BB278093F2019093F301A093F401B0935D
:10192000F5018091410490914204A0914304B0914B
:101930004404BC01CD0124E630E040E050E00E94C8
:10194000149D2093050230930602409307025093A2
:1019500008028091900190919101AA2797FDA0958E
:10196000BA2F8093180290931902A0931A02B09391
:101970001B0280916E0A9927AA27BB2780932B020E
:1019800090932C02A0932D02B0932E028091700AA6
:101990009927AA27BB2780933E0290933F02A093EA
:1019A0004002B09341028091710A9091720AB8018D
:1019B0000E94CB9CCB01AA27BB2780935102909316
:1019C0005202A0935302B09354028091730A9091F3
:1019D000740AAA2797FDA095BA2F8093640290936A
:1019E0006502A0936602B093670280915205992721
:1019F000AA27BB278093770290937802A09379025D
:101A0000B0937A02809127059927AA27BB27809354
:101A10008A0290938B02A0938C02B0938D028091E6
:101A200028059927AA27BB278093B0029093B1027B
:101A3000A093B202B093B3021F910F9108950024B6
:101A400022273327442751E0BB27EE27FF27A0E1B9
:101A5000660F771F881F991F001C221F331F441F0A
:101A6000660F771F881F991F001C221F331F441FFA
:101A70002AF4050E2B1F3E1F4F1F04C0051A2B0B07
:101A80003E0B4F0B550FBB1FEE1F587F556047FD98
:101A90005250AA95E9F6E695B7955795E695B7950C
:101AA0005795852F9B2F08952227332741E05527EF
:101AB00068E0880F991F221F331F880F991F221F6C
:101AC000331F1AF4240F351F02C0241B350B440F9B
:101AD000551F487F456037FD42506A9551F756952E
:101AE000479556954795842F0895AA2797FF04C0D8
:101AF000809590958A1F9A1F77FF04C06095709516
:101B00006A1F7A1F669F9001779FA001679F300D23
:101B1000411D5A1F300D411D5A1F889FF001999F8A
:101B20002E0F3F1F401D511D899F300D411D5A1F13
:101B3000300D411D5A1FCA01B901112480CF4FB782
:101B400020E430E0F8948091C9008F778093C90039
:101B50008091C9008F7B8093C9008091C9008F7DDF
:101B60008093C900832F99278093CD002093CC00C8
:101B70008091C80082608093C80088E18093C9008A
:101B80008091CA008F778093CA008091CA008F7BB2
:101B90008093CA008091CA008F7D8093CA00809193
:101BA000CA008F7E8093CA008091CA00877F80938D
:101BB000CA008091C9008B7F8093C9008091CA00C0
:101BC00084608093CA008091CA0082608093CA00BA
:101BD0008091C80087FF03C08091CE00F9CF80912B
:101BE000C90080688093C9004FBF08950F931F9369
:101BF000CF93DF93482F4F5F893108F08BC08091DE
:101C00007309841720F44F5F409373094150CB014F
